:020000040800F2
:10000000809F012061020008C1360008072E000809
:10001000BD3600086F040008C53B00080000000062
:10002000000000000000000000000000A101000826
:100030007304000800000000FD01000809380008F2
:100040007B0200087B0200087B0200087B0200089C
:100050007B0200087B0200087B0200087B0200088C
:10006000E90A00087B0200087B0200087B02000806
:100070007B0200087B0200087B0200087B0200086C
:100080007B0200087B0200087B0200087B0200085C
:100090007B0200087B0200087B0200087B0200084C
:1000A0007B0200087B0200087B0200087B0200083C
:1000B0007B0200087B020008013900087B0200086F
:1000C0007B0200087B0200087B0200087B0200081C
:1000D0007B0200087B0200087B0200087B0200080C
:1000E0007B0200087B0200087B0200087B020008FC
:1000F0007B0200087B0200087B0200087B020008EC
:100100007B0200087B0200087B0200087B020008DB
:100110007B0200087B0200087B0200087B020008CB
:100120007B0200087B0200087B0200087B020008BB
:100130007B020008810500087B0200087B020008A2
:100140007B0200087B0200087B0200087B0200089B
:100150007B0200087B0200087B0200087B0200088B
:100160007B0200087B0200087B0200087B0200087B
:100170007B0200087B0200087B02000800000000F0
:100180007B0200087B020008DFF810D000F032F993
:100190000048004789760008AFF30080809F012067
:1001A0002C4B19680868B0E8F04F80F30988BFF35A
:1001B0006F8F4FF0000080F311887047000000003F
:1001C00008480068006880F308884FF0000080F35A
:1001D000148862B661B6BFF34F8FBFF36F8F00DF35
:1001E00000BF00BF08ED00E0DFF80C00016841F43B
:1001F00070010160704700BF88ED00E0EFF30980F7
:10020000BFF36F8F134B1A681EF0100F08BF20ED5D
:10021000108A20E9F04F106009B44FF0500080F3CD
:100220001188BFF34F8FBFF36F8F12F017FF4FF09E
:10023000000080F3118809BC19680868B0E8F04F25
:100240001EF0100F08BFB0EC108A80F30988BFF3CE
:100250006F8F704750C00120EFF30580704700009A
:100260000648804706480047FEE7FEE7FEE7FEE750
:10027000FEE7FEE7FEE7FEE7FEE7FEE7ED380008F3
:10028000890100082DE9F05F0546002092469B4653
:1002900088460646814640241BE02846414647469C
:1002A000224600F097F853465A46C01A914110D39F
:1002B00011461846224600F07EF82D1A67EB010819
:1002C0004F4622460120002100F075F817EB000987
:1002D0004E41201EA4F10104DFDC484631462A4687
:1002E0004346BDE8F09F00000649074A08685043AE
:1002F00043F2390210440860400870470149086021
:1003000070470000BC0000206D4EC64110B5431A76
:10031000934209D28318881803E010F8011D03F8EE
:10032000011D521EF9D210BD40EA01039B0703D004
:1003300009E008C9121F08C0042AFAD203E011F824
:10034000013B00F8013B521EF9D210BDD2B201E0D0
:1003500000F8012B491EFBD270470022F6E710B5CA
:1003600013460A4604461946FFF7F0FF204610BD23
:1003700030B504460020034600E05B1C934203D2E4
:10038000E05CCD5C401BF8D030BD30B50B4601467B
:1003900000202022012409E021FA02F59D4205D324
:1003A00003FA02F5491B04FA02F52844151EA2F1CE
:1003B0000102F1DC30BD202A04DB203A00FA02F110
:1003C000002070479140C2F1200320FA03F3194343
:1003D00090407047202A04DB203A21FA02F00021E5
:1003E000704721FA02F3D040C2F120029140084345
:1003F00019467047064C074D06E0E06840F00103DF
:1004000094E8070098471034AC42F6D3FFF7C0FEDB
:10041000E44501082446010870B58C1810F8015B0A
:1004200015F0070301D110F8013B2A1106D110F88D
:10043000012B03E010F8016B01F8016B5B1EF9D191
:100440002B0705D40023521E0DD401F8013BFAE717
:1004500010F8013BCB1A921C03E013F8015B01F882
:10046000015B521EF9D5A142D8D3002070BD00BF58
:10047000FEE7704710B50146002226E002EB820439
:100480000B6903EBC4000023036043608360C36017
:10049000036243624FF0004303604FF48C434360B8
:1004A000436823F00043436001F1480343F822000E
:1004B000032A07D202EB82040B6903EBC40328333F
:1004C000C36001E00B69C360521C042AD6D3002428
:1004D000CC650C668C66CC668C650B6803F5805326
:1004E0000C69DC6010BD10B50146002222E002EB71
:1004F0008204CB6803EBC400002303604360836085
:10050000C36001F1180343F82200036843F4801329
:100510000360032A07D202EB8204CB6803EBC40317
:100520002833C36001E0CB68C360036843F4400331
:100530000360521C042ADAD300248C620B6803F592
:100540008053CC681C6110BD38B504460020009073
:10055000206800F58050806940F48011206800F523
:1005600080508161206800F58050806900900120F2
:1005700000F040FB0099206800F58050816138BD93
:1005800010B5024800F0D2FB10BD00006C4C0020FA
:1005900030B503461479557944EA0520084C0C44DB
:1005A0002064D4782406957844EA0544557844EAD2
:1005B0000524157844EA0500014C0C44606430BD04
:1005C0000080024010B5A4B0044601208DF83C0024
:1005D0008DF83D0000200D908DF84B0001208DF826
:1005E0004A0000208DF8480001208DF830000020DE
:1005F0008DF84C008DF83B0014908DF854001D9040
:100600008DF878001F908DF882008DF880004FF4EF
:1006100080401090C010119000208DF881000BA92F
:10062000204600F095F901208DF80C008DF80D00A2
:100630008DF81D008DF80E00002005908DF81C002F
:100640008DF81E00089001208DF824008DF804001C
:1006500000040290800106904012049001208DF861
:10066000250000200A9000906946204600F010F90D
:1006700024B010BD0020704710B501F06BF910BD1B
:1006800010B5024800F054FE002010BD6C4C002054
:1006900070B504460D46164633462A4621460448A0
:1006A00000F078FD10B14FF0FF3070BD0020FCE786
:1006B0006C4C002070B504460D46164633462A465B
:1006C0002146044800F091FF10B14FF0FF3070BD9B
:1006D0000020FCE76C4C00202DE9F04F80460C46D2
:1006E000164608F118031A69D3F810904FF0000C61
:1006F00053F82210A568E246086800F00040B0F107
:10070000004F04D003F1140050F8220010B1022071
:10071000BDE8F08F0CF1010C2868886048686FF321
:100720000C00D5F804B040EA0B004860207800F0D7
:10073000010038B1086820F44000D4F814B040EA51
:100740000B000860207800F0200038B1086820F025
:100750004060D4F810B040EA0B000860207800F048
:10076000040018B1086840F080000860086840F094
:100770008050086000BF00BF00BFBFF35F8F00BFA5
:1007800000BF00BF086840F0004008605DE00868F6
:1007900020F00050086026B1086840F080400860F2
:1007A00003E0086820F08040086000BF521C042A63
:1007B00000D3121F00BF53F82210086820F08050A9
:1007C0000860086800F00040B0F1004F04D003F169
:1007D000140050F82200E8B14A4653F822100027CE
:1007E00014E000BF00BF00BFBFF35F8F00BF00BFBA
:1007F00000BF086820F00040086000BF521C042AB7
:1008000000D3121F00BF53F822107F1C6745E8D3A6
:1008100002207DE70CF1010CAD682868886048680B
:100820006FF30C00D5F804B040EA0B0048600AF101
:10083000010A00BF00BF00BFBFF35F8F00BF00BF52
:1008400000BF086840F000400860A86800289ED1FA
:1008500026B1086840F08040086003E0086820F096
:1008600080400860086840F00050086003F1140000
:10087000D3F824B040F822B01A6172B60AF1010030
:10088000D3F828B05844986262B6002040E70000D0
:1008900070B505460C46286800F5805086692B48DF
:1008A0000640207B08B9012000E000208006617B23
:1008B00040EA4160617F09B9012100E0002140EA7E
:1008C0000150A17B40EA415061690843217F40EA21
:1008D000C110A17F40EA8110216A084394F82410D6
:1008E00040EA81000643286800F580508661286848
:1008F00000F580508669012000F07CF9286800F539
:10090000805086612179A06840EA4160A16908436E
:100910002169084394F8251040EAC110A16A40EA11
:1009200081002168084340F40001286800F58050E8
:100930000160286800F580500668012000F05AF92F
:10094000286800F58050066070BD0000233FDEF887
:1009500070B505460C46286806683A480640207C73
:1009600008B9012000E00020C005617C09B901211F
:1009700000E0002140EA8150A1680843E17F40EA9D
:10098000014061690843A17F09B9012100E000210C
:1009900040EA4130217F40EA0130A16908432179D2
:1009A00040EA812094F8201009B9012100E00021DB
:1009B00040EA4120E17B40EAC110616A084394F8B3
:1009C000281040EA01100643286806602868066877
:1009D000012000F00FF928680660286886694FF644
:1009E00041700640A06C000494F84C1009B9012134
:1009F00000E0002140EAC110216D084394F8551031
:100A0000012900D100E0002140EAC10094F856100D
:100A1000012900D100E0002140EA810094F854103F
:100A2000012900D100E0002140EA41000643286886
:100A3000866128688669012000F0DCF828688661F4
:100A400070BD00000F8120FF2DE9F843044600200F
:100A500000904FF00108A66E04F1480050F82650AF
:100A6000E76E2FE0286A58B9684600F005FC009848
:100A700010B94FF0000803E0009828620098A860C1
:100A8000B8F1000F1ED0A06D10B91648686002E0E2
:100A90004FF48C40686000BF00BF00BFBFF35F8FA2
:100AA00000BF00BF00BF286840F00040286000BFC2
:100AB000761C042E00D3361F00BF04F1480050F806
:100AC00026507F1E17B1B8F1000FCBD1E06EB842AF
:100AD00006D00021206800F580508160A666E76698
:100AE000BDE8F8830046008010B5042000F024FE25
:100AF00010BD704770B50446B3F5804F13D1D1E9EE
:100B0000000540EA05108D6840EA05208D692843FC
:100B10008D8940EA054054F82250064E354028435E
:100B200044F8220003E06FF0704044F822000020F7
:100B300070BD00000000F0CF70B50246086852F8A2
:100B4000200020F001000E6842F82600886808287E
:100B500001D1402300E00023486818438E683043E9
:100B6000CE6830430E6930434E693043CE6930431E
:100B70000E6A30434E6A30438E6A3043CE6A304349
:100B80000E6B40EA060488690443C86B0443074DB2
:100B900045F4806545F4E025086852F82000A84334
:100BA00020430E6842F82600002070BD7FFB08003D
:100BB00010B50346D1E9000440EA04108C6840EA0D
:100BC00004208C8940EA0444088A401E44EA005408
:100BD000087D801E44EA00608C692043541C53F851
:100BE000244004F040442043541C43F824000020D7
:100BF00010BD000070B5044600F0ACFE0646254668
:100C0000681C10B104480078054400BF00F0A2FE43
:100C1000801BA842FAD370BD10C0012010B5044655
:100C2000204600F00BF800F08000802803D1024835
:100C3000006808F023F810BD1CC001200146D1F85F
:100C40008C007047024609B901207047106800689F
:100C5000C0F3001081F828001068006800F0600000
:100C6000486210680068C0F3402080F0010081F8FD
:100C7000200010680068C0F30040C8771068006862
:100C8000C0F3403080F00100887710680068C0F33E
:100C9000003008771068006800F400608861106810
:100CA000006800F48040486110680068C0F380501C
:100CB00080F00100487410680068C0F3C05080F0F4
:100CC0000100087410680068C0F3C010C873106891
:100CD000006800F46020886010680068C0F380201D
:100CE000087110688069C0F3400081F854001068F2
:100CF0008069C0F3C01080F0010081F84C001068DA
:100D0000806900F03000086510688069000C886414
:100D100010688069C0F3800081F85600106880690F
:100D2000C0F3C00081F8550000208EE710B50446DE
:100D3000206800F58050406900F0400040280FD145
:100D4000206800F58050C06900F04000402807D1BD
:100D50004249206800F580504161204600F0B0FA19
:100D6000206800F58050406900F0010078B12068EB
:100D700000F58050C06900F0010040B14FF0011152
:100D8000206800F580504161204600F01DFC20687D
:100D900000F58050406900F40040B0F5004F3DD1AF
:100DA000206800F58050C06900F40040B0F5004FA5
:100DB00034D1D4F8880040F00800C4F888002068D6
:100DC00000F58050406900F40050B0F5005F15D187
:100DD000206800F58050406921490840C4F88C0023
:100DE000206800F58050C06920F4C031206800F50B
:100DF0008050C161E020C4F884000CE0206800F558
:100E00008050406948F280610840C4F88C00206836
:100E100000F5805041612046FFF700FF2068806B9D
:100E200000F0080008280BD12068C06A00F06000BC
:100E3000C4F89400204600F02BF90020C4F8940078
:100E40000848006800F4002030B14FF40020054944
:100E50000860204600F0C8FB10BD00004000010003
:100E600000207E00143C014038B504460CB9012036
:100E700038BDD4F8840028B92320C4F88400204663
:100E800000F05CF800BF002000902A48006840F4A1
:100E90008040284908600846006800F480400090BF
:100EA00000BF00BF2448006820F400002249086009
:100EB00008460068A16808431F49086008460068A2
:100EC000206800F58050006840F00101206800F5BE
:100ED0008050016000F03EFD05460DE000F03AFD57
:100EE000401BB0F5FA7F07D90420C4F88800E02041
:100EF000C4F884000120BBE7206800F5805000683A
:100F000000F001000028E9D12046FFF75BFB2046F6
:100F1000FFF7E9FA2046FFF7ADFA002120466268A4
:100F2000FFF736FB0020C4F888001020C4F88400C6
:100F300000209DE7443802400438014010B586B0D7
:100F40000446142101A8FFF708FA4C49206888429A
:100F50007ED100BF00BF002000904948006840F0EB
:100F60000070474908600846006800F00070009073
:100F700000BF00BF00BF002000900846006840F09E
:100F8000806008600846006800F08060009000BF44
:100F900000BF00BF002000900846006840F00060DD
:100FA00008600846006800F00060009000BF00BFC5
:100FB00000BF00BF002000900846006840F0040019
:100FC00008600846006800F00400009000BF00BF01
:100FD00000BF002000900846006840F00100086053
:100FE0000846006800F00100009000BF00BF00BF8D
:100FF000002000900846006840F0020008600846A3
:10100000006800F00200009000BF00BF3220019095
:101010000220029000200390032004900B200590F2
:1010200001A9184800F096FB86200190022002904A
:1010300000200390032004900B20059001A9124882
:1010400000F088FB4FF4605001900220029000E015
:1010500011E000200390032004900B20059001A9CB
:101060000A4800F077FB002205213D2000F048FDF2
:101070003D2000F035FD06B010BD000000800240AC
:1010800030380240000802400000024000040240E4
:1010900070472DE9F05F04460F464FF00008C34645
:1010A00047B9D4F8880040F00100C4F88800012056
:1010B000BDE8F09FD4F88400232801D00120F7E791
:1010C000E66D04F1480050F82650E06EC0F10409C6
:1010D00042E0286800F4807018B1A969A167E96945
:1010E0006167286800F4007008B9E06F40B32868B1
:1010F00000F4007010B1002121666166D4F814A0DC
:10110000286800F4807040B12868C0F30D40A0F159
:10111000040A296821674FF0010BA86828621FFAAA
:101120008AF304F18001081F2A6A00F0D3F8206EC8
:10113000401C2066606E00EB0A0161660020286298
:1011400000BF761C042E00D3361F00BF04F14800F8
:1011500050F8265008F10108286800F0004020B936
:10116000C84502D2BBF1000FB3D0E06E00EB08011E
:10117000E166E06E10B12046FFF766FCE665BBF164
:10118000010F05D1E06F38600021E16700208FE793
:1011900001208DE72DE9F04705460E461746984693
:1011A0002868046904F01C044FF4784000EAC62063
:1011B00004434FF4F86000EA8710044324F002046B
:1011C00044F001042868046100F0C4FB81460BE090
:1011D00000F0C0FBA0EB0900B0F5803F02D3012076
:1011E000BDE8F0872868046904F001000028EFD109
:1011F0002868406980B2C8F800000020F0E72DE9B7
:10120000F047064606F11804A76AE56A4FF00108A0
:101210002AE04FF001097F1E04F1140050F8250068
:1012200020B9681C00F003054FF00009B9F1000F68
:101230001AD005EB8501F06850F8310000F000404D
:1012400080B904F1140151F8250000F0C7F900211C
:1012500004F1140040F82510681C00F00305A76293
:10126000E56201E04FF0000817B1B8F1000FD0D1EE
:101270000020BDE8F08700007CB504460D4806F06C
:1012800087FF054685B105F1200020600A482861E6
:101290004FF4C06120682B464122CDE900010021B6
:1012A000084607F0A1FF04E001200449087000206F
:1012B00020607CBD9C4201086199000818C0012093
:1012C00010B504460248006807F0D8FC10BD0000C5
:1012D0001CC00120F0B504460D4621462E460020D4
:1012E000A2F1200000270760078143810F680FB932
:1012F000086001E0376838603060086803E00789FB
:101300001F44078100680028F9D1F0BD70B504467C
:101310000D460DB9012070BDD4F88400102805D108
:1013200029462046FFF714FB0020F4E70120F2E7EE
:1013300070B506463068056925F01C0500F016FDFD
:1013400004461348844205D31248844202D245F031
:1013500008051AE00F48844205D30F48844202D2A0
:1013600045F00C0511E00C48844203D30B4884423D
:1013700000D20AE00948844205D30948844202D2D7
:1013800045F0040501E045F010053068056170BDC9
:10139000002D3101C00E16020087930300E1F50510
:1013A00080D1F00870B50446D4F8840010285FD1CD
:1013B0002320C4F884000121A1652068C06B40F49B
:1013C00002702168C8632068D0F80C0129490843DD
:1013D0002168C1F80C012068D0F8100140F4031016
:1013E0002168C1F810010421E1662046FFF72CFBBB
:1013F0002068006840F008002168086020680568DF
:101400000120FFF7F7FB206805602068006840F0C6
:10141000040021680860206805680120FFF7EAFBE6
:10142000206805602046FFF78FF8206800F580509F
:10143000806940F40051206800F580508161206887
:1014400000F58050806940F00201206800F580506E
:101450008161206800F58050C06907490843216810
:1014600001F58051C8612320C4F88400002070BDBC
:101470000120FCE760000200C1A001002DE9F0415D
:101480000446D4F88400232851D1C4F8840020688D
:1014900000F58050C06927490840216801F5805156
:1014A000C861206800F58050806920F400512068F0
:1014B00000F580508161206800F58050806920F03F
:1014C0000201206800F5805081612068006820F0EA
:1014D000040021680860206807680120FFF78AFB84
:1014E000206807602046FFF72FF82068006820F08A
:1014F000080021680860206807680120FFF77AFB70
:1015000020680760002508E004F1480050F82560D5
:10151000706840F0004070606D1C042DF4D3002111
:10152000A1651020C4F884000020BDE8F0810120EE
:10153000FBE700003E5FFEFF70B504460D463DB977
:10154000D4F8880040F00100C4F88800012070BD84
:10155000D4F88400232835D1696BE1630122294640
:101560002046FFF7B9F838B1D4F8880040F00200FF
:10157000C4F888000120EAE700BF00BF00BFBFF346
:101580004F8F00BF00BF00BF00BFA06A401CA06219
:10159000A06A042802D3A06A001FA06200BF2068CE
:1015A00000F58050406900F0040048B10421206833
:1015B00000F5805041610021206800F580504160B5
:1015C0000020C4E70120C2E710B5044602480068C5
:1015D00007F054FB10BD000020C0012010B50446E8
:1015E000204608F0E9F810BD70472DE9F0470546A0
:1015F0000E46174698462868046904F01C044FF408
:10160000784000EAC62004434FF4F86000EA8710EF
:10161000044344F0020444F001041FFA88F02968EE
:1016200048612868046100F095F981460BE000F0FC
:1016300091F9A0EB0900B0F5803F02D30120BDE88D
:10164000F0872868046904F001000028EFD100BF8A
:10165000F5E7000000B587B0142102A8FEF77DFE73
:101660002A48006808B107B000BD0120274908607A
:1016700000BF002001902648006840F00100244986
:1016800008600846006800F00100019000BF00BF3C
:1016900043F23F00029002200390002004900320B8
:1016A00005900C20069002A91A4800F053F84FF458
:1016B000F060029002200390002004900320059027
:1016C0000C20069002A9144800F044F84CF2B30034
:1016D00002900220039000200490032005900C202B
:1016E000069002A90D4800F035F84FF40070029002
:1016F0000220039000200490032005900C20069007
:1017000002A9074800F026F800BFACE700C001209E
:10171000383802400014024000100240000C024021
:101720000018024010B50446042C03D102F0C0FB9F
:1017300002F04EFC10BD000010B5044604480068DD
:10174000204020B1024804602046FFF7EBFF10BDA7
:10175000143C0140F8B502460B4600250024002049
:101760000021D6E0012606FA01F51E6806EA050406
:10177000AC4274D11E7906F00306012E04D01E7906
:1017800006F00306022E13D190684F000326BE40D8
:10179000B0434F00DE68BE40304390605068012681
:1017A0008E40B0431E79C6F300168E403043506021
:1017B0001E7906F00306032E09D0D0684F000326D9
:1017C000BE40B0434F009E68BE403043D0601E799B
:1017D00006F00306022E13D1CF0802F1200656F8B8
:1017E00027004E07F70E0F26BE40B0434F07FF0EEF
:1017F0001E69BE403043CF0802F1200646F827009C
:1018000010684F000326BE40B0431E7906F0030661
:101810004F00BE40304310605E6806F44036002E34
:1018200076D000BF002600963C4E366846F48046CF
:101830003A4F3E603E46366806F48046009600BF4A
:1018400000BF374E8F0856F827008E07370F0F2638
:10185000BE40B043334EB24202D1002624E057E0EE
:10186000314EB24201D101261EE0304EB24201D1CA
:10187000022619E02E4EB24201D1032614E02D4E6D
:10188000B24201D104260FE02B4EB24201D105260F
:101890000AE02A4EB24201D1062605E0284EB242A5
:1018A00001D1072600E008268F073F0FBE403043D6
:1018B0001B4E8F0846F82700224E3068A0435E6812
:1018C00006F4801606B120431E4E3060361D306887
:1018D000A0435E6806F4001606B12043194E361D7B
:1018E0003060184E361F3068A0435E6806F400363C
:1018F00006B12043134E361F3060361F3068A043B8
:101900005E6806F4803606B120430E4E083E306015
:10191000491C1029FFF426AFF8BD000044380240EE
:101920000838014000000240000402400008024064
:10193000000C024000100240001402400018024057
:10194000001C0240083C01400AB1816101E00B0427
:1019500083617047014800687047000008C001209B
:101960000148006870470000107AFF1F01480068B6
:1019700070470000147AFF1F01480068704700009C
:10198000187AFF1F03480068034909780844014991
:101990000860704708C0012010C0012010B50D4834
:1019A000006840F400700B4908600846006840F485
:1019B000806008600846006840F48070086003207A
:1019C00000F0DCF80F2000F007F800F05FF80020CE
:1019D00010BD0000003C02402DE9F04188B00446F3
:1019E0000027B84600BF002001902348006840F05F
:1019F0000400214908600846006800F004000190D6
:101A000000BF00BF02A903A800F08EF9069F1FB90E
:101A100000F0B2F9054602E000F0AEF945001748C3
:101A2000B5FBF0F0A0F1010815481649086040F236
:101A3000E7311448C160C0F8048000210161816071
:101A4000816100F0F9FE064696B90E4800F028FFC5
:101A500006466EB91E2000F043F8102C07D2002273
:101A600021461E2000F04CF80748046000E00126E3
:101A7000304608B0BDE8F0814038024040420F00D7
:101A800000080040600100200CC0012008B500BF24
:101A9000002000901148006840F480400F49086021
:101AA0000846006800F48040009000BF00BF00BFFF
:101AB00000200090081F006840F08050091F086057
:101AC0000846006800F08050009000BF00BF002270
:101AD0000F21901E00F014F808BD000044380240A9
:101AE00001460846002809DB00F01F0301229A4046
:101AF00043099B0003F1E023C3F8002100BF7047B6
:101B00002DE9F05F80460D461646002702F06CF87E
:101B1000074639462A46334601F00700C0F1070A56
:101B2000BAF1040F02D94FF0040A01E0C0F1070A2C
:101B3000D14600F1040ABAF1070F02D24FF0000AB1
:101B400001E0A0F1030AD4464FF0010A0AFA09FAAB
:101B5000AAF1010A0AEA020A0AFA0CFA4FF0010B8A
:101B60000BFA0CFBABF1010B0BEA030B4AEA0B047B
:101B70002146404602F040F8BDE8F09F00BF00F06B
:101B80000702064B19684FF6FF031940044B0B433D
:101B900043EA0221014B196000BF70470CED00E0E1
:101BA0000000FA0570B504460D460CB9012070BD61
:101BB0005848006800F00700A84209D255490D7046
:101BC0000846006800F00700A84201D00120EEE7B7
:101BD000207800F0020002281DD1207800F00400D7
:101BE000042805D14C48006840F4E0504A49086098
:101BF000207800F00800082805D14748006840F424
:101C00006040454908604448006820F0F000A16841
:101C1000084341490860207800F00100A8B36068DB
:101C2000012807D13C4808380068C0F34040B8B9E3
:101C30000120BCE76068022802D06068032807D151
:101C4000354808380068C0F3406048B90120AEE765
:101C5000314808380068C0F3400008B90120A6E701
:101C60002D48006820F00300616808432A49086095
:101C7000FFF770FE064609E0FFF76CFE801B41F29D
:101C80008831884202D9032091E707E022480068A2
:101C900000F00C006168B0EB810FEDD11D480068C9
:101CA00000F00700A84209D91A490D7008460068DB
:101CB00000F00700A84201D0012078E7207800F06A
:101CC0000400042807D11448006820F4E050E168BB
:101CD000084311490860207800F00800082808D15E
:101CE0000D48006820F46040216940EAC1000A49BB
:101CF000086000F051F808490968C1F30311074A68
:101D0000515CC8400649086006480068FFF764FE59
:101D100000204CE7003C02400838024084420108A1
:101D20000C0000200CC001200F2202600D4A126836
:101D300002F0030242600B4A126802F0F002826075
:101D4000084A126802F4E052C260064A126802F4BD
:101D50006042D2080261044A126802F007020A6077
:101D60007047000008380240003C0240014800680B
:101D7000704700000C00002000B5FFF7F7FF044992
:101D80000968C1F38221034A515CC84000BD0000CC
:101D900008380240944201082DE9F047002400254C
:101DA0000026A1462548006800F00C0020B1042858
:101DB00005D008283AD105E0DFF8849039E0DFF853
:101DC000849036E01D48001F006800F03F041B4867
:101DD000001F006800F4800078B11A481749091FF5
:101DE0000968C1F38811A0FB017001462246002357
:101DF0003846FEF747FA05460EE011480F49091F1D
:101E00000968C1F38811A0FB017001462246002336
:101E10003846FEF737FA05460848001F0068C0F349
:101E20000140401C4600B5FBF6F902E0DFF81090D7
:101E300000BF00BF4846BDE8F087000008380240F8
:101E40000024F40000C0A800F8B504460CB9012035
:101E5000F8BD207800F00100002874D0F94800682F
:101E600000F00C0004280DD0F648006800F00C00CB
:101E7000082813D1F348001F006800F48000B0F573
:101E8000800F0BD1EF4808380068C0F340400028AD
:101E900059D06068002856D10120D9E700BF60689A
:101EA000B0F5803F08D1E7480838006840F480303A
:101EB000E449083908601EE06068B0F5A02F0DD134
:101EC000E0480838006840F48020DE49083908609E
:101ED0000846006840F4803008600CE0D9480838B3
:101EE000006820F48030D749083908600846006847
:101EF00020F48020086000BF606890B1FFF72AFDE1
:101F0000054606E0FFF726FD401B642801D90320A3
:101F10009EE7CC4808380068C0F340400028F1D064
:101F200011E0FFF717FD054606E0FFF713FD401B24
:101F3000642801D903208BE7C24808380068C0F341
:101F400040400028F1D1207800F0020002285FD143
:101F5000BC48006800F00C0058B1BA48006800F0B6
:101F60000C0008281CD1B748001F006800F480004E
:101F7000B0B9B44808380068C0F3400020B1E06848
:101F8000012801D0012063E7AE480838006820F03E
:101F9000F800216940EAC100AA490839086037E021
:101FA000E06800B30120A8490860FFF7D3FC0546AC
:101FB00006E0FFF7CFFC401B022801D9032047E7CA
:101FC000A04808380068C0F340000028F1D09D48C0
:101FD0000838006820F0F800216940EAC1009949FA
:101FE0000839086014E0002097490860FFF7B2FC48
:101FF000054606E0FFF7AEFC401B022801D903208E
:1020000026E7904808380068C0F340000028F1D166
:10201000207800F0080008282CD16069A8B10120C0
:102020008A490860FFF796FC054606E0FFF792FC38
:10203000401B022801D903200AE782486C3000685F
:10204000C0F340000028F1D014E000207F49086070
:10205000FFF780FC054606E0FFF77CFC401B0228EA
:1020600001D90320F4E677486C300068C0F34000E3
:102070000028F1D1207800F00400042870D1002756
:1020800070483830006800F0805090B900BF0020E0
:1020900000906C483830006840F080506949383111
:1020A00008600846006800F08050009000BF00BF44
:1020B00001276748006800F48070B0B96448006880
:1020C00040F4807062490860FFF744FC054606E072
:1020D000FFF740FC401B022801D90320B8E65C480A
:1020E000006800F480700028F2D000BFA0680128CA
:1020F00008D154486830006840F001005149683107
:1021000008601DE0A06805280DD14E4868300068C1
:1021100040F004004B49683108600846006840F010
:10212000010008600CE047486830006820F00100BA
:102130004449683108600846006820F004000860DF
:1021400000BFA068A8B1FFF705FC054609E0FFF74E
:1021500001FC401B41F28831884202D9032077E616
:1021600026E0384868300068C0F340000028EED010
:1021700013E0FFF7EFFB054608E0FFF7EBFB401B22
:1021800041F28831884201D9032061E62D48683048
:102190000068C0F340000028EFD1012F07D1294883
:1021A0003830006820F0805026493831086000BF80
:1021B000A069002845D02348006800F00C000828DA
:1021C0005DD0A069022845D100201F490866FFF7AD
:1021D000C1FB054606E0FFF7BDFB401B022801D905
:1021E000032035E6174808380068C0F3406000282F
:1021F000F1D1D4E907010843616A40EA8111012263
:10220000A06AC2EB500041EA00412C20005D41EA87
:1022100000600C49091F086001200B490866FFF7A0
:1022200099FB054606E0FFF795FB401B022801D904
:1022300003200DE6034808380068C0F3406000281A
:10224000F1D049E00838024000004742800E474282
:1022500000700040002021490866FFF77BFB05461F
:1022600006E0FFF777FB401B022801D90320EFE5CA
:102270001B480068C0F340600028F2D12CE0A06940
:10228000012800D1E4E51648001D0668A069012870
:1022900020D006F48001E06981421BD106F03F01A5
:1022A000206A814216D147F6C0703040616AB0EBB7
:1022B000811F0FD106F440310122A06AC2EB500009
:1022C000B1EB004F06D106F070612C20005DB1EB40
:1022D000006F01D00120BBE50020B9E500004742B6
:1022E0000038024010B504460CB9012010BD606AE8
:1022F00038B96068B0F5827F00D105E00021E16166
:1023000002E00021216161610021A16294F8510085
:1023100028B9002084F85000204600F047F8022039
:1023200084F851002068006820F0400021680860AF
:10233000A08800F48270218901F404410843A18936
:1023400001F400610843217C01F002010843217D72
:1023500001F001010843218B01F400710843217F42
:1023600001F0380108432021095D01F08001084394
:10237000218D01F400510843216808600421A069FF
:1023800001EA104094F8241001F01001084321687C
:1023900048602068C06920F400602168C86100209E
:1023A0006065012084F8510000209FE710B586B0D9
:1023B0000446142101A8FDF7D0FF1B49206888427C
:1023C0002FD100BF002000901848006840F48050D2
:1023D000164908600846006800F48050009000BF6D
:1023E00000BF00BF0020009010481438006840F083
:1023F00002000E49143908600846006800F0020027
:10240000009000BF00BF3820019002200290002001
:102410000390032004900520059001A90448FFF7CC
:1024200099F906B010BD0000003001404438024068
:10243000000402402DE9FF5F0446884691461D4690
:102440000E9E012002900020019000BF94F85000E1
:10245000012803D1022004B0BDE8F09F012084F8D8
:10246000500000BFFFF776FA074694F851B0606855
:102470000390AA46BBF1010F0BD00398B0F5827F01
:1024800004D1A06810B9BBF1040F02D00220019062
:10249000DBE0B8F1000F03D0B9F1000F00D015B99F
:1024A00001200190D1E094F85100042802D00520C9
:1024B00084F8510000206065C4F83890E587A5874E
:1024C000C4F83080E586A5862064606420680068D2
:1024D00000F04000402805D02068006840F040002F
:1024E00021680860E068B0F5006F4AD1606810B1FB
:1024F000BAF1010F09D1206B00882168C860206BF8
:10250000801C2063E08E401EE08633E020688068F7
:1025100000F00200022810D1E08E70B1029801286C
:102520000BD1206B00882168C860206B801C206361
:10253000E08E401EE086002002902068806800F057
:10254000010068B1E08F58B12068C068A16B0880B5
:10255000A06B801CA063E08F401EE08701200290EA
:10256000FFF7F8F9C01BB04204D3701C10B1032070
:1025700001906AE0E08E0028C8D1E08F0028C5D124
:102580004AE0606810B1BAF1010F09D1206B007800
:1025900021680873206B401C2063E08E401EE0869B
:1025A00034E02068806800F00200022810D1E08E3C
:1025B00070B1029801280BD1206B00782168087354
:1025C000206B401C2063E08E401EE08600200290BD
:1025D0002068806800F0010068B1E08F58B1206881
:1025E000C068A16B0870A06B401CA063E08F401E08
:1025F000E08701200290FFF7ADF9C01BB04201D384
:10260000701C00B916B9032001901EE0E08E00286E
:10261000C7D1E08F0028C4D13A463146204601F0A8
:1026200051F820B101200190202060650DE0A068E4
:1026300050B900BF002000902068C068009020685A
:102640008068009000BF00BF00BF012084F85100E7
:1026500000BF002084F8500000BF0198FBE670B571
:1026600004460E4615460CB9012070BD94F8490089
:1026700028B9002084F84800204600F01FF804F133
:1026800008012068FEF758FA3146A2682068FEF774
:102690008FFA2946236BD4E90102FEF72BFAA168D1
:1026A000206850F8210040F00100A268216841F83C
:1026B0002200012084F849000020D6E710B5044626
:1026C000FEF7C8FF10BDF0B504460D4616462F466E
:1026D000B44694F84920012A01D0042A1FD100BF32
:1026E00094F84800012801D10220F0BD012084F8AF
:1026F000480000BF022084F84900194606E03878F7
:102700008CF800000CF1010C7F1C491E0029F6D149
:1027100084F8492000BF002084F8480001E001202F
:10272000E3E70020E1E7F0B504460D462E461746E4
:1027300094F8490001281ED100BF94F848000128F0
:1027400001D10220F0BD012084F8480000BF022022
:1027500084F84900194604E0387830707F1C761CF4
:10276000491E0029F8D1012084F8490000BF00204B
:1027700084F8480001E00120E4E70020E2E7704728
:102780007047000030B502460B4600BF92F83C008F
:10279000012801D1022030BD012082F83C0000BF99
:1027A000022082F83D00106844681068816824F0B7
:1027B00070041868044310684460184D1068A842FB
:1027C0001BD01068B0F1804F17D0154D1068A8428B
:1027D00013D0144D1068A8420FD0134D1068A842B2
:1027E0000BD0124D1068A84207D0114D1068A842B6
:1027F00003D0104D1068A84205D121F0800158681F
:10280000014310688160012082F83D0000BF002074
:1028100082F83C0000BF00BFBDE70000000001409F
:102820000004004000080040000C0040000401408B
:10283000004001400018004010B504460CB90120CA
:1028400010BD94F83D0028B9002084F83C002046D3
:1028500000F025F8022084F83D00211D206801F0D9
:1028600057F8012084F8460000BF84F83E0001219B
:102870003F200155402001554120015500BF00BFB8
:10288000012084F842004320015544200155452091
:10289000015500BF012084F83D000020D0E77047BB
:1028A000014691F83D00012801D001207047022027
:1028B00081F83D000868C06840F001000B68D860EE
:1028C0001A4B086898421BD00868B0F1804F17D0A7
:1028D000174B0868984213D0164B086898420FD0DF
:1028E000154B086898420BD0144B0868984207D0E3
:1028F000134B0868984203D0124B086898420CD1D9
:102900000868806800F00702062A0CD00868006892
:1029100040F001000B68186005E00868006840F0AE
:1029200001000B6818600020C0E7000000000140B3
:102930000004004000080040000C0040000401407A
:102940000040014000180040704710B50446206860
:102950000069C0F34000D8B12068C068C0F34000EF
:10296000B0B16FF002002168086101202077206873
:10297000806900F0030018B12046FFF7E5FF05E08D
:10298000204600F0DDF8204600F0A8F9002020776E
:1029900020680069C0F38000D8B12068C068C0F327
:1029A0008000B0B16FF00400216808610220207738
:1029B0002068806900F4407018B12046FFF7C4FF1A
:1029C00005E0204600F0BCF8204600F087F9002022
:1029D000207720680069C0F3C000D8B12068C068C3
:1029E000C0F3C000B0B16FF0080021680861042096
:1029F00020772068C06900F0030018B12046FFF777
:102A0000A3FF05E0204600F09BF8204600F066F9A1
:102A10000020207720680069C0F30010D8B120683A
:102A2000C068C0F30010B0B16FF0100021680861F9
:102A3000082020772068C06900F4407018B1204653
:102A4000FFF782FF05E0204600F07AF8204600F00C
:102A500045F9002020772068006900F0010058B196
:102A60002068C06800F0010030B16FF001002168FB
:102A70000861204600F0BAF920680069C0F3C01070
:102A800058B12068C068C0F3C01030B16FF080004A
:102A9000216808612046FFF772FE20680069C0F3D4
:102AA000801058B12068C068C0F3801030B16FF05A
:102AB000400021680861204600F0A4F92068006900
:102AC000C0F3401058B12068C068C0F3401030B166
:102AD0006FF02000216808612046FFF751FE10BD0D
:102AE00010B586B00446142101A8FDF736FC206815
:102AF000B0F1804F1DD100BF002000900E4800684B
:102B000040F001000C4908600846006800F0010030
:102B1000009000BF00BF082001900220029000201A
:102B20000390032004900120059001A90348FEF7BB
:102B300011FE06B010BD0000303802400000024017
:102B400070472DE9F04104460D461646002700BFA8
:102B500094F83C00012802D10220BDE8F081012058
:102B600084F83C0000BF36B1042E1BD0082E31D0B3
:102B70000C2E5ED145E02946206800F047FF206812
:102B8000806940F00800216888612068806920F031
:102B900004002168886120688069296908432168E8
:102BA000886148E02946206800F068FF2068806955
:102BB00040F40060216888612068806920F48060AA
:102BC0002168886120688069296940EA01202168BC
:102BD000886130E02946206800F08EFF2068C069D7
:102BE00040F008002168C8612068C06920F0040036
:102BF0002168C8612068C069296908432168C861E3
:102C000019E02946206800F0B3FF2068C06940F44D
:102C100000602168C8612068C06920F48060216874
:102C2000C8612068C069296940EA01202168C8613B
:102C300001E0012700BF00BF00BF002084F83C0076
:102C400000BF384689E710B504460CB9012010BD15
:102C500094F83D0028B9002084F83C00204600F09C
:102C600025F8022084F83D00211D206800F050FE68
:102C7000012084F8460000BF84F83E0001213F2077
:102C80000155402001554120015500BF00BF0120E2
:102C900084F8420043200155442001554520015548
:102CA00000BF012084F83D000020D0E708B501688E
:102CB000B1F1804F0FD100BF002100910649096892
:102CC00041F00101044A11601146096801F0010157
:102CD000009100BF00BF08BD4038024070470000AF
:102CE00070B504460D4615B994F83E000BE0042D6E
:102CF00002D13F20005D06E0082D02D14020005D9A
:102D000001E04120005D012801D0012070BD1DB906
:102D1000022084F83E000EE0042D03D102213F2062
:102D2000015508E0082D03D102214020015502E0A1
:102D300002214120015501222946206800F054FE5D
:102D400023492068884203D022492068884201D163
:102D5000012000E0002028B12068406C40F40040D1
:102D6000216848641A49206888421BD02068B0F165
:102D7000804F17D018492068884213D0174920681F
:102D800088420FD01649206888420BD0114920682C
:102D9000884207D013492068884203D0124920682E
:102DA00088420CD12068806800F00706062E0CD0FF
:102DB0002068006840F001002168086005E0206894
:102DC000006840F001002168086000209EE70000D4
:102DD00000000140000401400004004000080040E1
:102DE000000C0040004001400018004010B50446AF
:102DF00003492068884201D1FEF7C4FD10BD0000E0
:102E000000080040704700BFFEE738B504460020C8
:102E100000906A460121636920689847002802DA19
:102E20006FF0040038BD6A46012163692068984745
:102E3000002802DA6FF00400F4E7009800F00400C4
:102E400008B90120EEE76A460021636920689847C7
:102E5000002802DA6FF00400E4E7009800F48050E4
:102E6000B0F5805F1FD0009800F40050B0F5005F0F
:102E700007D1009800F48070B0F5807F01D1022066
:102E8000D0E7009800F40050B0F5005F01D10320B6
:102E9000C8E7009800F48070B0F5807F01D104206D
:102EA000C0E70520BEE76A461F216369206898478E
:102EB000002802DA6FF00400B4E7009800F48050B4
:102EC00008B90620AEE7009800F01C00182801D1D0
:102ED0000220A7E7009800F01C00082801D1032079
:102EE000A0E7009800F01C00142801D1042099E705
:102EF000052097E7F8B5044600270020009000253C
:102F000000266068002855D1A06808B1A0688047F5
:102F100020202060002513E06A46122128466369BC
:102F20009847002802DA6FF0040608E0009800F0E5
:102F30001F00A84202D12560002603E000BF6D1CDF
:102F40001F2DE9D900BF20681F2801D96FF00206A4
:102F500056BB4FF40042002123692068984700289F
:102F600026DB6A46002163692068984700281CDB3D
:102F7000A0698047074612E0A0698047C01BB0F5F2
:102F8000FA7F09D86A4600216369206898470028BB
:102F900005DA6FF0040607E06FF0010604E0009820
:102FA00000F400400028E7D104E06FF0040601E0DF
:102FB0006FF003065EB9A0698047074600BFA069AD
:102FC0008047C01BB0F5FA6FF9D901206060304628
:102FD000F8BD02462AB1C86818B1886808B1086906
:102FE00010B94FF0FF307047086890604B68D360AD
:102FF000CB6853618B6813610B6993610020F2E722
:1030000000B595B01C2212490EA8FDF77FF90021EA
:103010000EA805F08FFE0F4908601C220C491C31D8
:1030200007A8FDF773F9002107A805F083FE0A49F8
:1030300008601C22064938316846FDF767F900210F
:10304000684605F077FE0549086015B000BD000030
:103050003042010800000020040000200800002089
:1030600000B587B01C216846FDF777F94FF0204086
:103070002E4908602E4848600020886000212B48B7
:10308000C160016141618161C161016241624FF4CE
:10309000805181620021C1620163416381634164A7
:1030A0000F20009001900A2002900F200390102022
:1030B00004901120059000200690002269461B48CC
:1030C000FFF7CDFA08B1FDF714FD4FF02040194984
:1030D0000860174848600220886000211548C160D8
:1030E000016141618161C161016241624FF48051BE
:1030F00081620021C16201634163816341640F20E9
:10310000009001900A2002900F200390102004905C
:103110001120059000200690002269460548FFF71F
:103120009EFA08B1FDF7E5FC07B000BDC000002025
:10313000040100A01001002000B587B0142102A8EE
:10314000FDF70BF900BF002001908D48006840F0AA
:1031500010008B4908600846006800F010000190DC
:1031600000BF00BF00BF002001900846006840F08B
:10317000200008600846006800F02000019000BFB1
:1031800000BF00BF002001900846006840F08000AA
:1031900008600846006800F08000019000BF00BF92
:1031A00000BF002001900846006840F0040008605D
:1031B0000846006800F00400019000BF00BF00BF97
:1031C000002001900846006840F0010008600846B1
:1031D000006800F00100019000BF00BF00BF0020A8
:1031E00001900846006840F0020008600846006848
:1031F00000F00200019000BF00BF00BF002001905E
:103200000846006840F0400008600846006800F08A
:103210004000019000BF00BF00BF002001900846A1
:10322000006840F0080008600846006800F00800E8
:10323000019000BF00BF012242F63F015148FEF756
:1032400083FB01224FF4A0714F48FEF77DFB012262
:1032500048F610214D48FEF777FB012240F2C131BC
:103260004B48FEF771FB00224FF480414648FEF7C1
:103270006BFB01224FF655414648FEF765FB0122E4
:1032800041F248514448FEF75FFB0122D102434816
:10329000FEF75AFB42F63F00029001200390049093
:1032A0000320059002A93748FEF754FA4FF4A070A6
:1032B00002900120039004900320059002A9324857
:1032C000FEF748FA48F6102002900120039004907F
:1032D0000320059002A92D48FEF73CFA40F2C130C8
:1032E00002900120039004900320059002A9284831
:1032F000FEF730FA4FF48040029001200390022044
:1033000004900320059002A91F48FEF723FA4FF608
:10331000554002900120039004900320059002A9DB
:103320001C48FEF717FA41F2485002900120039022
:1033300004900320059002A91748FEF70BFA4FF4FA
:10334000006002900120039004900320059002A9E0
:103350001248FEF7FFF9042002904FF40410039086
:103360000120049002A90C48FEF7F4F9002205217F
:103370000820FEF7C5FB0820FEF7B2FB07B000BD32
:1033800030380240001002400014024000000240A9
:103390000004024000180240000C024000080240F5
:1033A00000B58BB0C0208B490870A8204870012060
:1033B00088701D20C870FF20874908704870887089
:1033C0000020C870C02085490870A82048700120DE
:1033D0008870DE20C870002108460EF047FF7D4847
:1033E000007800067B49497840EA014079498978AC
:1033F00040EA01207749C9780843020675480078F9
:1034000000067449497840EA01407249897840EAE7
:1034100001207049C978084300F47F4042EA002245
:103420006C48007800066B49497840EA01416948D8
:10343000807841EA00206749C978084300F47F009A
:1034400042EA10226348007801066248407841EA67
:1034500000416048807841EA00205E49C97808430D
:1034600042EA10605E4908605B48007800065A49ED
:10347000497840EA01405849897840EA0120564994
:10348000C978084302065448007800065249497832
:1034900040EA01405049897840EA01204E49C97804
:1034A000084300F47F4042EA00224B4800780006BF
:1034B0004949497840EA01414748807841EA00207B
:1034C0004549C978084300F47F0042EA1022424887
:1034D000007801064048407841EA00413E48807843
:1034E00041EA00203C49C978084342EA10603D495E
:1034F00008603A48007800063849497840EA0140B7
:103500003649897840EA01203449C97808430206DF
:103510003248007800063149497840EA01402F4995
:10352000897840EA01202D49C978084300F47F409A
:1035300042EA00222948007800062849497840EAF2
:1035400001412648807841EA00202449C97808438F
:1035500000F47F0042EA10222048007801061F484C
:10356000407841EA00411D48807841EA00201B492B
:10357000C978084342EA10601B4908601B481C498F
:103580000022194BCDE900210290164A144919482E
:1035900004F04AFE174805F0B9F8164890F82D00D7
:1035A000C0F3800018B1134805F0F0F902E01148AB
:1035B00005F0B2F810490F4805F014F91C220F4924
:1035C00004A8FCF7A3FE0B4904A805F0B3FB0BB05D
:1035D00000BD000044C0012048C001204CC00120B3
:1035E00038C001203CC0012040C0012065240108F2
:1035F00031590008744D002055570008C442010895
:1036000010B50E480E4908604FF4827048600021E2
:103610000B488160C160016141614FF400718161BB
:103620003821C16100210162416281620A21C162C7
:10363000FEF758FE08B1FDF75CFA10BD00300140FE
:1036400040C3012000B589B00020079008901C21DC
:103650006846FCF782FE4FF0804017490860002062
:1036600048600021144881607721C1600021016118
:103670008161FFF7E8FA08B1FDF73BFA00200790F7
:10368000089007A90C48FFF77DF808B1FDF731FA5B
:10369000602000903C2001900020029004900C22B9
:1036A00069460548FFF74DFA08B1FDF722FA0248CE
:1036B000FFF716FA09B000BD98C3012000BFFEE76E
:1036C00000BFFEE77CB504460D4616461648006866
:1036D0001821B0FBF1F01549B0FBF1F04FF47A710D
:1036E000484301906068B0F5827F0DD12B460022DF
:1036F00080212046009600F01BF898B1606D40F0E4
:103700002000606503207CBD00BF019800B908E07F
:103710000198401E019020688068C0F3C010002806
:10372000F3D100BF0020EEE70C00002040420F0064
:103730002DE9F84F04460D4690461E46DDF82890C8
:10374000FEF708F9A0EB0900371AFEF703F98246E5
:103750002C480068C0F3CB307843009045E0701CE3
:10376000002842D0FEF7F6F8A0EB0A00B84200D2DB
:10377000A7BB2068406820F0E000216848606068CE
:10378000B0F5827F0DD1A068B0F5004F03D0A068DE
:10379000B0F5806F05D12068006820F040002168F6
:1037A0000860A06AB0F5005F0DD100BF2068006816
:1037B00020F40050216808602068006840F4005040
:1037C0002168086000BF012084F8510000BF00207C
:1037D00084F8500000BF0320BDE8F88FFFE7009891
:1037E00000B900270098401E00902068806828409B
:1037F000A84201D1012000E000204045AFD10020C7
:10380000EAE700000C00002010B500BF502080F354
:103810001188BFF34F8FBFF36F8F00BF10F0D6FA40
:1038200018B14FF080500449086000BF002080F3B9
:10383000118800BF10BD000004ED00E000B593B09A
:10384000302107A8FCF789FD142102A8FCF785FDAB
:1038500000BF002001902348006840F080502149BB
:1038600008600846006800F08050019000BF00BF6B
:1038700000BF002001901C48006840F480401A49B5
:1038800008600846006800F48040019000BF00BF57
:10389000012007900004089002200D9041050E9130
:1038A00006210F917821109102211191042112918A
:1038B00007A8FEF7C9FA08B1FDF71BF90F2002901F
:1038C00002200390002004904FF4A0500590069031
:1038D000032102A8FEF766F908B1FDF70AF913B053
:1038E00000BD0000403802400070004003480068FE
:1038F00040F47000014908607047000088ED00E066
:1039000010B50248FFF721F810BD0000600100204B
:1039100010B50268294B98420ED0B0F1804F0BD001
:10392000274B984208D0274B984205D0264B984207
:1039300002D0264B984203D122F070024B681A4302
:103940001E4B984220D0B0F1804F1DD01C4B9842A6
:103950001AD01C4B984217D01B4B984214D01B4BCB
:10396000984211D01A4B98420ED01A4B98420BD065
:10397000194B984208D0194B984205D0184B9842E1
:1039800002D0184B984203D122F44072CB681A43FC
:1039900022F080034C6943EA040202608B68C36230
:1039A0000B688362054B984202D0084B984201D1C4
:1039B0000B6903630123436110BD00000000014057
:1039C0000004004000080040000C004000040140DA
:1039D0000040014000440140004801400018004000
:1039E000001C00400020004030B501F01F050124FC
:1039F00004FA05F3046A9C430462046A01F01F059B
:103A000002FA05F52C43046230BD000030B5056AAA
:103A100025F001050562026A4368846924F0700498
:103A200024F003040D682C4322F002028D682A431F
:103A3000104DA84200D103E00F4DA84206D100BFAF
:103A400022F00802CD682A4322F00402094DA84260
:103A500002D0094DA84207D123F4807323F40073E8
:103A60004D692B438D692B43436084614D684563E9
:103A7000026230BD000001400004014030B5056A1B
:103A800025F010050562026A4368846924F4E04465
:103A900024F440740D6844EA052422F020028D6865
:103AA00042EA0512124DA84200D103E0114DA8428E
:103AB00007D100BF22F08002CD6842EA051222F051
:103AC00040020B4DA84202D00A4DA84209D123F46E
:103AD000806323F400634D6943EA85038D6943EAFB
:103AE0008503436084614D688563026230BD0000D8
:103AF000000001400004014030B5056A25F48075DE
:103B00000562026A4368C46924F0700424F0030467
:103B10000D682C4322F400728D6842EA0522124D92
:103B2000A84200D103E0114DA84207D100BF22F402
:103B30000062CD6842EA052222F480620A4DA84262
:103B400002D00A4DA84209D123F4805323F4005334
:103B50004D6943EA05138D6943EA05134360C46167
:103B60004D68C563026230BD0000014000040140A1
:103B700030B5056A25F480550562036A4468C26958
:103B800022F4E04222F440720D6842EA052223F456
:103B900000538D6843EA0533084DA84202D0084D12
:103BA000A84204D124F480444D6944EA8514446059
:103BB000C2614D680564036230BD00000000014031
:103BC0000004014000BFFEE70FB4054B10B503A988
:103BD000044A029800F034F810BC5DF814FB0000B1
:103BE000095A0008E0C0012002480068C0F3022022
:103BF000704700000CED00E010B5002804DB0A0758
:103C0000130E054A135406E00A07140E034A00F087
:103C10000F031B1FD45410BD00E400E018ED00E0BA
:103C200002E008C8121F08C1002AFAD17047704785
:103C3000002001E001C1121F002AFBD170470000E3
:103C40002DE9FF4F8BB09A460F460546002606E049
:103C500025280BD052460D9990476D1C761C28786C
:103C60000028F5D10FB03046BDE8F08F0024A04603
:103C70000122604900E0044315F8013F203B02FAAD
:103C800003F00842F7D128782E2817D115F8010F34
:103C900044F004042A280ED06FF02F022878A0F1F7
:103CA000300109290AD808EB880102EB410100EB39
:103CB00001086D1CF2E757F8048B6D1C2878692801
:103CC0003ED006DC0028CDD063280BD0642804D178
:103CD00036E0732810D075284BD052460D99904786
:103CE000761C85E017F8040B8DF8000000208DF895
:103CF0000100E946012003E057F8049B4FF0FF3034
:103D000061074FF0000401D40AE0641C44450DDA59
:103D10008442FADB19F804100029F6D106E0641C8D
:103D20008442FCDB19F804100029F8D1264404E091
:103D300019F8010B52460D999047641EF8D257E0CE
:103D400001CF4FF00A0B002802DA40422D2102E099
:103D5000210504D52B218DF82410012103E0E10772
:103D600005D02021F7E70DF1200908910CE0002192
:103D7000F9E701CF4FF00A0BF9E75946FCF705FBCD
:103D800001F1300209F8012D0028F6D1ADEB090050
:103D900000F1200B600701D44FF00108D84502DD87
:103DA000A8EB0B0000E000208046002406E009A8F4
:103DB0005246005D0D999047641C761C0898844219
:103DC000F5DB04E0302052460D999047761CB8F19F
:103DD0000001A8F10108F5DC05E019F8010B5246D5
:103DE0000D999047761CBBF10001ABF1010BF4DC9F
:103DF0006D1C34E70928010070B504460025082C25
:103E000000DA03E00125A4F10800C4B20448005D13
:103E100040F002010122284600F074F970BD000054
:103E20004844010810B500F0D7F9FA20FCF7E2FE8B
:103E300000240CE04FF49661204600F02DF8204657
:103E400000F008F8204601F005FE601CC4B2102CFA
:103E5000F0DB10BD70B504460025082C00DA03E045
:103E60000125A4F10800C4B20A48005D40F0010138
:103E700001230722284600F055FA2046FFF7BCFF31
:103E80000448005D40F0040101230822284600F0A8
:103E900049FA70BD4844010870B504460D462046F5
:103EA00000F020FA2946204600F0D6F970BD000047
:103EB0002DE9F041002701224F21384600F022F978
:103EC00005460DB9BDE8F081002474E03C48005D72
:103ED000284000286DD03B48005D40F002010122DF
:103EE000384600F00FF900F00F06042E2FD006DC44
:103EF000002E53D0012E07D0022E58D105E0062EF9
:103F000043D00C2E53D104E052E0204601F0A2FD34
:103F10004EE004EBC4102C4A8118204600F014F93E
:103F200004EBC411284A114481F880002748005D41
:103F300001280BD104EBC4101346184490F88020DC
:103F400004EBC410C11820460EF00AFE30E004EB6A
:103F5000C4101D4A8118204600F0F6F804EBC41185
:103F6000194A114481F880001848005D01280BD1DE
:103F700004EBC4101346184490F8802004EBC410DE
:103F8000C11820460EF0ECFD12E00E48005D40F036
:103F900005010122384600F0B5F809E00948005D46
:103FA00040F006010122384600F0ACF800E000BF06
:103FB00000BF601CC4B2082C88DB00BF82E7000091
:103FC00050440108484401086C9201206CC701204C
:103FD0002DE9F041012701224F21384600F092F8E7
:103FE00005460DB9BDE8F08108247DE0A4F1080084
:103FF0004049085C2840002874D0A4F108003E4ADB
:10400000105C40F002010122384600F07BF800F01D
:104010000F06042E2FD006DC002E55D0012E07D01F
:10402000022E5DD105E0062E43D00C2E58D104E0BF
:1040300057E0204601F00EFD53E004EBC4102F4A78
:104040008118204600F080F804EBC4112B4A11447B
:1040500081F880002A48005D01280BD104EBC410D0
:104060001346184490F8802004EBC410C118204671
:104070000EF076FD35E004EBC410204A811820468E
:1040800000F062F804EBC4111C4A114481F880006E
:104090001B48005D01280BD104EBC41013461844E3
:1040A00090F8802004EBC410C11820460EF058FD93
:1040B00017E0A4F10800104A105C40F0050101224D
:1040C000384600F01FF80CE0A4F108000A4A105C22
:1040D00040F006010122384600F014F801E001E04A
:1040E00000BF00BF601CC4B2102CFFF67FAF00BF42
:1040F00078E7000050440108484401086C92012010
:104100006CC70120F8B504460D4616460020009005
:1041100044B905F1C04733466A4639460848FEF7B8
:10412000D2FA0AE0012C08D105F1C84733466A46A5
:1041300039460448FEF7C7FA00BF9DF80000F8BDF5
:10414000C0000020100100202DE9F04704460E4673
:10415000002537464FF47A78A946082C00DA04E0A7
:104160004FF00109A4F10800C4B207E0A8F1010072
:104170001FFA80F8B8F1000F00D10BE01548005D80
:1041800040F0050101224846FFF7BCFF00F00100A6
:104190000028EBD000BF0CE00E48015D012248462C
:1041A000FFF7B0FF38707F1C681CC5B2702D00D1BE
:1041B0000BE00848005D40F0050101224846FFF78A
:1041C000A1FF00F001000028E6D100BF2846BDE8AD
:1041D000F08700004844010810B5002413E00B48A4
:1041E000005D40F0010101238022002000F09AF8D8
:1041F0000648005D40F0010101238022184600F0CE
:1042000091F8601CC4B2082CE9DB10BD48440108D9
:104210002DE9F04104460E461746204601F09AFC6F
:104220004FF00008082C00DA04E04FF00108A4F178
:104230000800C4B2002508E0725D0648015D012354
:10424000404600F06FF8681CC5B2BD42F4DBBDE823
:10425000F0810000484401082DE9F04104460F4672
:104260000025A846082C00DA04E04FF00108A4F16C
:104270000800C4B21A48005D40F003010122404624
:10428000FFF740FF054645F080051548005D40F00A
:10429000030101232A46404600F044F84FF4E13080
:1042A000B0FBF7F086B2F2B20D48015D0123404643
:1042B00000F038F832120A48005D40F00101012395
:1042C000404600F02FF805F07F050548005D40F0FE
:1042D000030101232A46404600F024F8BDE8F0819E
:1042E0004844010870B504460025082C00DA03E0B4
:1042F0000125A4F10800C4B20948005D40F00301A3
:1043000001230B22284600F00DF80548005D40F01F
:1043100002010123C122284600F004F870BD00000C
:10432000484401082DE9FF4104460D461E4644B9A4
:1043300005F1C047334602AA39460848FEF7F3F9AB
:104340000AE0012C08D105F1C847334602AA3946D4
:104350000348FEF7E8F900BFBDE8FF81C000002078
:104360001001002010B50446102C69D2DFE804F0DB
:10437000080E141A20262C32383E444A50565C62ED
:10438000012240213048FDF7DFFA5AE00122802166
:104390002D48FDF7D9FA54E0012211022A48FDF711
:1043A000D3FA4EE0012251022748FDF7CDFA48E04A
:1043B000012211462548FDF7C7FA42E001220221F9
:1043C0002248FDF7C1FA3CE0012204211F48FDF715
:1043D000BBFA36E0012208211C48FDF7B5FA30E0AF
:1043E000012210211948FDF7AFFA2AE001224021ED
:1043F0001748FDF7A9FA24E0012291021548FDF7BC
:10440000A3FA1EE00122D1021248FDF79DFA18E03E
:10441000012211030F48FDF797FA12E00122510320
:104420000C48FDF791FA0CE0012291030948FDF7D1
:104430008BFA06E00122D1030648FDF785FA00E079
:1044400000BF00BF10BD0000000402400010024089
:10445000000C02400018024010B50446102C72D225
:10446000DFE804F0080E141B22282E343A40464D93
:10447000545B6269002240213448FDF765FA63E02D
:10448000002280213148FDF75FFA5DE000224FF401
:1044900080712E48FDF758FA56E000224FF4007163
:1044A0002A48FDF751FA4FE0002201212848FDF784
:1044B0004BFA49E0002202212548FDF745FA43E086
:1044C000002204212248FDF73FFA3DE000220821A6
:1044D0001F48FDF739FA37E0002210211C48FDF78C
:1044E00033FA31E0002240211A48FDF72DFA2BE083
:1044F00000224FF480611848FDF726FA24E00022DC
:104500004FF400611448FDF71FFA1DE000224FF43C
:1045100080511148FDF718FA16E000224FF40051BF
:104520000D48FDF711FA0FE000224FF480410A48D0
:10453000FDF70AFA08E000224FF400410648FDF7B3
:1045400003FA01E0FFE700BF00BF10BD0004024016
:1045500000100240000C02400018024010B5002478
:104560000DE0E0B24FF6FF72062100F03DF8E0B238
:1045700040F20E72052100F037F8601CC4B2102C16
:10458000EFDB10BD30B52DED028B81B00546B0EEEE
:10459000408A9FED130A28EE000AF3EE080A80EE27
:1045A000201ABCEEC10A10EE104A00200090042030
:1045B0008DF80000200A8DF80100E0B28DF80200AD
:1045C0002846FFF749FF03226946064806F0AEF881
:1045D0002846FFF7C7FE01B0BDEC028B30BD0000DE
:1045E00000FF7F4740C30120F8B506460D4614463C
:1045F000002000908DF8005020128DF80100E0B2EC
:104600008DF802003046FFF727FF03226946034872
:1046100006F08CF83046FFF7A5FEF8BD40C3012038
:104620002DE9F04104460D4600BF05F003000028C7
:1046300008D000BF0BA34FF4B67216A11DA0FFF760
:10464000C3FA00BF00BF2E4606F0DEF80746A0689A
:1046500000683060A0680660384606F0E1F8BDE802
:10466000F08100002E2E2F4D6964646C65776172B5
:1046700065732F54686972645F50617274792F4C4E
:104680007749502F7372632F636F72652F6D656D5D
:10469000702E63006D656D705F667265653A206DA2
:1046A000656D2070726F7065726C7920616C6967DE
:1046B0006E656400417373657274696F6E202225A4
:1046C0007322206661696C6564206174206C696E78
:1046D0006520256420696E2025730A0070B50546A3
:1046E00006F092F80646A8680468002C16D02068E8
:1046F000A968086000BF04F00300002808D000BFCC
:1047000009A34FF48C7214A11CA0FFF75DFA00BF3F
:1047100000BF304606F084F8204670BD304606F0F3
:104720007FF80020F9E700002E2E2F4D6964646C9D
:104730006577617265732F54686972645F50617246
:1047400074792F4C7749502F7372632F636F7265A2
:104750002F6D656D702E63006D656D705F6D616CA2
:104760006C6F633A206D656D702070726F7065724A
:104770006C7920616C69676E6564000041737365D4
:104780007274696F6E2022257322206661696C65E0
:1047900064206174206C696E6520256420696E2038
:1047A00025730A0070B50546002411E004EB4400AF
:1047B000094901EBC000067D4EB104EB440001EB5A
:1047C000C0008068A84202D1204600F087F9641C2E
:1047D0000A2CEBDB70BD00007C9101202DE9FF5F0E
:1047E0000646894617464FF00A0AD346D0460024AB
:1047F0000A200390002002900190009000BF73E017
:1048000004EB4400764901EBC000057DB8F10A0FC6
:1048100002D10DB9A04665E0002D63D000BF012D87
:104820000AD0022D08DA00BF6EA340F223127BA14A
:104830008AA0FFF7C9F900BF00BFAEB104EB440185
:10484000674A02EBC1013068496888420CD13FB128
:1048500004EB4400114601EBC0008068B84203D16C
:10486000204604B0BDE8F09F012D28D104EB4400A0
:104870005B4951F8300080B104EB440001EBC0000B
:10488000418A029881422DDB039404EB4400544991
:1048900001EBC000408A029024E004EB4400504940
:1048A00001EBC000418A019881421BDBA24604EB68
:1048B00044004B4901EBC000408A019012E0022DF8
:1048C00010DB04EB4400464901EBC000418A00982C
:1048D000814207DBA34604EB4400414901EBC000E1
:1048E000408A0090601C04B20A2C89DB09F00200A7
:1048F00028B9B8F10A0F05D109F0010010B94FF03D
:10490000FF30AEE7B8F10A0F01DA444631E0BBF1FF
:104910000A0F11DA5C4600BF04EB4400304951F83D
:10492000300040B100BF2FA340F26D1255A14BA043
:10493000FFF74AF900BF0CE0BAF10A0F01DA54465A
:1049400007E003980A2801DA039C02E04FF0FF30E9
:1049500087E700BF0A2C08DB00BF22A340F27F12CA
:104960004EA13EA0FFF730F900BF00BF204600F087
:10497000B5F800BF0A2C08DB00BF1AA340F283126F
:1049800046A136A0FFF720F900BF00BF00BF04EB2F
:104990004400134901EBC000007D40B100BF11A3EA
:1049A0004FF4C27242A12DA0FFF70EF900BF00BF65
:1049B00036B104EB44010A4A02EBC1013068486099
:1049C000002004EB4401064A02EBC101488204EBDB
:1049D0004400114601EBC0008760204641E700001B
:1049E0007C9101202E2E2F4D6964646C6577617275
:1049F00065732F54686972645F50617274792F4CCB
:104A00007749502F7372632F636F72652F697076C9
:104A1000342F6574686172702E6300007374617462
:104A200065203D3D204554484152505F5354415408
:104A3000455F50454E44494E47207C7C207374614D
:104A40007465203E3D204554484152505F535441C7
:104A500054455F535441424C450000004173736517
:104A60007274696F6E2022257322206661696C65FD
:104A700064206174206C696E6520256420696E2055
:104A800025730A006172705F7461626C655B695DB9
:104A90002E71203D3D204E554C4C000069203C209D
:104AA0004152505F5441424C455F53495A450000C2
:104AB0006172705F7461626C655B695D2E737461B5
:104AC0007465203D3D204554484152505F53544148
:104AD00054455F454D5054590000000010B5044640
:104AE00004EB44000C4951F8300060B104EB440180
:104AF000094A52F8310004F05FFE002004EB440143
:104B0000054A42F83100002004EB4401024A02EB5E
:104B1000C101087510BD00007C910120F0B587B07F
:104B200007460D4600BF002D0AD100BF2EA340F25C
:104B30008A223BA13EA0FFF747F800BF07B0F0BDB7
:104B400000BF7C682088B0F5807F08D120790628D6
:104B500005D16079042802D16088082803D038463E
:104B600004F02AFEEAE7D4F80E000690A06905904A
:104B7000686808B9002607E005986968884201D18D
:104B8000012000E0002006460EB1012000E00220D6
:104B9000034604F1080206A9284600F0CBFCE08891
:104BA000B0F5807F03D0B0F5007F15D113E086B15A
:104BB000022206AB04F10800291DCDE90232CDE93D
:104BC000001005F1260302462231284600F05CFB66
:104BD00000E000BF01E000E000BF00BF384604F085
:104BE000EBFD00BFAAE700002E2E2F4D6964646C18
:104BF0006577617265732F54686972645F50617282
:104C000074792F4C7749502F7372632F636F7265DD
:104C10002F697076342F6574686172702E6300009E
:104C20006E6574696620213D204E554C4C00000095
:104C3000417373657274696F6E202225732220663A
:104C400061696C6564206174206C696E65202564FF
:104C500020696E2025730A002DE9FE4304460F46A5
:104C60001546A94600BF002C08D100BF5DA340F245
:104C70001E326AA16DA0FEF7A7FF00BF00BF00BFF4
:104C800047B900BF57A340F21F3272A167A0FEF7D9
:104C90009BFF00BF00BF00BF002D08D100BF51A384
:104CA0004FF448726EA161A0FEF78EFF00BF00BFF7
:104CB0002146286801F0B9F910B1DFF8B48186E027
:104CC000287800F0F000E02816D101208DF80400CB
:104CD00000208DF805005E208DF80600687800F051
:104CE0007F008DF80700A8788DF80800E8788DF827
:104CF00009000DF1040869E02868A1680840D4E9BA
:104D00000112114088420ED0288880B24FF6A96166
:104D1000884208D0E06810B104F10C0903E06FF09C
:104D20000300BDE8FE835348007800EB4000524981
:104D300001EBC000007D02281BDB4E48007800EB31
:104D4000400001EBC0008068A04212D149490978B7
:104D500001EB4101484A02EBC101D9F80000496862
:104D6000884206D1434802783946204600F086F84A
:104D7000D7E7002622E006EB46003F4901EBC000E2
:104D8000007D022818DB06EB460001EBC0008068BE
:104D9000A04211D106EB4601374A02EBC101D9F816
:104DA00000004968884207D13248067032463946C9
:104DB000204600F063F8B4E7701CC6B20A2EDADBB6
:104DC0003A464946204600F00DF9AAE700BF4FF4E5
:104DD0000060434604F1260239460090204600F068
:104DE00025FD9EE72E2E2F4D6964646C65776172F8
:104DF00065732F54686972645F50617274792F4CC7
:104E00007749502F7372632F636F72652F697076C5
:104E1000342F6574686172702E6300006E6574696A
:104E20006620213D204E554C4C00000041737365B7
:104E30007274696F6E2022257322206661696C6529
:104E400064206174206C696E6520256420696E2081
:104E500025730A007120213D204E554C4C00000066
:104E600069706164647220213D204E554C4C0000F5
:104E7000E0420108B00000207C910120F8B5054611
:104E80000E46144600BF04EB4400314901EBC0005C
:104E9000007D022808DA00BF2EA340F2EE223BA1DB
:104EA00046A0FEF791FE00BF00BF04EB4400284976
:104EB00001EBC000007D022839D104EB440001EB76
:104EC000C000408AB0F58E7F11DD04EB44000A4635
:104ED00002EBC000011D284600F09CFA38BB0320FD
:104EE00004EB44011A4A02EBC10108751FE004EB10
:104EF0004400174901EBC000408AB0F5877F16DBFC
:104F000004EB44000B4603EBC00000F10C0204EB81
:104F1000440003EBC000011D284600F087FA30B9B9
:104F2000032004EB44010A4A02EBC10108754FF467
:104F30000060009004EB4400054901EBC00000F163
:104F40000C0305F126023146284600F06FFCF8BD3F
:104F50007C9101202E2E2F4D6964646C65776172FF
:104F600065732F54686972645F50617274792F4C55
:104F70007749502F7372632F636F72652F69707654
:104F8000342F6574686172702E6300006172705F07
:104F90007461626C655B6172705F6964785D2E73C9
:104FA00074617465203E3D204554484152505F5322
:104FB000544154455F535441424C4500417373651D
:104FC0007274696F6E2022257322206661696C6598
:104FD00064206174206C696E6520256420696E20F0
:104FE00025730A002DE9FE4F81460F46164609F14A
:104FF000260A4FF0FF3002900020019049463868A1
:1050000001F013F838B9387800F0F000E02802D049
:105010000FB1386818B96FF00F00BDE8FE8F4A462F
:1050200001213846FFF7DAFB8046B8F1000F02DABB
:105030004FFA88F0F1E700BFB8F17F0F08D300BF47
:105040005FA340F2C1326CA16FA0FEF7BDFD00BFAF
:1050500000BF08F0FF0404EB4400754901EBC000F9
:10506000007D70B90120019004EB4401704A02EB0D
:10507000C101087504EB4400114601EBC000C0F803
:10508000089000BF04EB4400694901EBC000007DBB
:1050900001280FD004EB440001EBC000007D022882
:1050A00008DA00BF46A340F2CD3262A156A0FEF757
:1050B0008BFD00BF00BF019800B93EB93946484694
:1050C00000F0A8F902900EB90298A6E700BF46B911
:1050D00000BF3BA340F2E13260A14BA0FEF774FD9C
:1050E00000BF00BF04EB4400514901EBC000007D4C
:1050F000022811DB5C4804704FF40060009004EB60
:10510000440001EBC00000F10C0352463146484612
:1051100000F08CFB029050E004EB4400444901EBAA
:10512000C000007D012848D14FF0000B354618E043
:1051300000BF6889298988420AD1286840B100BF28
:105140001FA340F2F13249A12FA0FEF73DFD00BFA1
:1051500000BF287B00F0400010B14FF0010B02E0CF
:105160002D68002DE4D100BFBBF1000F07D03246FF
:105170004FF420710E2004F013F9054603E0354684
:10518000284604F029FDA5B104EB4400284951F854
:10519000300030B104EB4401254A52F8310004F0EC
:1051A0000BFB04EB4400224941F8305000200290F0
:1051B00002E04FF0FF30029000BF02982DE70000A0
:1051C0002E2E2F4D6964646C6577617265732F5460
:1051D000686972645F50617274792F4C7749502FFF
:1051E0007372632F636F72652F697076342F6574E5
:1051F000686172702E63000074797065206F766547
:1052000072666C6F77000000417373657274696F2A
:105210006E2022257322206661696C6564206174AA
:10522000206C696E6520256420696E2025730A0054
:105230007C9101206172705F7461626C655B695D75
:105240002E7374617465203D3D2050454E44494E97
:1052500047206F7220535441424C45007120213D3C
:10526000204E554C4C000000B00000206E6F2070A6
:1052700061636B65742071756575657320616C6C15
:105280006F776564210000002DE9FC5F06460F463C
:1052900090469946DDE90CAB0020019000BF002E3E
:1052A00008D100BF31A340F257423EA141A0FEF712
:1052B0008BFC00BF00BF4FF420721C210E2003F0B6
:1052C000E5FD05461DB94FF0FF30BDE8FC9F00BF6E
:1052D00068891C2808DA00BF24A340F262423FA17B
:1052E00034A0FEF771FC00BF00BF6C680F9802F09D
:1052F00074F9E08000BF96F82C00062808D000BFA3
:105300001AA340F2694242492AA0FEF75DFC00BFA1
:1053100000BFD9F80000A060B9F80400A081DBF854
:105320000000C4F81200BBF80400E082DAF80000C4
:10533000C4F80E000E980068A0614FF480702080C1
:1053400008206080062020710420607140F606006D
:1053500043463A4629460090304600F067FA284610
:1053600004F02AFA00250198AFE700002E2E2F4DF9
:105370006964646C6577617265732F5468697264DF
:105380005F50617274792F4C7749502F7372632F7D
:10539000636F72652F697076342F657468617270FF
:1053A0002E6300006E6574696620213D204E554CC9
:1053B0004C000000417373657274696F6E20222582
:1053C0007322206661696C6564206174206C696E6B
:1053D0006520256420696E2025730A006368656373
:1053E0006B207468617420666972737420706275D2
:1053F000662063616E20686F6C64207374727563DD
:1054000074206574686172705F68647200000000E7
:10541000A045010870B504460D46034A29462046BA
:1054200000F004F870BD0000E04201087FB50446BA
:105430000D4616460121074A201D04F126038DE87A
:1054400025000391324619462046FFF71DFF04B0A0
:1054500070BD0000E642010870B5002464E004EB72
:105460004400334901EBC000057D002D5BD004EB07
:10547000440001EBC000408A401C04EB44012C4A6C
:1054800002EBC101488204EB4400114601EBC0006D
:10549000408AB0F5967F0DDA04EB440001EBC000C2
:1054A000007D01280AD104EB440001EBC000408AD2
:1054B000052803DB2046FFF711FB34E004EB440032
:1054C0001B4901EBC000007D032807D1042004EB39
:1054D0004401174A02EBC101087524E004EB4400C3
:1054E000134901EBC000007D042807D1022004EB22
:1054F00044010F4A02EBC101087514E004EB4400BB
:105500000B4901EBC000007D01280CD104EB4402E3
:105510000B4603EBC202111D04EB440203EBC20273
:105520009068FFF777FF641C0A2C98DB70BD0000C1
:105530007C9101202DE9F84305460E461746984612
:1055400000BF95F82C00062808D000BF2EA340F21B
:10555000A9123BA143A0FEF737FB00BF00BF5EB11D
:10556000306848B12946306800F05FFD20B93078D6
:1055700000F0F000E02803D16FF00F00BDE8F883E1
:105580002A4641463046FFF729F90446002C01DA45
:1055900060B2F3E7022004EB44013C4A02EBC10194
:1055A000087504EB4400114601EBC000856004EB74
:1055B000440001EBC0003968C160B9880182002055
:1055C00004EB440102EBC101488204EB44001146A4
:1055D00051F83000B0B104EB440051F83090002095
:1055E00004EB440142F831004FF400603B4605F102
:1055F000260249460090284600F018F9484604F073
:10560000DBF800BF0020B9E72E2E2F4D6964646CD3
:105610006577617265732F54686972645F50617257
:1056200074792F4C7749502F7372632F636F7265B3
:105630002F697076342F6574686172702E63000074
:105640006E657469662D3E6877616464725F6C652F
:105650006E203D3D204554485F4857414444525FC9
:105660004C454E00417373657274696F6E2022253C
:105670007322206661696C6564206174206C696EB8
:105680006520256420696E2025730A007C91012025
:105690002DE9F04104460E464FF00E0860890E28B1
:1056A00000DC4FE0E07B18B996F83000401CE07356
:1056B0006568AF89287800F00100B0B1287801282A
:1056C00009D1687888B9A8785E280ED1607B40F04F
:1056D0001000607309E006221D492846FAF748FECB
:1056E00018B9607B40F008006073082F03D0B7F54D
:1056F000C16F22D110E096F82D0000F0080000B92B
:1057000020E04146204604F0BBFA00B11AE03146E1
:10571000204600F017FE11E096F82D0000F008007A
:1057200000B90FE04146204604F0AAFA00B109E0B2
:1057300031462046FFF7F2F900E003E000BF002009
:10574000BDE8F081204604F037F80020F8E70000BB
:10575000E0420108704700009AB00646642101A8A3
:10576000FAF7FBFD00240027A046A146354600BFFE
:105770002C48FDF74AFB044695F82D00C0F3800045
:1057800058B1012C09DC2848FBF778FE284602F0C6
:10579000C3FF284603F02AF83FE095F82D00C0F338
:1057A0008000002839D1012C37DD022C06D0032CD3
:1057B0000AD0042C0ED0052C17D111E04FF400694B
:1057C0004FF48048012711E04FF000094FF4804862
:1057D00001270BE04FF400694FF00008012705E0B6
:1057E0004FF00009C846012700E000BF00BFA7B185
:1057F00001A90D48FBF726FACDF81C90CDF81880CA
:1058000001A90948FBF782FD0748FBF7CBFD2846B5
:1058100003F0BCF8284603F04FF8642003F016F9B3
:10582000A6E70000544D00206C4C00202DE9F04705
:1058300005460E4617469846DDF82090484601F08A
:10584000CCFE82460E21304603F0A3FA00B122E0DE
:105850007468A4F80CA0D8F800002060B8F8040020
:10586000A0803868C4F80600B888608100BF95F849
:105870002C00062808D000BF08A34FF4997215A188
:1058800021A0FEF7A1F900BF00BF31462846AA6952
:105890009047BDE8F0876FF00100FAE72E2E2F4DFC
:1058A0006964646C6577617265732F5468697264AA
:1058B0005F50617274792F4C7749502F7372632F48
:1058C0006E657469662F65746865726E65742E63A3
:1058D000000000006E657469662D3E68776164643F
:1058E000725F6C656E206D75737420626520362062
:1058F000666F722065746865726E65745F6F75742B
:105900007075742100000000417373657274696FD3
:105910006E2022257322206661696C6564206174A3
:10592000206C696E6520256420696E2025730A004D
:1059300010B5044600BF44B900BF0CA34FF4F17288
:1059400011A115A0FEF740F900BF00BF732084F835
:105950002E0074212F200155194860611948A0615B
:10596000204601F09BFC002010BD00002E2E2F4C85
:105970005749502F5461726765742F65746865725A
:105980006E657469662E63006E6574696620213DDC
:10599000204E554C4C000000417373657274696F62
:1059A0006E2022257322206661696C656420617413
:1059B000206C696E6520256420696E2025730A00BD
:1059C000594C0008B174000806460024354600BF53
:1059D0004FF0FF310B48006803F078F90028F7D149
:1059E00000BF284601F052FD04463CB1294620463E
:1059F0002A69904710B1204603F0DEFE002CF0D15A
:105A0000E6E700001CC0012038B504468DF8000010
:105A100069460320ABBE204638BD000010B5002407
:105A2000002210210A48FBF78FFF0A20FBF7E2F85B
:105A3000012210210648FBF787FF00BF04E0204643
:105A400000F008F8601CC4B2102CF8DB10BD000098
:105A50000000024010B50446102C69D2DFE804F0C3
:105A6000080E141A20262C32383E444A50565C62E6
:105A7000012210213048FBF767FF5AE00122042180
:105A80002D48FBF761FF54E0012211032B48FBF77F
:105A90005BFF4EE0012291022848FBF755FF48E0EA
:105AA000012211022548FBF74FFF42E0012251037A
:105AB0002348FBF749FF3CE00122D1022048FBF7D5
:105AC00043FF36E0012211461B48FBF73DFF30E063
:105AD000012211461B48FBF737FF2AE00122110281
:105AE0001948FBF731FF24E0012240211648FBF75B
:105AF0002BFF1EE00122D1031448FBF725FF18E01D
:105B00000122D1021248FBF71FFF12E00122D1024D
:105B10000E48FBF719FF0CE0012251020B48FBF77E
:105B200013FF06E0012240210348FBF70DFF00E0D0
:105B300000BF00BF10BD000000180240000C024072
:105B40000010024000040240001402400000024025
:105B50000008024010B50446102C74D2DFE804F0AF
:105B6000080E141B222930373D434A50575E656C9E
:105B7000002210213548FBF7E7FE65E000220421F2
:105B80003248FBF7E1FE5FE000224FF480513048DD
:105B9000FBF7DAFE58E000224FF480612C48FBF757
:105BA000D3FE51E000224FF480712948FBF7CCFE70
:105BB0004AE000224FF400512648FBF7C5FE43E0BF
:105BC00000224FF400612348FBF7BEFE3CE00022B8
:105BD00001211E48FBF7B8FE36E0002201211E48D5
:105BE000FBF7B2FE30E000224FF480711B48FBF758
:105BF000ABFE29E0002240211848FBF7A5FE23E078
:105C000000224FF400411648FBF79EFE1CE00022E4
:105C10004FF400611348FBF797FE15E000224FF4A4
:105C200000610F48FBF790FE0EE000224FF4007178
:105C30000B48FBF789FE07E0002240210348FBF7F1
:105C400083FE01E0FFE700BF00BF10BD0018024067
:105C5000000C024000100240000402400014024008
:105C6000000002400008024070B505460C4622467E
:105C70000321284600F03AF970BD00002DE9FF5FCE
:105C800005468A46654880680390039800780007B7
:105C9000860E142E00DAB7E06889042800D2B3E03B
:105CA0006868047814B1082C70D100E0A6E0DFF831
:105CB0006C9109F114095948007D00F0F000E028CA
:105CC00000D1A5E0554A1168506900F0AEF900B165
:105CD0009EE02889082800D296E006F10E012846A9
:105CE00003F057F8002840D0288930441FFA80FB81
:105CF0002889584500DD8BE04FF4207259460E206C
:105D000003F0C4F8074607B982E0798906F1080074
:105D1000814203D2384603F04FFD79E0324678687D
:105D20000399FAF7F3FA3146384603F0A9FF002841
:105D30000DD000BF00BF3AA3B62247A154A0FDF783
:105D400043FF00BF00BF384603F036FD60E0294640
:105D5000384603F07DFB18B1384603F02DFD57E0BF
:105D6000284603F029FD3D4611E006F10E012846C4
:105D700003F086FF58B100BF00BF29A3C7224EA180
:105D800043A0FDF721FF00BF00BF41E024E0D5F8AC
:105D900004803146284602F0FCFFE0B96F68D9F86C
:105DA0000000F8601D4800693861002088F8000094
:105DB000A8F80200FF20387200207881012000211D
:105DC000FF230A46CDE9010A00914946284600F022
:105DD000A1FB834600BF11E0032C0ED00B2C0CD08E
:105DE0000C2C0AD0042C08D0052C06D00D2C04D085
:105DF0000E2C02D0112C00D000BF00BF00BF2846DF
:105E000003F0DAFCBDE8FF9F284603F0D5FCF9E774
:105E1000284603F0D1FC00BFF4E70000C4C601200F
:105E20002E2E2F4D6964646C6577617265732F54F3
:105E3000686972645F50617274792F4C7749502F92
:105E40007372632F636F72652F697076342F696385
:105E50006D702E630000000069636D705F696E7085
:105E600075743A206D6F76696E6720722D3E706191
:105E7000796C6F616420746F2069636D7020686550
:105E800061646572206661696C65640A00000000E7
:105E9000417373657274696F6E20222573222066C8
:105EA00061696C6564206174206C696E652025648D
:105EB00020696E2025730A0069636D705F696E70DA
:105EC00075743A20726573746F72696E67206F72B1
:105ED0006967696E616C20702D3E7061796C6F61CD
:105EE00064206661696C65640A0000002DE9FF4763
:105EF0000746884691464FF420722421222002F062
:105F0000C5FF05460DB9BDE8FF8700BF6889242895
:105F100008D200BF19A34FF4B47226A130A0FDF738
:105F200053FE00BF00BFD7F804A06C6884F800805F
:105F300084F801900020A080E08079686A6802F10E
:105F400008001C22FAF7E2F9DAF80C00039003A823
:105F500000F048FD06465EB100206080012000216F
:105F6000FF2303AACDE901060091284600F0D2FAEA
:105F7000284603F021FC00BFC5E700002E2E2F4D60
:105F80006964646C6577617265732F5468697264C3
:105F90005F50617274792F4C7749502F7372632F61
:105FA000636F72652F697076342F69636D702E632D
:105FB00000000000636865636B207468617420668C
:105FC0006972737420706275662063616E20686FF9
:105FD0006C642069636D70206D6573736167650023
:105FE000417373657274696F6E2022257322206677
:105FF00061696C6564206174206C696E652025643C
:1060000020696E2025730A0070B505460C462246AD
:106010000B212846FFF76AFF70BD00BFEFF3058034
:1060200008B1012070470020FCE718B50246009235
:10603000D04300B10AB9012018BD91F82D0000F03D
:10604000020008B90020F7E74868904201D100201B
:10605000F2E700988B681840D1E901342340984258
:1060600008D1886822EA00008C68E343984201D195
:106070000120E1E70020DFE72DE9F74F8CB004466F
:106080000F464FF00008B98CA1F11400C11700EBC6
:106090005171C1F3CF0A1420059060680990DDF8B2
:1060A000249099F8000000F00F001421B1EB800F4C
:1060B00004D06FF005000FB0BDE8F08F00BF60891D
:1060C00014280BDA00BF72A34FF43F727FA186A0A1
:1060D000FDF77AFD00BF6FF00500ECE700BFB9F8EF
:1060E000060001F07AFA04900498C0F30C000790BF
:1060F000049800F400500390208914381FFA80FBA4
:10610000BDE04FF6FF7000EACA00584501DD584671
:1061100003E04FF6FF7000EACA0008904FF42072C7
:1061200014210E2002F0B2FE054605B9ADE000BF15
:106130006889142808DA00BF55A34FF4497274A186
:1061400069A0FDF741FD00BF00BF142268680999EE
:10615000FAF7DCF8D5F8049008980A9054E06189C1
:106160000598081A80B2029000BF618905988142A3
:1061700008DA00BF46A340F22D326DA15AA0FDF708
:1061800023FD00BF00BF02990A98884201DA0A98ED
:1061900000E002988046B8F1000F03D1002005907E
:1061A000246831E000F068FC06461EB9284603F07A
:1061B00003FB6AE061680598084433464122414682
:1061C000CDE90008002003F00FF80B900B9830B9D0
:1061D000304600F057FC284603F0EEFA55E0204622
:1061E00003F0FAFC74615648306128460B9903F0BD
:1061F00025F80A98A0EB080080B20A900A9810B11E
:1062000000200590246800BF0A980028A7D10598AF
:10621000404480B20590B88C1438584501DB012009
:1062200000E0002006900798C0F30C000490069848
:1062300008B1039818B1049840F4005004900498F1
:1062400001F0CBF9A9F806000899143188B201F0E1
:10625000C4F9A9F802000020A9F80A007B692946C0
:1062600038460E9A9847284603F0A6FA0898ABEBF2
:1062700000001FFA80FB0798504480B20790BBF1E2
:10628000000F7FF43EAF002015E74FF0FF3012E71C
:106290002E2E2F4D6964646C6577617265732F547F
:1062A000686972645F50617274792F4C7749502F1E
:1062B0007372632F636F72652F697076342F697004
:1062C000345F667261672E63000000006970345F9E
:1062D0006672616728293A207062756620746F6F54
:1062E0002073686F72740000417373657274696F14
:1062F0006E2022257322206661696C6564206174BA
:10630000206C696E6520256420696E2025730A0063
:1063100074686973206E65656473206120706275AE
:106320006620696E206F6E65207069656365210067
:10633000702D3E6C656E203E3D20706F66660000DD
:10634000D57100082DE9F04707460E467D6828788C
:106350000421B1EB201F05D0384603F02DFA0020B0
:10636000BDE8F087287800074FEA9068688801F058
:1063700034F981463989494503DD4946384603F0F9
:1063800077FB7889404505DB3889484502DBB8F161
:10639000140F04DA384603F00FFA0020E0E728690A
:1063A0004D494861E86808610846007D00F0F0004A
:1063B000E0280AD196F82D0000F0010018B17068AD
:1063C00008B134461CE000241AE0304600F088F89A
:1063D00008B1344614E000243F48007D7F280FD0E8
:1063E0003E48046809E0B44200D105E0204600F0D0
:1063F00077F800B103E000BF2468002CF3D100BFA0
:10640000354908693146FFF710FE28B93248007C4B
:1064100000F0F000E02804D1384603F0CDF9002068
:106420009EE724B9384603F0C7F9002098E7E888CA
:106430004FF63F71084038B1384600F055F907462D
:106440000FB900208CE77D682348046046608560B2
:1064500028780007800E204988814146384603F09D
:106460000FFC687A01280DD0062806D011280ED11D
:10647000314638460CF09AF922E03146384605F0AC
:1064800045FD1DE031463846FFF7F8FB18E012499C
:1064900048692146FFF7C9FD70B90F48007D00F03B
:1064A000F000E02808D00FFA88F1384603F095FA9A
:1064B00002213846FFF7D8FB384603F07DF900BFCC
:1064C00000BF002004490860486088608881086136
:1064D000486100BF44E70000C4C60120500000200E
:1064E00010B5044694F82D0000F0010070B160680A
:1064F00060B1074840696168884205D0044948692D
:106500002146FFF792FD08B1012010BD0020FCE7F5
:10651000C4C601202DE9FE4F07460C461546984695
:10652000DDE90C9A0E9EA34625B10CB1206808B98E
:1065300006F1040B43462A4659463846CDE9009AEF
:10654000029600F003F8BDE8FE8F00002DE9F84F39
:1065500005460F4690469A46DDF828B00C9E00BFCF
:10656000A87B012808D000BF37A34FF4557243A180
:1065700045A0FDF729FB00BF00BFB8F1000F46D0D2
:106580004FF014091421284602F003FC18B16FF0F3
:106590000100BDE8F88F6C6800BF6889142808D234
:1065A00000BF29A34FF4627241A137A0FDF70CFB95
:1065B00000BF00BF84F808A00B986072D8F80000F4
:1065C000206148464FEAE97109EB9171C1F38701F7
:1065D00041F04001217084F801B0288900F0FDFFEE
:1065E00060800020E0803E48008800F0F6FFA08038
:1065F0003B480088401C3A4908801FB93948006868
:10660000E06001E03868E0600020608109E06889AE
:10661000142802DA6FF00100BBE76C682069009073
:10662000E846B08C48B12889B18C884205DD4246E5
:1066300031462846FFF720FDABE742462946304663
:1066400073699847A5E700002E2E2F4D6964646C8E
:106650006577617265732F54686972645F50617207
:1066600074792F4C7749502F7372632F636F726563
:106670002F697076342F6970342E6300702D3E724E
:106680006566203D3D203100417373657274696F0A
:106690006E2022257322206661696C656420617416
:1066A000206C696E6520256420696E2025730A00C0
:1066B000636865636B2074686174206669727374C3
:1066C00020706275662063616E20686F6C64207351
:1066D00074727563742069705F68647200000000F2
:1066E000B2000020284401082DE9F14F84B004983D
:1066F0004568287800F00F001421B1EB800F00D01E
:1067000011E1E88800F069FFC0F30C004FF6FF715B
:1067100001EAC00A688800F060FF07462878000791
:10672000810E02910299B94200DDFCE00298381A0C
:1067300087B2049802F02AFE06467D48018888192F
:106740000A280ADD3146284600F0E6FC20B17848E8
:10675000008830440A2800DDE5E07648046811E04E
:106760006069E968884209D1A0692969884205D130
:10677000A089A988884201D1012000E0002000B151
:1067800002E02468002CEBD100BF34B93146284622
:1067900000F0A8FB044694B9C5E0E88800F01DFFAE
:1067A000C0F30C0058B9E08900F017FFC0F30C00EB
:1067B00028B11422294604F10800F9F7A7FDE8885A
:1067C000012121EA50100190019850B10AEB070114
:1067D00088B2504503DB4FF6EB71884200DD80E064
:1067E00000BF2046019A049900F098F983460BF106
:1067F000010000B975E04E48008830444C490880DB
:10680000019840B10AEB070188B2A083A17F41F053
:106810000101A17700BFBBF1010F60D1A08B143043
:1068200080B2009060684068D0F800906068456869
:10683000142204F108012846F9F768FD009800F0D9
:10684000CCFE68800020E8806881606804900DE0DC
:10685000D9F8040003901421484603F011FA494680
:10686000049802F0EBFC0398D0F80090B9F1000F07
:10687000EED130480068844202D14FF000080EE0AB
:106880002C48D0F8008006E0D8F80000A04200D1E3
:1068900004E0D8F80080B8F1000FF5D100BF414600
:1068A000204600F0BDFA049802F070FD064600BFD5
:1068B0001F480088B04208DA00BF1FA340F29B22A5
:1068C0002CA133A0FDF780F900BF00BF1848008855
:1068D000801B17490880049805B0BDE8F08F0020A0
:1068E000FAE700BF44B900BF13A34FF42A7232A1E4
:1068F00027A0FDF769F900BF00BF606890B900BF2D
:106900000C480068844208D000BF0BA340F2AB22C1
:106910002CA11FA0FDF758F900BF00BF00212046A1
:1069200000F07EFA00BF049802F046FF0020D3E793
:10693000DCC00120D8C001202E2E2F4D6964646C6C
:106940006577617265732F54686972645F50617214
:1069500074792F4C7749502F7372632F636F726570
:106960002F697076342F6970345F667261672E63A9
:106970000000000069705F72656173735F7062751B
:1069800066636F756E74203E3D20636C656E00001B
:10699000417373657274696F6E20222573222066BD
:1069A00061696C6564206174206C696E6520256482
:1069B00020696E2025730A0069707220213D204EE7
:1069C000554C4C006E6F74206669727374616C7400
:1069D000686F756768206A75737420656E71756578
:1069E0007565640010B502462148016821E091F800
:1069F0002D0000F00100D8B191F82D00C0F3800007
:106A0000B0B14868A0B110688B681840D1E9013472
:106A10002340984201D1084610BD91F82D0000F0A6
:106A2000020028B91068CB68984201D10846F3E704
:106A300009680029DBD10F480068A0B10D48006843
:106A400090F82D0000F0010068B10A48006890F845
:106A50002D00C0F3800030B106480068406810B1D6
:106A600010787F2801D10020D6E702480068D3E7DC
:106A7000500000205400002010B5052001F030FB2C
:106A800010BD000010B5044600BF002C08D100BFA7
:106A900006A34FF4317214A116A0FDF795F800BFBC
:106AA00000BF2146052001F04DFA10BD2E2E2F4DBE
:106AB0006964646C6577617265732F546869726488
:106AC0005F50617274792F4C7749502F7372632F26
:106AD000636F72652F697076342F6970345F6672E8
:106AE00061672E63000000007020213D204E554C50
:106AF0004C000000417373657274696F6E2022252B
:106B00007322206661696C6564206174206C696E13
:106B10006520256420696E2025730A002DE9F74F52
:106B200084B006468846002501200190D8F804006C
:106B300002900299488800F050FD83460298007840
:106B40000007800E03900398584503DD681E07B0C8
:106B5000BDE8F08F0398ABEB00001FFA80FB0299B1
:106B6000C88800F03AFDC0F30C004FF6FF7101EA4F
:106B7000C00A00BF00BFD8F8044000202060A4F87D
:106B800004A00AEB0B00E080E088504502DA4FF0E9
:106B9000FF30DCE7D6F804903EE0D9F80470A08816
:106BA000B988884220DAC4F800909DB1A088E988AD
:106BB000884203DBE088B988884202DD4FF0FF306D
:106BC000C5E7C5F80080E888A18888420BD000207E
:106BD000019008E0E088B988884202DD4FF0FF307C
:106BE000B5E7C6F804801AE0A088B988884202D1C7
:106BF0004FF0FF30ABE7A088F988884202DA4FF007
:106C0000FF30A4E72DB1E888B988884201D0002080
:106C10000190D7F800903D46B9F1000FBDD100BFFB
:106C2000B9F1000F28D1002D17D000BFE888A18846
:106C3000884208DD00BF3EA34FF4DB724BA153A096
:106C4000FCF7C2FF00BF00BFC5F80080E888A1883C
:106C5000884211D0002001900EE000BF706840B162
:106C600000BF33A34FF4DF7252A148A0FCF7ACFF82
:106C700000BF00BFC6F80480069820B9B07F00F0BE
:106C80000100002851D00198002848D0706818B140
:106C900070684068808810B1002001903FE0254670
:106CA000D4F800900BE0D9F80440E888A188884225
:106CB00002D00020019005E02546D4F80090B9F1FB
:106CC000000FF0D100BF0198002828D000BF7068E5
:106CD00040B900BF16A340F2DF1244A12BA0FCF77D
:106CE00073FF00BF00BF00BF70684068A04208D1BA
:106CF00000BF0FA34FF4F0723CA124A0FCF764FF87
:106D000000BF00BF00BF206840B100BF08A34FF420
:106D1000F1723AA11DA0FCF757FF00BF00BF019818
:106D200008B1012013E7002011E700200FE7000061
:106D30002E2E2F4D6964646C6577617265732F54D4
:106D4000686972645F50617274792F4C7749502F73
:106D50007372632F636F72652F697076342F697059
:106D6000345F667261672E630000000063686563CC
:106D70006B20667261676D656E747320646F6E2739
:106D800074206F7665726C617000000041737365EA
:106D90007274696F6E2022257322206661696C65AA
:106DA00064206174206C696E6520256420696E2002
:106DB00025730A006E6F2070726576696F75732097
:106DC000667261676D656E742C2074686973206DDE
:106DD00075737420626520746865206669727374C7
:106DE00020667261676D656E7421000073616E6963
:106DF000747920636865636B0000000076616C69DC
:106E0000646174655F646174616772616D3A6E6537
:106E100078745F70627566213D4E554C4C000000E1
:106E200070B504460D460E480068A04203D10C49D7
:106E3000206808600EE000BF002D08D100BF09A344
:106E400040F2451216A11DA0FCF7BEFE00BF00BF18
:106E5000206828602146042001F074F870BD00000D
:106E6000D8C001202E2E2F4D6964646C6577617245
:106E700065732F54686972645F50617274792F4C26
:106E80007749502F7372632F636F72652F69707625
:106E9000342F6970345F667261672E6300000000F2
:106EA00073616E69747920636865636B206C696EC9
:106EB0006B6564206C697374000000004173736536
:106EC0007274696F6E2022257322206661696C6579
:106ED00064206174206C696E6520256420696E20D1
:106EE00025730A0070B505460E46042001F0F8F837
:106EF000044664B93146284600F00EF9B04203DB7F
:106F0000042001F0EDF804460CB9002070BD2021EA
:106F10002046F9F722FA0F20E07706480068206043
:106F2000044804601422294604F10800F9F7EEF938
:106F30002046EBE7D8C001202DE9F04704468846FB
:106F4000002500BFA04507D100BF40A3AB224EA142
:106F500050A0FCF739FE00BF00BFB8F1000F0DD004
:106F600000BFD8F80000A04207D000BF37A3AD2271
:106F700052A148A0FCF728FE00BF00BF6068D0F80F
:106F80000490B9F80400002824D16768D9F80000FB
:106F90006060142204F108017868F9F7B7F901215B
:106FA0003846FFF731F8384602F0F0F9064600BFE0
:106FB000A819B0F5803F07DB00BF24A3BC2244A181
:106FC00034A0FCF701FE00BF00BFA81985B2384607
:106FD00002F0F2FB67681CE0D7F80490BA46D9F8D3
:106FE0000070504602F0D2F9064600BFA819B0F56D
:106FF000803F07DB00BF15A3CC2235A125A0FCF7FD
:10700000E3FD00BF00BFA81985B2504602F0D4FBD3
:1070100000BF002FE0D141462046FFF701FF00BF2F
:1070200033480088A84207DA00BF08A3D22231A162
:1070300018A0FCF7C9FD00BF00BF2D480088401B09
:107040002B4908802846BDE8F08700002E2E2F4DE2
:107050006964646C6577617265732F5468697264E2
:107060005F50617274792F4C7749502F7372632F80
:10707000636F72652F697076342F6970345F667242
:1070800061672E63000000007072657620213D204C
:1070900069707200417373657274696F6E20222586
:1070A0007322206661696C6564206174206C696E6E
:1070B0006520256420696E2025730A00707265764C
:1070C0002D3E6E657874203D3D2069707200000091
:1070D00070627566735F6672656564202B20636CF1
:1070E000656E203C3D2030786666666600000000D4
:1070F000DCC0012069705F72656173735F706275D7
:1071000066636F756E74203E3D2070627566735FB6
:1071100066726565640000002DE9F84F05468946F2
:10712000002700BF0026B2460020009083461B487F
:10713000046821E06069E968884207D1A06929698B
:10714000884203D1A089A988884201D0012000E0AB
:10715000002068B10BF1010B1EB92646CDF800A046
:1071600006E0E07FF17F884202DC2646CDF800A0F1
:10717000206800B1A2462468002CDBD12EB1304635
:107180000099FFF7D9FE804647444F4502DABBF12C
:10719000010FC7DC3846BDE8F88F0000D8C00120D9
:1071A00070B500250A4804680FE0E07F002805DD7F
:1071B000E07F401EE0772546246806E026462468E6
:1071C00029463046FFF7B8FE00BF002CEDD170BD58
:1071D000D8C0012070B505462C4600BF002C08D150
:1071E00000BF0FA340F2CE221CA11FA0FCF7ECFCB5
:1071F00000BF00BF00BFAC4208D000BF08A340F2F0
:10720000CF2223A118A0FCF7DFFC00BF00BF6069FC
:1072100010B1606902F0D0FA2046FFF733FC70BD70
:107220002E2E2F4D6964646C6577617265732F54DF
:10723000686972645F50617274792F4C7749502F7E
:107240007372632F636F72652F697076342F697064
:10725000345F667261672E63000000007063722005
:10726000213D204E554C4C00417373657274696F1B
:107270006E2022257322206661696C65642061742A
:10728000206C696E6520256420696E2025730A00D4
:10729000706372203D3D2070000000002DE9F04138
:1072A000A2B004460027B8460026642109A8F9F7D1
:1072B00054F86B486B49086000208DF81C00802052
:1072C0008DF81D00E1208DF81E0000208DF81F00B4
:1072D0008DF8200088208DF8210007A848604FF421
:1072E0000001604881606049C160604901614FF4FC
:1072F000C0614161FAF734FBC0B28DF81F00FAF7A4
:1073000035FBC0B28DF82000FAF736FBC0B28DF81D
:10731000210007A8534948600846F9F7A5FD07462C
:1073200038215348F9F719F82120514908604FF4E2
:1073300040004861002008614E4800F0BBFE062076
:1073400084F82C0047484068007884F826004548B7
:1073500040684178272001554248406881782820BC
:10736000015540484068C178292001553D48406892
:1073700001792A2001553B48406841792B2001556D
:1073800040F2DC50A08494F82D0040F00A0084F80C
:107390002D000322002101200BF080FF36490860F8
:1073A0000322002101200BF079FF344908601C22E0
:1073B00033496846F8F7AAFF2146684601F0BAFC4F
:1073C00030493148FBF705FE2F48FBF793FD002FAE
:1073D00041D12D48FBF719FD0646012E06DC20465B
:1073E00001F004FA204601F097F936E0022E06D0AB
:1073F000032E09D0042E0BD0052E11D10DE04FF431
:1074000000654FF4804810E000254FF480480CE000
:107410004FF400654FF0000807E00025A84604E09F
:107420004FF400654FF4804800BF00BF09A90D4824
:10743000F9F708FC0F95CDF8388009A90948F9F744
:1074400065FF0848F9F7AEFF204601F09FFA204695
:1074500001F032FA01E0F9F74CFB22B0BDE8F0810F
:10746000008002406C4C0020CC4B00202C4B0020B4
:107470001C4D00209C4201081CC0012020C001209E
:10748000A842010824C00120544D002038B504460C
:10749000002000900448007818B969460348F9F7BD
:1074A000F8FD009838BD000018C001206C4C002089
:1074B0002DE9F0418CB080460D46002400260027BF
:1074C00030216846F8F749FF30216846F8F745FF54
:1074D0002E4629E0042C04D36FF00B000CB0BDE85D
:1074E000F08104EB440170684DF82100708904EBD1
:1074F00044016A4602EB8101486054B104EB440048
:10750000694601EB8001601E00EB400002EB800049
:107510008160306830B9002004EB44016A4602EB18
:1075200081018860641C3668002ED3D128890D49FA
:107530004860C1F808D008464563284602F04CFB75
:1075400008490948F9F7F8FF00BF4FF0FF31074835
:10755000006801F0BBFB0028F7D10348F9F74FFEA4
:107560003846BBE71C4D00206C4C002020C0012099
:107570002DE9F041044625466868804703F0DCF9B0
:1075800006460D49286809684718B81BB0F1004F36
:1075900001D3012000E0002030B12968881922467B
:1075A000064903F051FA04E022460449384603F044
:1075B0004BFABDE8F0810000A800002071750008BA
:1075C0000146080601F47F4240EA022001F47F02EE
:1075D00040EA122040EA1160704701460806000C9C
:1075E00040EA11207047000008B50020009000BF5D
:1075F0006846804208D000BF0CA340F251121749E0
:1076000017A0FCF7E1FA00BF00BF00BF00BF03F006
:107610003BF900F063F900F03DFD00F0D5FF0BF001
:10762000B9F804F067FC03F0AFFA08BD2E2E2F4D19
:107630006964646C6577617265732F5468697264FC
:107640005F50617274792F4C7749502F7372632F9A
:10765000636F72652F696E69742E63008C44010834
:10766000417373657274696F6E20222573222066E0
:1076700061696C6564206174206C696E65202564A5
:1076800020696E2025730A00FAF788F9FCF7D6F80E
:10769000FBF752FDFBF7D6FFFBF7B2FFFBF7E0FC71
:1076A000FEF7BCF90C210448FBF71AFBFBF7A8FC1A
:1076B00001F0D8F900BFFEE798C301200146002081
:1076C000842901D0CA1C10447047000070B50546DB
:1076D00005B970BD05F00300002813D000BF00BF3E
:1076E0003DA340F2732248A150A0FCF76DFA00BF01
:1076F00000BF00BF03F088F80646304603F090F85C
:1077000000BFE6E7A5F1080452480068844205D3AB
:1077100005F10C0050490968884213D900BF00BF29
:107720002DA340F27F224DA140A0FCF74DFA00BFEF
:1077300000BF00BF03F068F80646304603F070F85B
:1077400000BFC6E74C4803F0D9F82079002816D1CD
:1077500000BF00BF20A34FF4237248A133A0FCF761
:1077600033FA00BF00BF444803F0E0F800BF03F065
:107770004BF80646304603F053F800BFA9E7204611
:1077800000F026F9002816D100BF00BF12A340F276
:10779000952244A125A0FCF717FA00BF00BF364888
:1077A00003F0C4F800BF03F02FF80646304603F09C
:1077B00037F800BF8DE700202071474800688442F9
:1077C00001D245480460204602F0D4FA2A4803F06A
:1077D000ADF800BF7DE700002E2E2F4D6964646C6C
:1077E0006577617265732F54686972645F50617266
:1077F00074792F4C7749502F7372632F636F7265C2
:107800002F6D656D2E6300006D656D5F6672656539
:107810003A2073616E69747920636865636B2061D7
:107820006C69676E6D656E7400000000417373656E
:107830007274696F6E2022257322206661696C65FF
:1078400064206174206C696E6520256420696E2057
:1078500025730A0040000020440000206D656D5F24
:10786000667265653A20696C6C6567616C206D6550
:107870006D6F727900000000480000206D656D5F3B
:10788000667265653A20696C6C6567616C206D6530
:107890006D6F72793A20646F75626C6520667265EF
:1078A000650000006D656D5F667265653A20696C04
:1078B0006C6567616C206D656D6F72793A206E6FD3
:1078C0006E2D6C696E6B65643A20646F75626C65D1
:1078D00020667265650000004C00002010B500BFF6
:1078E00000BF194820F003001849086008460468E2
:1078F0004FF4C86020800020608020714FF4C86081
:1079000002F040FE124908600120096808714FF436
:10791000C8600F49096808800D49096848800B480C
:1079200000680C4908600C4802F0F0FF00280AD0FB
:1079300000BF00BF09A340F21F2214A11AA0FCF748
:1079400043F900BF00BF10BDAB4D01204000002037
:10795000440000204C000020480000202E2E2F4D17
:107960006964646C6577617265732F5468697264C9
:107970005F50617274792F4C7749502F7372632F67
:10798000636F72652F6D656D2E6300006661696CB3
:10799000656420746F20637265617465206D656D28
:1079A0005F6D757465780000417373657274696FFB
:1079B0006E2022257322206661696C6564206174E3
:1079C000206C696E6520256420696E2025730A008D
:1079D0002DE9F0410446204600F084F90546208850
:1079E00002F0D0FD0646608802F0CCFD07462088F4
:1079F000B0F5C86F10D86088B0F5C86F0CD8608833
:107A0000A84202D03888A84206D1064800688642BB
:107A100005D07088A84202D00020BDE8F081012086
:107A2000FBE70000440000202DE9F0478146B9F152
:107A3000000F02D10020BDE8F08709F1030020F01B
:107A4000030085B20C2D00D20C25B5F5C86F01D806
:107A50004D4501DA0020EEE75C4802F04FFF5C483C
:107A6000006800F03FF90646A6E0304602F08AFDC5
:107A70000446207900287CD1218806F10800081AE4
:107A8000A84276D3218806F10800091A05F11400EE
:107A9000814229D306F1080028441FFA80F800BF6C
:107AA000B8F5C86F08D100BF4AA340F2873255A18C
:107AB00059A0FCF789F800BF00BF404602F062FD04
:107AC000074600213971218839807E80A4F8008022
:107AD000012020713888B0F5C86F07D0388802F0CF
:107AE00051FDA0F8028001E00120207138480068B3
:107AF000844227D13648D0F800A004E0BAF800004C
:107B000002F040FD82469AF8040018B14C48006823
:107B10008245F3D12E48C0F800A000BF0068484954
:107B2000096888420CD02A480068007940B100BF3B
:107B300028A340F2B53243A137A0FCF745F800BFB7
:107B400000BF00BF214802F0F1FE00BF04F10800B1
:107B500028443B490968884208D900BF1DA340F268
:107B6000B9323FA12CA0FCF72FF800BF00BF00BF27
:107B700000E01DE004F0030040B100BF15A340F297
:107B8000BB3243A124A0FCF71FF800BF00BF00BF19
:107B900004F0030040B100BF0EA340F2BD3248A183
:107BA0001DA0FCF711F800BF00BF04F1080042E778
:107BB000304602F0E7FC0688C5F5C860B0423FF6E3
:107BC00054AF024802F0B2FE002034E74800002023
:107BD0004C0000202E2E2F4D6964646C6577617215
:107BE00065732F54686972645F50617274792F4CA9
:107BF0007749502F7372632F636F72652F6D656DB8
:107C00002E630000696E76616C6964206E6578741D
:107C10002070747200000000417373657274696FA4
:107C20006E2022257322206661696C656420617470
:107C3000206C696E6520256420696E2025730A001A
:107C4000440000206D656D5F6D616C6C6F633A2060
:107C5000216C667265652D3E7573656400000000D9
:107C60006D656D5F6D616C6C6F633A20616C6C6FFC
:107C70006361746564206D656D6F7279206E6F74D9
:107C80002061626F76652072616D5F656E642E00A3
:107C90006D656D5F6D616C6C6F633A20616C6C6FCC
:107CA0006361746564206D656D6F72792070726FA9
:107CB0007065726C7920616C69676E65642E000076
:107CC0006D656D5F6D616C6C6F633A2073616E6999
:107CD000747920636865636B20616C69676E6D659C
:107CE0006E740000014602480088081A80B270478E
:107CF000400000202DE9F84F81468B460BF1030030
:107D000020F0030085B20C2D00D20C25B5F5C86F0C
:107D100001D85D4502DA0020BDE8F88F00BF5C485D
:107D20000068814503D35B480068814508D300BFE4
:107D300059A340F2D12264A169A0FBF745FF00BF1F
:107D400000BF53480068814503D35248006881450D
:107D500009D300BF02F058FD0090009802F060FDCA
:107D600000BF4846D8E7A9F108063046FFF7BAFF3A
:107D700007463188C81B08381FFA80FA00BF5545EE
:107D800008DD00BF44A34FF439725FA154A0FBF794
:107D90001BFF00BF00BF554501DD0020BCE7554576
:107DA00001D14846B8E7604802F0A8FD308802F0EB
:107DB000E9FB04462079002833D100BF3088B0F5B4
:107DC000C86F08D100BF34A340F2F52257A144A0E8
:107DD000FBF7FAFE00BF00BF2088009007F1080003
:107DE00028441FFA80F856480068A04204D1404653
:107DF00002F0C8FB52490860404602F0C3FB04464B
:107E000000202071009820806780A6F800802088DC
:107E1000B0F5C86F04D0208802F0B4FBA0F802804F
:107E200031E005F1140050452DD807F10800284431
:107E30001FFA80F800BF3088B0F5C86F08D100BFC6
:107E400015A340F2163239A125A0FBF7BDFE00BFF5
:107E500000BF404602F096FB044639480068844261
:107E600001D237480460002020713088208067806C
:107E7000A6F800802088B0F5C86F04D0208802F0F2
:107E800081FBA0F80280284802F050FD484643E7F5
:107E900040000020440000202E2E2F4D6964646CA9
:107EA0006577617265732F54686972645F5061729F
:107EB00074792F4C7749502F7372632F636F7265FB
:107EC0002F6D656D2E6300006D656D5F7472696D59
:107ED0003A206C6567616C206D656D6F727900008A
:107EE000417373657274696F6E2022257322206658
:107EF00061696C6564206174206C696E652025641D
:107F000020696E2025730A006D656D5F7472696D5E
:107F10002063616E206F6E6C7920736872696E6B7E
:107F2000206D656D6F72790048000020696E766182
:107F30006C6964206E6578742070747200000000B3
:107F40004C00002070B504460D4600BF0D2C09DB27
:107F500000BF0AA34FF4D57214A11BA0FBF734FE97
:107F600000BF70BD00BF05B9FBE7214951F82400EF
:107F70002946FCF755FB00BFF3E700002E2E2F4DDE
:107F80006964646C6577617265732F5468697264A3
:107F90005F50617274792F4C7749502F7372632F41
:107FA000636F72652F6D656D702E63006D656D700A
:107FB0005F667265653A2074797065203C204D4596
:107FC0004D505F4D41580000417373657274696F85
:107FD0006E2022257322206661696C6564206174BD
:107FE000206C696E6520256420696E2025730A0067
:107FF0008843010870B504460D4600BF002C08D127
:1080000000BF09A340F2951213A118A0FBF7DCFDF5
:1080100000BF00BF04B105B970BD29462046FCF77A
:10802000FFFA00BFF8E700002E2E2F4D6964646C44
:108030006577617265732F54686972645F5061720D
:1080400074792F4C7749502F7372632F636F726569
:108050002F6D656D702E6300696E76616C696420AA
:10806000706F6F6C2064657363000000417373650B
:108070007274696F6E2022257322206661696C65B7
:1080800064206174206C696E6520256420696E200F
:1080900025730A0010B5002406E0054951F82400B4
:1080A00000F008F8601C84B20D2CF6D310BD00005F
:1080B0008843010810B50023846823604368DB1CF3
:1080C00023F00301002207E083681B680B608368CC
:1080D000196003881944521C43889342F4DC10BD94
:1080E00070B5044600BF0D2C0ADB00BF09A340F2A7
:1080F000571214A11BA0FBF767FD00BF002070BD45
:1081000000BF224951F82400FCF7E8FA054628464A
:10811000F5E700002E2E2F4D6964646C657761725F
:1081200065732F54686972645F50617274792F4C63
:108130007749502F7372632F636F72652F6D656D72
:10814000702E63006D656D705F6D616C6C6F633A6E
:108150002074797065203C204D454D505F4D41584D
:1081600000000000417373657274696F6E202225F0
:108170007322206661696C6564206174206C696E8D
:108180006520256420696E2025730A008843010854
:1081900010B5044600BF002C08D100BF07A34FF460
:1081A0009E7212A116A0FBF70FFD00BF00BF0CB915
:1081B000002010BD2046FCF791FAFAE72E2E2F4D35
:1081C0006964646C6577617265732F546869726461
:1081D0005F50617274792F4C7749502F7372632FFF
:1081E000636F72652F6D656D702E6300696E7661C9
:1081F0006C696420706F6F6C2064657363000000AD
:10820000417373657274696F6E2022257322206634
:1082100061696C6564206174206C696E65202564F9
:1082200020696E2025730A002DE9F05F04460E4692
:1082300017469846DDE90AB900BF002C0BD100BFF4
:1082400049A340F2271255A15BA0FBF7BDFC00BF7C
:108250000020BDE8F09F00BF00BFB9F1000F0AD1B8
:1082600000BF41A34FF494725DA153A0FBF7ACFC97
:1082700000BF0020EDE700BF06B9624E07B9614FAD
:10828000B8F1000F01D1DFF87C8100206060A060B0
:10829000E0605D4860610020A08484F82D00E0610A
:1082A000C4F820B05948007884F830000C98206158
:1082B00043463A463146204600F0F8F92046C84782
:1082C00008B10020C5E700BF94F83000FF2802D1B4
:1082D000002084F830004FF0000A4D48056829E07E
:1082E00000BFA54208D100BF1FA340F28B1249A1D5
:1082F00031A0FBF769FC00BF00BF0AF1010A00BF13
:10830000BAF1FF0F08DD00BF17A340F28D1246A19E
:1083100029A0FBF759FC00BF00BF95F8300094F886
:108320003010884205D194F83000401C84F83000A9
:1083300002E02D68002DD3D100BF002DC4D194F8E8
:108340003000FE2803D100203049087004E094F882
:108350003000401C2D4908702D48006820602C48D2
:108360000460204675E700002E2E2F4D6964646C72
:108370006577617265732F54686972645F506172CA
:1083800074792F4C7749502F7372632F636F726526
:108390002F6E657469662E63000000006E65746957
:1083A000665F6164643A20696E76616C6964206E10
:1083B0006574696600000000417373657274696FCB
:1083C0006E2022257322206661696C6564206174C9
:1083D000206C696E6520256420696E2025730A0073
:1083E0006E657469665F6164643A204E6F20696EE1
:1083F00069742066756E6374696F6E20676976654F
:108400006E00000028440108A586000858000020DE
:10841000500000206E6574696620616C726561644D
:108420007920616464656400746F6F206D616E799A
:10843000206E65746966732C206D61782E207375CB
:1084400070706F72746564206E756D6265722069FC
:10845000732032353500000070B504460D462946BC
:10846000204604F04BFD294620460AF061FB70BD12
:1084700010B503460868DC68A04201D1012000E085
:10848000002030B909B9002000E00868D860012058
:1084900010BD0020FCE70000F8B505460C46164666
:1084A00000BF002C08D100BF18A340F2CB1224A1BA
:1084B00027A0FBF789FB00BF00BF00BF46B900BF84
:1084C00012A34FF4E6721EA121A0FBF77DFB00BFB3
:1084D00000BF20686968884201D1012000E00020C7
:1084E00090B9206800906868306069463046FFF7B0
:1084F000B3FF0CB9002000E0206868600121284625
:1085000000F064F80120F8BD0020FCE72E2E2F4D6E
:108510006964646C6577617265732F54686972640D
:108520005F50617274792F4C7749502F7372632FAB
:10853000636F72652F6E657469662E6300000000BC
:10854000696E76616C696420706F696E7465720023
:10855000417373657274696F6E20222573222066E1
:1085600061696C6564206174206C696E65202564A6
:1085700020696E2025730A0010B5034608689C68C0
:10858000A04201D1012000E0002030B909B900204B
:1085900000E008689860012010BD0020FCE70000A2
:1085A00002466AB10748016808E091F83000401CB3
:1085B000C0B2904201D10846704709680029F4D141
:1085C0000020F9E7500000207047000070B5044615
:1085D0000D4600BF002C08D100BF12A340F26D323F
:1085E0001DA126A0FBF7F0FA00BF00BF94F82D00F4
:1085F00000F0040020B194F82D0000F0010000B953
:1086000070BD05F0010050B1606840B194F82D00D4
:1086100000F0080018B1211D2046FCF7FBFE00BF4A
:10862000EEE700002E2E2F4D6964646C6577617251
:1086300065732F54686972645F50617274792F4C4E
:108640007749502F7372632F636F72652F6E657455
:1086500069662E63000000006E657469665F697369
:108660007375655F7265706F7274733A20696E76A8
:10867000616C6964206E657469660000417373659E
:108680007274696F6E2022257322206661696C65A1
:1086900064206174206C696E6520256420696E20F9
:1086A00025730A0003466FF00B0070472DE9F84F61
:1086B00080460C4615461E464FF00009CA4604B9CE
:1086C000114C05B9104D06B90F4E0CB1206808B910
:1086D000012000E00020074627B16A4621464046B7
:1086E000FFF7DAFE4A4629464046FFF745FF524665
:1086F00031464046FFF7BCFE27B96A462146404650
:10870000FFF7CAFEBDE8F88F284401080149086058
:10871000704700005400002010B5044600BF002C34
:1087200009D100BF10A340F29B321CA123A0FBF78C
:108730004BFA00BF10BD00BF94F82D0000F00100FF
:1087400078B100BF94F82D0000F0FE0084F82D00F1
:1087500000BF94F82D0000F0080010B12046FCF78F
:1087600021F800BFE6E700002E2E2F4D6964646CEF
:108770006577617265732F54686972645F506172C6
:1087800074792F4C7749502F7372632F636F726522
:108790002F6E657469662E63000000006E65746953
:1087A000665F7365745F646F776E3A20696E766199
:1087B0006C6964206E6574696600000041737365BE
:1087C0007274696F6E2022257322206661696C6560
:1087D00064206174206C696E6520256420696E20B8
:1087E00025730A0000B1C1617047000010B504464E
:1087F00000BF002C09D100BF0FA340F206421BA10D
:1088000023A0FBF7E1F900BF10BD00BF94F82D00D5
:1088100000F0040070B100BF94F82D0000F0FB00E0
:1088200084F82D0000BF00BFE06910B12046E16967
:10883000884700BF00BFE7E72E2E2F4D6964646CA8
:108840006577617265732F54686972645F506172F5
:1088500074792F4C7749502F7372632F636F726551
:108860002F6E657469662E63000000006E65746982
:10887000665F7365745F6C696E6B5F646F776E3A89
:1088800020696E76616C6964206E657469660000AB
:10889000417373657274696F6E202225732220669E
:1088A00061696C6564206174206C696E6520256463
:1088B00020696E2025730A0010B5044600BF002C05
:1088C00009D100BF11A34FF478721DA125A0FBF7B9
:1088D0007BF900BF10BD00BF94F82D0000F004002C
:1088E00090B900BF94F82D0040F0040084F82D00EA
:1088F00000BF03212046FFF769FE00BFE06910B109
:108900002046E169884700BF00BFE3E72E2E2F4DC8
:108910006964646C6577617265732F546869726409
:108920005F50617274792F4C7749502F7372632FA7
:10893000636F72652F6E657469662E6300000000B8
:108940006E657469665F7365745F6C696E6B5F7585
:10895000703A20696E76616C6964206E6574696630
:1089600000000000417373657274696F6E202225E8
:108970007322206661696C6564206174206C696E85
:108980006520256420696E2025730A0010B5044611
:1089900000BF002C09D100BF0EA34FF454721AA1DE
:1089A00020A0FBF711F900BF10BD00BF94F82D0007
:1089B00000F0010058B900BF94F82D0040F001000C
:1089C00084F82D0000BF03212046FFF7FFFD00BF04
:1089D000EAE700002E2E2F4D6964646C65776172A2
:1089E00065732F54686972645F50617274792F4C9B
:1089F0007749502F7372632F636F72652F6E6574A2
:108A000069662E63000000006E657469665F7365B9
:108A1000745F75703A20696E76616C6964206E656A
:108A200074696600417373657274696F6E202225E4
:108A30007322206661696C6564206174206C696EC4
:108A40006520256420696E2025730A0070B50446F0
:108A500025460DB1294600E0012108460AF0D0F96B
:108A6000002070BD10B50AF099FA002010BD10B5B5
:108A7000FDF7D3FA10B10BF09FF910BD0BF096F98A
:108A8000FBE7F8B504460D46A06840B1E06830B198
:108A90000020009094E80F000AF02DFCF8BD0022A1
:108AA000D4E900010AF0FAFBF8E700002DE9FF41E4
:108AB00007460D4614460295002001903DB98020DE
:108AC00000909DE8070087E80700BDE8FF810020CF
:108AD00003900026601C08B9761E03E014B12646F8
:108AE00006B90126FDF799FAB0B103AA01A92846F3
:108AF0000AF034FF012802D11020009001E000208C
:108B000000900398B8B14FF080500E490860BFF351
:108B10004F8FBFF36F8F0EE0324601A928460AF04F
:108B200069FE012802D11020009004E00EB9002057
:108B300000E0402000909DE8070087E8070000BFA4
:108B4000C3E7000004ED00E077B581B006461446A7
:108B500000200090254605B90125FDF75EFAA8B171
:108B600000236A4602A930460AF056FD012802D0C9
:108B7000FF2004B070BD009890B14FF080500949BB
:108B80000860BFF34F8FBFF36F8F09E000232A46C1
:108B900002A930460AF06CFC012801D0FF20E8E76A
:108BA0000020E6E704ED00E010B50446606820B15F
:108BB000012061680AF05DFB10BD01200AF048FB4E
:108BC000FAE7000038B50446002500200090FDF7C4
:108BD00024FA90B1694620460AF09CFD012801D094
:108BE000FF2038BD009888B14FF0805008490860D8
:108BF000BFF34F8FBFF36F8F08E000231A4619466B
:108C000020460AF035FC012800D0FF252846E8E779
:108C100004ED00E0F8B506460C46002000900EB9C1
:108C20008020F8BD0025601C08B96D1E03E014B15A
:108C3000254605B90125FDF7F0F998B16A460021EE
:108C400030460AF08BFE012801D0FF20E9E70098AA
:108C500080B14FF0805008490860BFF34F8FBFF3D9
:108C60006F8F07E0294630460AF0DEFE012801D06A
:108C7000FF20D6E70020D4E704ED00E038B5044635
:108C8000002500200090FDF7C8F990B16946204604
:108C90000AF040FD012801D0FF2038BD009888B1BE
:108CA0004FF0805008490860BFF34F8FBFF36F8FBC
:108CB00008E000231A46194620460AF0D9FB01288D
:108CC00000D0FF252846E8E704ED00E0F8B50646A9
:108CD0000C46002000900EB98020F8BD0025601CD5
:108CE00008B96D1E03E014B1254605B90125FDF74D
:108CF00094F998B16A46002130460AF02FFE012807
:108D000001D0FF20E9E7009880B14FF0805008497A
:108D10000860BFF34F8FBFF36F8F07E029463046DF
:108D20000AF082FE012801D0FF20D6E70020D4E718
:108D300004ED00E07FB504460D46606998B1A06976
:108D400088B1B4F90800FEF7B9FC0646D4E905106D
:108D5000CDE9006102902B462269D4E900100AF0A7
:108D6000B7FF039013E0B4F90800FEF7A7FC06462E
:108D700003A8CDE90060238A9AB22B46D4E90010FB
:108D80000AF074FF012802D0002004B070BD0398DF
:108D9000FBE770B504460D4600222946204600F048
:108DA00001F870BD2DE9F04704460D46904600BF1E
:108DB00044B900BF1CA340F2DF1227A129A0FAF793
:108DC00003FF00BF00BF14B1B5F5803F02D30120FF
:108DD000BDE8F0870DB90020FAE7AEB22089304433
:108DE00080B2B04201DA0120F2E794F80C9009F069
:108DF000800038B16068471B04F11000874209D237
:108E00000120E5E7B8F1000F02D06068471B01E0E0
:108E10000120DDE76760608930446081208930444B
:108E200020810020D4E700002E2E2F4D6964646C51
:108E30006577617265732F54686972645F506172FF
:108E400074792F4C7749502F7372632F636F72655B
:108E50002F706275662E63007020213D204E554CA8
:108E60004C000000417373657274696F6E20222597
:108E70007322206661696C6564206174206C696E80
:108E80006520256420696E2025730A002DE9FE4FB8
:108E900082460E4690465746B8F1010F0AD0B8F107
:108EA000410F06D0B8F5C17F0BD0B8F5207F7DD13A
:108EB0006AE000BF42463146002000F037F9044620
:108EC000AEE0002400200290B14600BF0C20FFF766
:108ED00007F9054645B900F0A9FD14B1204600F098
:108EE0006BFC0020BDE8FE8FF81C20F00300C0F5ED
:108EF000147080B2484501DD484605E0F81C20F0BA
:108F00000300C0F5147080B283460020CDE90080D4
:108F100005F110003844C01C20F003015B464A46AE
:108F2000284600F074FD00BF287900F003000028F7
:108F300008D000BF3CA34FF4807247A152A0FAF7BB
:108F400043FE00BF00BF00BFF81C20F00300C0F5C7
:108F50001470002808D100BF33A34FF4817254A1CC
:108F600049A0FAF731FE00BF00BF0CB92C4601E062
:108F7000029805600295A9EB0B001FFA80F9002703
:108F8000B9F1000FA2DC4BE0F81C20F00301F01C4B
:108F900020F00300084485B205F110001FFA80F9A3
:108FA000F01C20F00300A84206D800E02BE0F01CE3
:108FB00020F00300484501D9002093E74846FEF71A
:108FC00033FD04460CB900208CE70020CDE9008079
:108FD00004F110003844C01C20F00301334632462F
:108FE000204600F014FD00BF207900F0030040B1DE
:108FF00000BF0DA34FF491723AA123A0FAF7E4FD4C
:1090000000BF00BF0CE000BF00BF07A340F2271263
:109010003FA11DA0FAF7D8FD00BF00BF002061E707
:1090200000BF20465EE700002E2E2F4D6964646C61
:109030006577617265732F54686972645F506172FD
:1090400074792F4C7749502F7372632F636F726559
:109050002F706275662E6300706275665F616C6C5E
:109060006F633A207062756620712D3E7061796C75
:109070006F61642070726F7065726C7920616C69C9
:10908000676E656400000000417373657274696FF8
:109090006E2022257322206661696C6564206174EC
:1090A000206C696E6520256420696E2025730A0096
:1090B000504255465F504F4F4C5F42554653495AB8
:1090C00045206D75737420626520626967676572FB
:1090D000207468616E204D454D5F414C49474E4DAF
:1090E000454E5400706275665F616C6C6F633A2028
:1090F000706275662D3E7061796C6F61642070726C
:109100006F7065726C7920616C69676E65640000D0
:10911000706275665F616C6C6F633A206572726F26
:109120006E656F7573207479706500002DE9FC41E0
:1091300007460D46144600BF412C0AD0012C08D02A
:1091400000BF0EA34FF4A57218A11DA0FAF73CFDB5
:1091500000BF00BF0B20FEF7C3FF064616B9002074
:10916000BDE8FC8100202B462A463946CDE9004067
:10917000304600F04CFC3046F2E700002E2E2F4D1A
:109180006964646C6577617265732F546869726491
:109190005F50617274792F4C7749502F7372632F2F
:1091A000636F72652F706275662E6300696E7661FB
:1091B0006C696420706275665F7479706500000088
:1091C000417373657274696F6E2022257322206665
:1091D00061696C6564206174206C696E652025642A
:1091E00020696E2025730A002DE9FC5F05460C46B8
:1091F00017469846DDE90C9BAA460AF1030020F0C9
:1092000003002044584502D90020BDE8FC9FB9F175
:10921000000F06D00AF1030020F0030000EB09065E
:1092200000E000260220234622463146CDE90070A8
:10923000404600F0ECFB4046E7E7000070B506460C
:109240000D4600BF0EB1002D09D100BF1BA340F297
:10925000593226A133A0FAF7B7FC00BF70BD00BF9A
:10926000344604E020892989084420812468206844
:109270000028F7D100BF20896189884208D000BF4B
:109280000EA340F2623231A126A0FAF79DFC00BF86
:1092900000BF00BF206840B100BF08A340F26332A6
:1092A00036A120A0FAF790FC00BF00BF20892989D1
:1092B00008442081256000BFD0E700002E2E2F4DEE
:1092C0006964646C6577617265732F546869726450
:1092D0005F50617274792F4C7749502F7372632FEE
:1092E000636F72652F706275662E63002868202197
:1092F0003D204E554C4C2920262620287420213D07
:10930000204E554C4C29202870726F6772616D6D2C
:1093100065722076696F6C617465732041504929CC
:1093200000000000417373657274696F6E2022251E
:109330007322206661696C6564206174206C696EBB
:109340006520256420696E2025730A00702D3E7407
:109350006F745F6C656E203D3D20702D3E6C656EB8
:1093600020286F66206C61737420706275662069B6
:109370006E20636861696E2900000000702D3E6EEA
:10938000657874203D3D204E554C4C000146002030
:1093900002E0421C90B209680029FAD1704700002F
:1093A0002DE9F04180460E4614462189324640465A
:1093B000FFF76CFD074617B90020BDE8F081214694
:1093C000384600F045F8054600BF45B100BF05A38B
:1093D00040F224520FA114A0FAF7F6FB00BF00BF21
:1093E0003846EAE72E2E2F4D6964646C657761720A
:1093F00065732F54686972645F50617274792F4C81
:109400007749502F7372632F636F72652F70627587
:10941000662E6300706275665F636F7079206661A7
:10942000696C656400000000417373657274696F54
:109430006E2022257322206661696C656420617448
:10944000206C696E6520256420696E2025730A00F2
:109450002DE9F04105460C460026002700BF25B146
:109460001CB12889218988420CDA00BF44A340F24C
:10947000C9324FA15AA0FAF7A7FB00BF6FF00F0047
:10948000BDE8F08100BF00BF6889801B6189C91BEE
:10949000884203D36089A0EB070802E06889A0EB4B
:1094A00006086268D1196A6890194246F6F72EFFDD
:1094B0004644474400BF6889B04208D200BF30A389
:1094C00040F2D93250A146A0FAF77EFB00BF00BFA0
:1094D00000BF6089B84208D200BF29A340F2DA3247
:1094E0004FA13FA0FAF770FB00BF00BF6089B842F0
:1094F00001D8002724686889B04211D100262D6860
:1095000000BF65B95CB100BF1DA34FF479724BA1D8
:1095100033A0FAF759FB00BF6FF00F00B0E700BFB0
:10952000002C13D06089218988420FD100BF2068A8
:1095300058B100BF12A340F2E93244A128A0FAF7C3
:1095400043FB00BF6FF005009AE700BF002D13D06A
:109550006889298988420FD100BF286858B100BFA7
:1095600007A340F2EE3239A11DA0FAF72DFB00BF90
:109570006FF0050084E700BF002C85D100207FE755
:109580002E2E2F4D6964646C6577617265732F545C
:10959000686972645F50617274792F4C7749502FFB
:1095A0007372632F636F72652F706275662E63002E
:1095B000706275665F636F70793A20746172676577
:1095C00074206E6F742062696720656E6F756768BE
:1095D00020746F20686F6C6420736F757263650010
:1095E000417373657274696F6E2022257322206641
:1095F00061696C6564206174206C696E6520256406
:1096000020696E2025730A006F66667365745F7447
:109610006F203C3D20705F746F2D3E6C656E0000C6
:109620006F66667365745F66726F6D203C3D207077
:109630005F66726F6D2D3E6C656E0000705F746FBB
:1096400020213D204E554C4C000000007062756694
:109650005F636F7079282920646F6573206E6F7463
:1096600020616C6C6F77207061636B65742071751D
:1096700065756573210000002DE9F05F804689461D
:1096800016461D464FF0000AD34600BFB8F1000F42
:109690000BD100BF21A340F20A422CA133A0FAF75C
:1096A00093FA00BF0020BDE8F09F00BF00BFB9F1F2
:1096B000000F0AD100BF19A340F20B4235A12BA025
:1096C000FAF782FA00BF0020EDE700BF444620E031
:1096D00035B16089A84203DC6089281A85B217E099
:1096E0006089401B87B2B74200DD37466268511976
:1096F00009EB0A003A46F6F709FE0BEB07001FFAE2
:1097000080FB0AEB07001FFA80FAF01B86B20025E7
:1097100024680EB1002CDBD15846C4E72E2E2F4D05
:109720006964646C6577617265732F5468697264EB
:109730005F50617274792F4C7749502F7372632F89
:10974000636F72652F706275662E63007062756656
:109750005F636F70795F7061727469616C3A2069E0
:109760006E76616C69642062756600004173736592
:109770007274696F6E2022257322206661696C65A0
:1097800064206174206C696E6520256420696E20F8
:1097900025730A00706275665F636F70795F706130
:1097A000727469616C3A20696E76616C69642064D8
:1097B00061746170747200002DE9F0470446002C5A
:1097C0000ED100BF44B900BF38A34FF4377243A194
:1097D00045A0FAF7F9F900BF00BF0020BDE8F08707
:1097E00000265EE001F010F8824600BFA07B002852
:1097F00008DC00BF2DA340F2F12245A13AA0FAF700
:10980000E3F900BF00BFA07B401E00F0FF0884F812
:109810000E80504601F004F8B8F1000F3FD12768E0
:10982000207B00F00F05607B00F00200002814D0C0
:10983000A14600BFD9F81000002808D100BF1BA323
:1098400040F2FF2238A128A0FAF7BEF900BF00BFFE
:109850002046D9F8101088471DE0022D04D121467A
:109860000C20FEF76FFB16E0012D04D121460B20E2
:10987000FEF768FB0FE01DB92046FDF727FF0AE061
:1098800000BF00BF09A340F20F3230A116A0FAF7C3
:109890009BF900BF00BF701CC6B23C4600E000242C
:1098A00000BF002C9ED1304698E700002E2E2F4D91
:1098B0006964646C6577617265732F54686972645A
:1098C0005F50617274792F4C7749502F7372632FF8
:1098D000636F72652F706275662E63007020213D84
:1098E000204E554C4C000000417373657274696FD3
:1098F0006E2022257322206661696C656420617484
:10990000206C696E6520256420696E2025730A002D
:10991000706275665F667265653A20702D3E72658D
:1099200066203E203000000070632D3E6375737426
:109930006F6D5F667265655F66756E6374696F6E85
:1099400020213D204E554C4C00000000696E766190
:109950006C6964207062756620747970650000001F
:1099600070B50446254629460748FEF743FB0748DD
:109970000078012806D100200449087004480068D6
:10998000FFF77CF970BD00009C42010818C001205F
:109990001CC0012070B500BF00F036FF0546002056
:1099A00009490870284600F03BFF00BF07480468DB
:1099B00006E0606F18B1204602F054FA70BDE4680A
:1099C000002CF6D100BFF9E7CCC001206C000020CC
:1099D00010B50446FFF7DEFF10BD70B504460D4616
:1099E00001222946204600F001F870BD70B50546F9
:1099F0000C461646002C04DA6142284600F040F975
:109A000070BD324621462846FFF7CCF9F8E770B51D
:109A1000DDE904450026066041600281438104734C
:109A20004573012686730026C67370BD70B500F0BD
:109A3000EBFE05460C48047801200B4908702846C7
:109A400000F0EEFE7CB900BF0021084808F040FE9F
:109A500040B100F0D9FE05460020034908702846B1
:109A600000F0DEFE00BF70BDCCC00120D19900081F
:109A70002DE9F04106460F4600BF002E08D100BF79
:109A80002CA34FF4CC7237A13CA0FAF79DF800BF8D
:109A900000BF3089B84201DCBDE8F0813089C01BCD
:109AA0001FFA80F83D46344613E06089281A85B2D3
:109AB0002089A0EB08002081246800BF44B900BFC2
:109AC0001CA340F2AF1237A12CA0FAF77DF800BF1B
:109AD00000BF6089A842E8DB207B00F00F0000286F
:109AE0001BD16089A84218D0607B00F002000028DA
:109AF00013D1A088001B284481B22046FEF7FAF853
:109B0000044600BF44B900BF0AA340F2BD122BA116
:109B10001AA0FAF759F800BF00BF6581608920815B
:109B2000206810B12068FFF747FE0020206000BFCA
:109B3000B2E700002E2E2F4D6964646C6577617268
:109B400065732F54686972645F50617274792F4C29
:109B50007749502F7372632F636F72652F70627530
:109B6000662E6300706275665F7265616C6C6F6310
:109B70003A207020213D204E554C4C0041737365B6
:109B80007274696F6E2022257322206661696C658C
:109B900064206174206C696E6520256420696E20E4
:109BA00025730A00706275665F7265616C6C6F6325
:109BB0003A207120213D204E554C4C006D656D5F63
:109BC0007472696D2072657475726E65642071209F
:109BD0003D3D204E554C4C0070B50446002C18D02D
:109BE00000BF00F011FE0546A07B401CA073284674
:109BF00000F016FE00BF00BFA07B002808DC00BFFD
:109C000004A340F242320FA113A0F9F7DDFF00BF19
:109C100000BF70BD2E2E2F4D6964646C6577617234
:109C200065732F54686972645F50617274792F4C48
:109C30007749502F7372632F636F72652F7062754F
:109C4000662E63007062756620726566206F7665A9
:109C500072666C6F77000000417373657274696F90
:109C60006E2022257322206661696C656420617410
:109C7000206C696E6520256420696E2025730A00BA
:109C80002DE9F04104460D4600BF44B900BF18A3BA
:109C900040F24B2222A125A0F9F796FF00BF00BF9A
:109CA00014B1B5F5803F02D30120BDE8F0810DB9B4
:109CB0000020FAE7AEB200BF6089B0420ADA00BF06
:109CC0000BA340F2552223A118A0F9F77DFF00BF96
:109CD0000120EAE700BF6768606828446060608927
:109CE000801B60812089801B20810020DDE700002F
:109CF0002E2E2F4D6964646C6577617265732F54E5
:109D0000686972645F50617274792F4C7749502F83
:109D10007372632F636F72652F706275662E6300B6
:109D20007020213D204E554C4C000000417373655E
:109D30007274696F6E2022257322206661696C65DA
:109D400064206174206C696E6520256420696E2032
:109D500025730A00696E6372656D656E745F6D616F
:109D6000676E6974756465203C3D20702D3E6C659E
:109D70006E0000002DE9F041044600BF3B4800683A
:109D8000844208D200BF3AA340F2DF1244A14AA0A5
:109D9000F9F71AFF00BF00BF00BF514800688442B6
:109DA00008D300BF32A34FF4F0724EA142A0F9F7DE
:109DB0000BFF00BF00BF00BF2079002808D000BF04
:109DC0002BA340F2E1124EA13BA0F9F7FDFE00BF2C
:109DD00000BF00BF2088B0F5C86F08D900BF24A31A
:109DE0004FF4F2724DA134A0F9F7EEFE00BF00BFB0
:109DF000208800F0C7FB0546AC4219D02879B8B9D5
:109E000037480068854213D04F480068A84201D106
:109E10004D480460288820802888B0F5C86F07D096
:109E20002046FDF75FFF0746288800F0ABFB478020
:109E3000608800F0A7FB0646A64215D0307998B995
:109E400041480068A04201D13F4806602088308028
:109E50002088B0F5C86F07D03046FDF743FF0746AE
:109E6000208800F08FFB4780BDE8F0814000002093
:109E70002E2E2F4D6964646C6577617265732F5463
:109E8000686972645F50617274792F4C7749502F02
:109E90007372632F636F72652F6D656D2E630000A3
:109EA000706C75675F686F6C65733A206D656D20C7
:109EB0003E3D2072616D0000417373657274696F7D
:109EC0006E2022257322206661696C6564206174AE
:109ED000206C696E6520256420696E2025730A0058
:109EE00044000020706C75675F686F6C65733A2082
:109EF0006D656D203C2072616D5F656E64000000D1
:109F0000706C75675F686F6C65733A206D656D2D59
:109F10003E75736564203D3D20300000706C7567B0
:109F20005F686F6C65733A206D656D2D3E6E657868
:109F300074203C3D204D454D5F53495A455F414C8F
:109F400049474E45440000004C0000202DE9F041F7
:109F500005460E461C4807681C480068001D08F0AE
:109F60000FFE50B91948006890F82C100120884065
:109F700017490968814316480160681C38B936B131
:109F800012480168091D134808F044FE1AE07C19C4
:109F90000E4800684460BC4207D20C480168091DA5
:109FA0000D48006808F01CFE0CE008480168091D17
:109FB0000A48006808F014FE09480068844201D28B
:109FC00007480460BDE8F08164C0012050C0012052
:109FD00068C00120B0C6012058C0012054C0012033
:109FE00080C0012010B5044608F020FE2348006818
:109FF000401C224908602248006840B9204804609B
:10A000000846006801280DD100F0BEF90AE01D489D
:10A01000006838B91A480068C06AE16A884201D805
:10A020001748046018480068401C1749086094F8F5
:10A030002C1001208840154909680843134908601D
:10A04000E16A01EB8101124A02EB8100211D08F057
:10A05000E1FD08F015FE0B48006868B1084800688B
:10A06000C06AE16A884207D24FF08050094908600F
:10A07000BFF34F8FBFF36F8F10BD000060C0012092
:10A0800050C001206CC001207CC0012068C00120AC
:10A09000E0C3012004ED00E010B516E008F0C6FDB5
:10A0A0000C48C068C468201D08F06AFD0A480068B2
:10A0B000401E0949086009480068401E07490860B9
:10A0C00008F0DEFD204600F05FF804480068002834
:10A0D000E4D110BD9CC6012060C001205CC00120FD
:10A0E00070B504460D46206C70B1216CE0680144E7
:10A0F000E160D4E90210884201D32168E16028467A
:10A10000226CE168F6F702F970BD2DE9F0410446D2
:10A110000F4615464FF00008A66B206C48B9206822
:10A1200000282CD1A06809F0F5FE80460020A06030
:10A1300025E07DB93946226C6068F6F7E7F8216CB6
:10A14000606808446060D4E90101884217D3206840
:10A15000606014E03946226CE068F6F7D7F8216CAD
:10A16000E068411AE1602168E068884203D2216C0E
:10A17000A068411AE160022D01D106B1761E701C63
:10A18000A0634046BDE8F08110B5044694F859003C
:10A1900030B9206B08F092FD204608F08FFD1AE0E0
:10A1A00094F85900012803D1204608F087FD12E0F9
:10A1B00094F85900022801D1012000E0002050B994
:10A1C00000BF502080F31188BFF34F8FBFF36F8F14
:10A1D00000BF00BFFEE710BD01464A6A22B10A6B0C
:10A1E0001268C2F1200000E00020704730B54FF443
:10A1F0008033174800F007042CB1C01D20F0070081
:10A20000134C041B1B1B0246124C22600024114DF0
:10A210006C60D018083820F007000F4C2060002434
:10A220000D4D2D686C600C4D2D682C601146441A44
:10A230004C60094C24680C60084D4C682C60084D3B
:10A240004C682C604FF00044064D2C6030BD00007F
:10A25000A84D002010000020180000202000002041
:10A260001C0000202C00002000BFFFF715FF06484F
:10A2700000680128F9D94FF0805004490860BFF305
:10A280004F8FBFF36F8FF0E7E0C3012004ED00E0D4
:10A2900010B5044654B10020A06020600021E160A8
:10A2A00000231A461946204609F0E2F810BD2DE9B0
:10A2B000F04106460D4617469846069C0DB92460A7
:10A2C00000E02760E66325640121204609F084F858
:10A2D000BDE8F0812DE9FF5F81460E469246DDE93B
:10A2E0000E7B109CAAF10100216B01EB800828F085
:10A2F000070808F0070008B9012000E0002050B965
:10A3000000BF502080F31188BFF34F8FBFF36F8FD2
:10A3100000BF00BFFEE786B1002507E0715D04F1D4
:10A3200034004155705D00B902E06D1C182DF5D365
:10A3300000BF00214B20015502E0002084F83400CA
:10A34000202F00D31F27E762E76400202065201D2F
:10A3500008F043FC04F1180008F03FFC2461C7F149
:10A360002000A06164620020606584F858004946BE
:10A370004046039A00F0C4F92060BBF1000F01D001
:10A38000CBF80040BDE8FF9F10B5002407E004EBC8
:10A3900084010F4A02EB810008F012FC641C202C9F
:10A3A000F5D30C4808F00CFC0B4808F009FC0B48EE
:10A3B00008F006FC0A4808F003FC0A4808F000FC14
:10A3C00004480949086004480849086010BD0000B5
:10A3D000E0C3012060C6012074C6012088C60120A8
:10A3E0009CC60120B0C6012054C0012058C00120E5
:10A3F00010B50146164800E0006803688B42FBD3A5
:10A400000246436813448B4204D143684C6823449A
:10A41000436001460A464B6813440468A34211D1C5
:10A420000C4C03682468A34208D04B680468646835
:10A4300023444B6003681B680B6005E0054B1B68F9
:10A440000B6001E003680B60884200D0016010BD22
:10A45000100000201800002070B5054608F0E6FB4B
:10A46000A86B08B9012400E0002408F009FC20468C
:10A4700070BD70B5054608F0D9FBA86BE96B884242
:10A4800001D1012400E0002408F0FAFB204670BD51
:10A490000A490968096809B9012100E0002121B1D0
:10A4A0004FF0FF31064A116006E004490968C968A7
:10A4B000C868034A416811607047000054C0012019
:10A4C00080C001200E480068401C08B9012000E04F
:10A4D000002050B900BF502080F31188BFF34F8F88
:10A4E000BFF36F8F00BF00BFFEE700BF502080F3B7
:10A4F0001188BFF34F8FBFF36F8F00BF00BFFEE720
:10A500008CC0012070B5044608F090FB94F94550CA
:10A5100010E0606A08B9012000E0002038B904F1B9
:10A52000240009F0B7FD18B108F0A4FC00E003E036
:10A53000681E45B2002DECDC00BFFF2084F845000A
:10A5400008F09EFB08F072FB94F9445010E020697B
:10A5500008B9012000E0002048B904F1100009F01A
:10A5600099FD08B108F086FC681E45B200E001E0E4
:10A57000002DECDC00BFFF2084F8440008F080FBD5
:10A5800070BD0000014602480068084470470000A2
:10A59000400000202DE9F04104464FF0000808F08B
:10A5A00055FD4948006808B9FFF720FE4748006894
:10A5B0002040002870D1D4B1083404F00700B0B1B5
:10A5C00004F00700C0F10800044404F0070008B9D3
:10A5D000012000E0002050B900BF502080F3118816
:10A5E000BFF34F8FBFF36F8F00BF00BFFEE7002C9C
:10A5F00052D03748006884424ED8364E30460568FF
:10A6000001E02E462D686868A04202D22868002822
:10A61000F7D12D48006885423ED0306800F1080827
:10A62000286830606868001B102819D92F1907F0B6
:10A63000070008B9012000E0002050B900BF5020F9
:10A6400080F31188BFF34F8FBFF36F8F00BF00BF40
:10A65000FEE76868001B78606C603846FFF7C8FE4C
:10A660001B4968680968081A1949086008460068A3
:10A6700019490968884203D21548006816490860DC
:10A680001249686809680843686000202860134818
:10A690000068401C1149086009F048FD08F00700F7
:10A6A00008B9012000E0002050B900BF502080F31D
:10A6B0001188BFF34F8FBFF36F8F00BF00BFFEE75E
:10A6C0004046BDE8F0810000180000202C0000206A
:10A6D0001C0000201000002020000020240000208A
:10A6E0000648006830B10549096801F15000096D5C
:10A6F000491C0160014800687047000050C00120FB
:10A70000001F4FF080730360001F21F001030360FE
:10A71000001F054B036014380260001F6FF0020336
:10A720000360203870470000C5A40008F8B506464D
:10A730000C4615464FF47A702B46084A2146009085
:10A740003046F7F777FE10B14FF0FF30F8BD2A46DC
:10A7500002492046F5F7DAFD0020F7E77C9A012050
:10A76000F9F760FB00BF4FF4FA7008F049FBFAE715
:10A77000F9F7F4FE00BF002400BF06E0B2EE080ABD
:10A780002046F9F7FFFE601CC4B2102CF6DB6420F3
:10A7900008F036FBEFE7F8F703FE00F091FF00BF8B
:10A7A000642008F02DFBFBE7F0B587B004460D46AA
:10A7B0001646FEF75CF90746AEB1324601A821689D
:10A7C000FEF774F901A807C804AB07C30498102862
:10A7D00006D105982860FEF74AF9C01B07B0F0BD06
:10A7E0004FF0FF30FAE74FF0FF3201A82168FEF783
:10A7F0005DF901A807C804AB07C305982860FEF7F8
:10A8000036F9C01BEAE7000010B54FF0FF310348EE
:10A810000068FEF7FFF9012010BD0000B80000201D
:10A8200010B5044602480068FEF7CCF910BD0000E0
:10A83000B80000202DE9F04100F07EF8074600BF87
:10A840000F4804680CB9BDE8F0816068381AB0F1AF
:10A85000004F01D3012000E0002000B1F3E70849D8
:10A8600020680860A568E6680649606808602146B7
:10A870000A20FDF767FB0DB13046A847E0E700006E
:10A88000A4000020A800002010B50348FEF78CF9B2
:10A890000249086010BD000030440108B8000020E3
:10A8A0007FB504460D46094B0FCB8DE80F00009590
:10A8B00000216846FEF7E5F82060206818B94FF0DF
:10A8C000FF3004B070BD0020FBE7000038440108F1
:10A8D00070B505460E46002231462868FEF734F969
:10A8E00008B9002401E04FF0FF34204670BD014656
:10A8F000086808B9002070470120FCE710B504463D
:10A900004FF0FF312068FEF785F910BD1CB50446F5
:10A910000020009001906846FEF746F9206020680C
:10A9200010B94FF0FF301CBD0020FCE710B5044605
:10A930002068FEF747F910BD10B5F7F70BF810BD0A
:10A940002DE9F04188B004460D4616461F46DDF855
:10A9500038801C2101A8F5F700FD019402950FFA3B
:10A9600088F0ADF80C000597314601A8FEF7E2F932
:10A9700008B0BDE8F08100002DE9F04104460E4624
:10A98000174600BFB4F1804F08D300BF09A340F2BF
:10A99000291215A122A0F9F717F900BF00BFFFF790
:10A9A000CBFF05193A463146284600F04DF8BDE880
:10A9B000F08100002E2E2F4D6964646C6577617202
:10A9C00065732F54686972645F50617274792F4C9B
:10A9D0007749502F7372632F636F72652F74696D9F
:10A9E000656F7574732E630054696D656F7574209F
:10A9F00074696D6520746F6F206C6F6E672C206DAD
:10AA00006178206973204C5749505F55494E543343
:10AA1000325F4D41582F34206D7365637300000021
:10AA2000417373657274696F6E20222573222066EC
:10AA300061696C6564206174206C696E65202564B1
:10AA400020696E2025730A002DE9F04106460F4665
:10AA500090460A20FDF744FB0446002C0CD100BFB1
:10AA600007D100BF20A3BE222CA13CA0F9F7ACF86F
:10AA700000BF00BFBDE8F08100202060A760C4F8DF
:10AA80000C8066603F48006810B93E480460F1E7FA
:10AA90003C49606809684968401AB0F1004F01D329
:10AAA000012000E0002028B13648006820603548C9
:10AAB000046017E03348056811E0286850B1606809
:10AAC00029684968401AB0F1004F01D3012000E025
:10AAD000002018B1286820602C6002E02D68002D4D
:10AAE000EBD100BF00BFC5E72E2E2F4D6964646C0B
:10AAF0006577617265732F54686972645F50617223
:10AB000074792F4C7749502F7372632F636F72657E
:10AB10002F74696D656F7574732E63007379735F3D
:10AB200074696D656F75743A2074696D656F7574BD
:10AB300020213D204E554C4C2C20706F6F6C204DC9
:10AB4000454D505F5359535F54494D454F5554201F
:10AB5000697320656D70747900000000417373653E
:10AB60007274696F6E2022257322206661696C659C
:10AB700064206174206C696E6520256420696E20F4
:10AB800025730A00A400002010B5012408E006493E
:10AB900001EBC40251F834000449FFF7EDFE641CD8
:10ABA000032CF4D310BD00000C440108717500089B
:10ABB00070B51548006810B94FF0FF3070BDFFF751
:10ABC000BBFE0446104800684068001BB0F1004F0F
:10ABD00001D3012000E0002008B10020EEE70A4880
:10ABE00000684068051B00BFB5F1004F08D300BFE7
:10ABF00006A34FF4DC7212A116A0F8F7E5FF00BF20
:10AC000000BF2846DAE70000A40000202E2E2F4DBA
:10AC10006964646C6577617265732F5468697264E6
:10AC20005F50617274792F4C7749502F7372632F84
:10AC3000636F72652F74696D656F7574732E630031
:10AC4000696E76616C696420736C65657074696D9A
:10AC500065000000417373657274696F6E20222570
:10AC60007322206661696C6564206174206C696E72
:10AC70006520256420696E2025730A002DE9FF5F99
:10AC800004460E4600BF002C0AD100BF42A340F28A
:10AC90003D224DA153A0F8F797FF00BFBDE8FF9FED
:10ACA00000BF00BF207D012808D100BF3AA34FF4A8
:10ACB000107256A14BA0F8F787FF00BF00BF207DA0
:10ACC0000A2807D121465E4803F0D2F9204600F059
:10ACD00083FF5FE04FF0000AD346276DD4F824804D
:10ACE000D4F89050D4F81090207DE8B9E08A38B3B9
:10ACF00000BF54480068A04205D152480068C068AF
:10AD0000504908600DE04F49086806E0C168A1425B
:10AD100002D1E168C16002E0C0680028F6D100BF3E
:10AD200000BF0020E0600BE0B246B4F816B000BFF0
:10AD30002146454803F09CF901204449087000BFB2
:10AD4000206F10B1206F05F0E8F9E06E10B1E06EF1
:10AD500005F0E3F9606F10B1606F05F0DEF9BAF14C
:10AD6000000F0AD0208B211D23464246CDE9001B4F
:10AD700002903946204605F0D5F8207D0390204604
:10AD800000F02AFF00BF1DB16FF00C014846A84734
:10AD900000BF00BF00BF81E72E2E2F4D6964646C99
:10ADA0006577617265732F54686972645F50617270
:10ADB00074792F4C7749502F7372632F636F7265CC
:10ADC0002F7463702E6300007463705F6162616E44
:10ADD000646F6E3A20696E76616C6964207063629C
:10ADE00000000000417373657274696F6E20222544
:10ADF0007322206661696C6564206174206C696EE1
:10AE00006520256420696E2025730A00646F6E2713
:10AE1000742063616C6C207463705F61626F727424
:10AE20002F7463705F6162616E646F6E20666F7213
:10AE3000206C697374656E2D70636273000000008E
:10AE400070000020640000206C00002074000020CE
:10AE500010B5044601212046FFF710FF10BD28B1B0
:10AE6000027D012A02D10246916100BF70470000B5
:10AE700070B505460C46164600BF002C08D100BF31
:10AE800007A340F20F3212A119A0F8F79DFE00BFF0
:10AE900000BF2046FFF7DCFF6FF00C0070BD000024
:10AEA0002E2E2F4D6964646C6577617265732F5423
:10AEB000686972645F50617274792F4C7749502FC2
:10AEC0007372632F636F72652F7463702E6300005B
:10AED0007463705F6163636570745F6E756C6C3A08
:10AEE00020696E76616C6964207063620000000006
:10AEF000417373657274696F6E2022257322206618
:10AF000061696C6564206174206C696E65202564DC
:10AF100020696E2025730A0070B505460120FDF7F3
:10AF2000DFF804461CBB00F0CBFF01F079FD0120E7
:10AF3000FDF7D6F80446CCB9092001F009FD01203F
:10AF4000FDF7CEF8044684B9082001F001FD012088
:10AF5000FDF7C6F804463CB9284601F0C5FC0120BF
:10AF6000FDF7BEF8044600BF00BF00BF00BF44B3FA
:10AF70009C212046F5F7F1F90C3465724FF4866098
:10AF8000A4F858004000E083A083FF2004F8010CDF
:10AF90004FF40670E0840620A0866086C01FA0845F
:10AFA0000120A08708480068606108480078A07404
:10AFB0004FF48660E0870648A0670648C4F888001A
:10AFC0000C3C204670BD0000600000207600002090
:10AFD000E9F7000800DD6D002DE9F04705460C4655
:10AFE00017464FF0040904B92E4C00BF002D0CD1B8
:10AFF00000BF2DA340F2A92237A13DA0F8F7E4FD40
:10B0000000BF6FF00F00BDE8F08700BF00BF287DD4
:10B0100000280BD000BF24A340F2AB223EA134A0F5
:10B02000F8F7D2FD00BF6FF00500ECE700BF37B9BD
:10B0300001F0F8FF07460FBB6FF00100E3E74FF0A8
:10B04000000819E03E4850F82800066810E0F08A31
:10B05000B8420CD146B1306830B12CB1206818B17B
:10B0600030682168884202D16FF00700CBE7F668AC
:10B07000002EECD108F10108C845E3DB34B12068AB
:10B0800020B10CB9002000E020682860EF8200BFEA
:10B090002C480068E8602B48056005F05DFE00BFA5
:10B0A0000020B0E7284401082E2E2F4D6964646CFF
:10B0B0006577617265732F54686972645F5061725D
:10B0C00074792F4C7749502F7372632F636F7265B9
:10B0D0002F7463702E6300007463705F62696E6426
:10B0E0003A20696E76616C696420706362000000CA
:10B0F000417373657274696F6E2022257322206616
:10B1000061696C6564206174206C696E65202564DA
:10B1100020696E2025730A007463705F62696E6433
:10B120003A2063616E206F6E6C792062696E6420D4
:10B13000696E20737461746520434C4F534544001D
:10B14000FC4301086400002010B5044600BF002C39
:10B150000BD100BF0CA34FF4F47217A11CA0F8F799
:10B1600033FD00BF6FF00F0010BD00BF207D012830
:10B1700005D000BF608B40F01000608300BF01214C
:10B18000204600F039F8EFE72E2E2F4D6964646CED
:10B190006577617265732F54686972645F5061727C
:10B1A00074792F4C7749502F7372632F636F7265D8
:10B1B0002F7463702E6300007463705F636C6F7331
:10B1C000653A20696E76616C696420706362000084
:10B1D000417373657274696F6E2022257322206635
:10B1E00061696C6564206174206C696E65202564FA
:10B1F00020696E2025730A003EB504460D4600BF47
:10B20000002C08D100BF55A34FF4AF725FA167A017
:10B21000F8F7DAFC00BF00BF002D56D0207D0428CF
:10B2200002D0207D072850D1A06F18B9208DB0F52D
:10B23000066F4AD000BFA07E00F0100040B900BFEA
:10B2400046A34FF4B27263A158A0F8F7BDFC00BF4B
:10B2500000BF208BE18A221DCDE900210290234608
:10B260002046626A216D04F05DFE204602F092FEE7
:10B2700000BF00BF5E480068A04205D15C4800687E
:10B28000C0685B4908600DE05949086806E0C1687C
:10B29000A14202D1E168C16002E0C0680028F6D195
:10B2A00000BF00BF0020E06000BF012051490870CE
:10B2B00000BF51480068A04202D105F01DFE02E027
:10B2C000204600F089FC00203EBD207D20B10128F1
:10B2D00024D002283AD12CE0E08AD8B100BF4748F8
:10B2E0000068A04205D145480068C068434908602D
:10B2F0000DE04249086806E0C168A14202D1E16858
:10B30000C16002E0C0680028F6D100BF00BF002085
:10B31000E06000BF204600F05FFC1BE0204601F02B
:10B320009DFB2146364802F0A3FE204600F04CFD6E
:10B3300010E000BF21462E4802F09AFE01202D4960
:10B34000087000BF204600F047FC03E0204600F0F4
:10B3500059F8B9E700BF0020B6E700002E2E2F4DA8
:10B360006964646C6577617265732F54686972648F
:10B370005F50617274792F4C7749502F7372632F2D
:10B38000636F72652F7463702E6300007463705F67
:10B39000636C6F73655F73687574646F776E3A2062
:10B3A000696E76616C6964207063620041737365D5
:10B3B0007274696F6E2022257322206661696C6544
:10B3C00064206174206C696E6520256420696E209C
:10B3D00025730A007063622D3E666C6167732026D8
:10B3E0002054465F5258434C4F53454400000000E0
:10B3F0006C00002074000020A000002064000020E9
:10B400006800002070B5054600BF45B900BF1EA307
:10B410004FF4CE7228A12BA0F8F7D6FB00BF00BFD7
:10B42000287D032804D004280AD0072818D10FE06B
:10B43000284604F01FFF04460CB90520287511E0CA
:10B44000284604F017FF04460CB90520287509E0CA
:10B45000284604F00FFF04460CB90920287501E0C6
:10B46000002070BD00BF1CB9284601F0FDFE09E0B8
:10B47000601C38B900BF688B40F00800688300BFCB
:10B480000020EEE72046ECE72E2E2F4D6964646C19
:10B490006577617265732F54686972645F50617279
:10B4A00074792F4C7749502F7372632F636F7265D5
:10B4B0002F7463702E63000070636220213D204E64
:10B4C000554C4C00417373657274696F6E20222570
:10B4D0007322206661696C6564206174206C696EFA
:10B4E0006520256420696E2025730A002DE9F05F30
:10B4F00080460D4691469A460A9F00BFB8F1000F5C
:10B5000007D100BF40A3A3224CA154A0F8F75CFBD5
:10B5100000BF00BF00BF002D07D100BF3AA3A42287
:10B5200058A14EA0F8F750FB00BF00BF07F0010084
:10B5300008B1042000E0002007F0020109B1002159
:10B5400000E00021084407F0080109B1002100E0F3
:10B550000021084407F0100109B1002100E000219A
:10B5600046180320FCF7BCFD041E05D12846FEF753
:10B5700023F90020BDE8F09FA772002020606560DD
:10B5800000BF2889B04207DA00BF1FA3B02246A13E
:10B5900032A0F8F719FB00BF00BF2889801B20816B
:10B5A00014212846FDF7F5FB20B1204604F0A8FD44
:10B5B0000020DFE760684068E060B8F81600FCF73C
:10B5C0000CF8E1680880B8F81800FCF706F8E168A4
:10B5D00048805046FBF7F4FFE1684860B346F11736
:10B5E00006EB91718910491D4FF6FF7202EA013195
:10B5F00041EA0900FBF7F1FFE16888810020E1687A
:10B6000048822046B6E700002E2E2F4D6964646CF8
:10B610006577617265732F54686972645F506172F7
:10B6200074792F4C7749502F7372632F636F726553
:10B630002F7463705F6F75742E6300007463705FA6
:10B640006372656174655F7365676D656E743A20DA
:10B65000696E76616C696420706362004173736522
:10B660007274696F6E2022257322206661696C6591
:10B6700064206174206C696E6520256420696E20E9
:10B6800025730A007463705F6372656174655F732C
:10B6900065676D656E743A20696E76616C696420C9
:10B6A0007062756600000000702D3E746F745F6CF0
:10B6B000656E203E3D206F70746C656E000000006A
:10B6C00010B590B040216846F4F747FE234824495E
:10B6D000086024484860244888602448C86024489A
:10B6E000086124484861244888612448C861244886
:10B6F000086224484862244888622448C862244872
:10B70000086324484863244888632448C8630024A5
:10B710001FE000204DF824002149085501F07CFC71
:10B720004DF8240004F2E9325DF824001D49FFF7CA
:10B7300053FC5DF82400FF2101F0F4FA4DF82400D9
:10B74000074A52F824105DF82400FFF788FB601CBC
:10B75000C4B2102CDDDB10B010BD00006D1B010861
:10B76000ECC601202D1C0108451C01085D1C0108C8
:10B77000751C01088D1C0108A51C0108BD1C0108D1
:10B78000D51C0108851B01089D1B0108B51B01087C
:10B79000CD1B0108E51B0108FD1B0108151C010854
:10B7A0006CC70120284401082DE9F04106460D46EA
:10B7B000174600BF002F08D100BF10A340F6C502F6
:10B7C0001AA124A0F8F700FA00BF00BF15B930464F
:10B7D000BDE8F081AC8C74B12820844202DD211ACE
:10B7E00089B200E000218846464501DA314600E092
:10B7F00041460E4600BF3046EAE700002E2E2F4D90
:10B800006964646C6577617265732F5468697264EA
:10B810005F50617274792F4C7749502F7372632F88
:10B82000636F72652F7463702E6300007463705FC2
:10B830006566665F73656E645F6D73735F6E657476
:10B8400069663A20696E76616C6964206473745F1E
:10B8500069700000417373657274696F6E202225F0
:10B860007322206661696C6564206174206C696E66
:10B870006520256420696E2025730A002DE9F843B0
:10B8800004460D460027B94600BF05F0030040B945
:10B8900000BF60A340F211426B496CA0F8F794F925
:10B8A00000BF00BF00BF002C08D100BF59A340F269
:10B8B000134270A165A0F8F787F900BF00BF05F03B
:10B8C000020000B1012707F0010008B1042000E0E8
:10B8D000002007F0020109B1002100E00021084426
:10B8E00007F0080109B1002100E00021084407F039
:10B8F000100109B1002100E0002100EB01094FF423
:10B90000207249463620FDF7C1FAB0F1000809D18E
:10B9100000BF608B40F08000608300BF4FF0FF30BD
:10B92000BDE8F88300BFB8F80A00484508DA00BF50
:10B9300038A340F2394257A144A0F8F745F900BFB7
:10B9400000BF00972A4641462046E36DFFF7CEFD33
:10B95000061E07D100BF608B40F08000608300BFEF
:10B96000701EDDE700BF307B00F0030040B100BF78
:10B9700028A340F2424256A134A0F8F725F900BFAF
:10B9800000BF00BF308940B100BF22A340F2434254
:10B9900055A12EA0F8F718F900BF00BFE06E08B956
:10B9A000E66607E0E06E00E0006801680029FBD170
:10B9B000066000BF0020A4F8680005F0020010B97E
:10B9C00005F0010010B1E06D401CE06505F00100DC
:10B9D00028B100BF608B40F02000608300BF70681A
:10B9E000FDF7D4FC34F8661F0844208034F866095B
:10B9F00070B100BF206F50B9E06E40B900BF05A321
:10BA000040F2654243A111A0F8F7DEF800BF00BF85
:10BA1000002085E72E2E2F4D6964646C6577617276
:10BA200065732F54686972645F50617274792F4C2A
:10BA30007749502F7372632F636F72652F74637031
:10BA40005F6F75742E63000048450108417373658C
:10BA50007274696F6E2022257322206661696C659D
:10BA600064206174206C696E6520256420696E20F5
:10BA700025730A007463705F656E71756575655F27
:10BA8000666C6167733A20696E76616C69642070D8
:10BA9000636200007463705F656E71756575655FE4
:10BAA000666C6167733A20636865636B20746861D4
:10BAB0007420666972737420706275662063616EAB
:10BAC00020686F6C64206F70746C656E00000000FD
:10BAD0007365672D3E746370686472206E6F7420A6
:10BAE000616C69676E6564007463705F656E717523
:10BAF0006575655F666C6167733A20696E76616C27
:10BB00006964207365676D656E74206C656E67741B
:10BB1000680000007463705F656E71756575655FC0
:10BB2000666C6167733A20696E76616C6964207136
:10BB300075657565206C656E6774680070B523481F
:10BB40000078401C2149087000BF2148046839E092
:10BB5000A07F1E490978884233D01C480078A0771E
:10BB6000A07E00F0010078B100BF608B40F00200C1
:10BB7000608300BF204601F077FB00BF608B4FF66B
:10BB8000FC710840608300BFA07E00F0080048B14F
:10BB900000BF608B4FF6F7710840608300BF2046FE
:10BBA000FFF730FCE568A06F48B100200949087034
:10BBB000204602F0EBFE0748007800B1C5E72C46AE
:10BBC00000E0E468002CC3D170BD000076000020C6
:10BBD0006C0000207400002010B5044600BF207DDA
:10BBE000012807D100BF06A3D42211A115A0F7F7A1
:10BBF000EBFF00BF00BF21460120FCF7A3F910BDF9
:10BC00002E2E2F4D6964646C6577617265732F54B5
:10BC1000686972645F50617274792F4C7749502F54
:10BC20007372632F636F72652F7463702E630000ED
:10BC30007463705F667265653A204C495354454E93
:10BC400000000000417373657274696F6E202225D5
:10BC50007322206661696C6564206174206C696E72
:10BC60006520256420696E2025730A002DE9F047C0
:10BC700005460C469146984635E02646246870688D
:10BC8000FDF784FB074600BFB5F86600B84208DA46
:10BC900000BF22A340F257422DA137A0F7F794FF2F
:10BCA00000BF00BF35F8660FC01B288030893C49B3
:10BCB000098808443A490880304604F021FA35F8EA
:10BCC000660900280FD000BF002C0BD1B8F1000F7F
:10BCD00008D100BF11A340F2614232A126A0F7F7BC
:10BCE00073FF00BF00BFB4B1E1684868FBF768FCB0
:10BCF0008246E1688889FBF770FC00F0030008B118
:10BD0000012000E000202189084450442D490968A1
:10BD1000401A0028B1DD2046BDE8F0872E2E2F4DB9
:10BD20006964646C6577617265732F5468697264C5
:10BD30005F50617274792F4C7749502F7372632F63
:10BD4000636F72652F7463705F696E2E630000000D
:10BD50007063622D3E736E645F71756575656C65A9
:10BD60006E203E3D20706275665F636C656E286E66
:10BD70006578742D3E702900417373657274696F24
:10BD80006E2022257322206661696C6564206174CF
:10BD9000206C696E6520256420696E2025730A0079
:10BDA000940000207463705F726563656976653A1C
:10BDB0002076616C6964207175657565206C656EAF
:10BDC000677468009000002010B5044600BF207D15
:10BDD000012807D100BF06A3DF2211A117A0F7F7A2
:10BDE000F3FE00BF00BF21460220FCF7ABF810BDF8
:10BDF0002E2E2F4D6964646C6577617265732F54C4
:10BE0000686972645F50617274792F4C7749502F62
:10BE10007372632F636F72652F7463702E630000FB
:10BE20007463705F667265655F6C697374656E3AA2
:10BE300020214C495354454E000000004173736566
:10BE40007274696F6E2022257322206661696C65A9
:10BE500064206174206C696E6520256420696E2001
:10BE600025730A0010B50446606F20B1606F04F0BE
:10BE700054F90020606710BD0D4801880088401CFF
:10BE80000B4A10800B48006818B10B4800888142AB
:10BE900005DA0A48006800F11402505C7047064851
:10BEA0000078081AC2B203480068805CF6E7000018
:10BEB0008800002084000020820000207C000020F8
:10BEC00070B50B48046810E0E568A07E00F008003B
:10BED00048B100BF608B4FF6F7710840608300BF28
:10BEE0002046FFF78FFA2C4600BF002CECD170BD26
:10BEF0006C00002010B5F4F7F7F9C0F30D0000F561
:10BF000040400149088010BD5C0000202DE9FE4F33
:10BF100005468B4600BF002D07D100BFE2A3832258
:10BF2000EEA1F4A0F7F750FE00BF00BFFB49686820
:10BF300008606889142800DAC8E3F94A1168506972
:10BF4000FAF773F828B9F648007D00F0F000E02811
:10BF500000D1BBE3F14909688889FBF73EFB001378
:10BF60008700142F02DB2889B84200DAAEE3A7F17C
:10BF70001400EC4908800020EB4908606889B84249
:10BF800008DBE8480088E949088039462846FDF77B
:10BF900077FE4AE000BF286838B900BFC2A3C222BA
:10BFA000E3A1D4A0F7F710FE00BF00BF142128467C
:10BFB000FDF766FE6889DD490880DA48008809884F
:10BFC000401A1FFA80FAD94801882846FDF758FE22
:10BFD00028684089504500DA78E328684068D249EB
:10BFE000086051462868FDF74BFE2889A0EB0A003F
:10BFF000288100BF688938B100BFABA3DF22D0A180
:10C00000BCA0F7F7E1FD00BF00BF00BF2889296889
:10C010000989884207D000BFA3A3E022CBA1B5A025
:10C02000F7F7D2FD00BF00BF00BFBC490968088810
:10C03000FBF7D3FAB94909680880B8490968488804
:10C04000FBF7CBFAB54909684880B44909684868E4
:10C05000FBF7B6FAB14909684860C4490860AF49BE
:10C0600009688868FBF7ACFAAC4909688860C04980
:10C070000860AA490968C889FBF7AFFAA7490968A7
:10C08000C881A64909688889FBF7A7FA00F03F0034
:10C09000B84908702889B8490880B648007800F087
:10C0A000030040B108460088401C088028890988A0
:10C0B000884200DD0AE34FF00009B048046873E0ED
:10C0C00000BF207D38B900BF77A3FB22ACA189A0B7
:10C0D000F7F77AFD00BF00BF00BF207D0A2807D117
:10C0E00000BF71A3FC22B0A182A0F7F76DFD00BFD5
:10C0F00000BF00BF207D012807D100BF6AA3FD2239
:10C10000B4A17CA0F7F760FD00BF00BF207A50B15A
:10C11000217A8348406890F83000401CC0B28142C8
:10C1200001D0A1463FE0208B7C49096809888842FC
:10C1300037D1E08A794909684988884231D17849FC
:10C140006068096988422CD175492068496988422C
:10C1500027D100BFE068A04208D100BF52A340F23F
:10C160000D12A6A163A0F7F72FFD00BF00BFB9F124
:10C17000000F07D0E068C9F80C0080480068E06054
:10C180007E48046000BFE068A04208D100BF46A31B
:10C1900040F21512A4A157A0F7F716FD00BF00BF8B
:10C1A00004E0A14600BFE468002C89D100BF002C48
:10C1B00078D1A848046839E000BF207D0A2808D05B
:10C1C00000BF39A340F21F12A3A14AA0F7F7FCFC5D
:10C1D00000BF00BF207A48B1217A5148406890F8EA
:10C1E0003000401CC0B2814200D01EE0208B4B4981
:10C1F00009680988884217D1E08A4849096849884E
:10C20000884211D146496068096988420CD1444985
:10C2100020684969884207D1204604F0B9FD2846C4
:10C22000FDF7CAFABDE8FE8F00BFE468002CC3D159
:10C23000A146954806681FE0307A50B1317A3848F7
:10C24000406890F83000401CC0B2814201D0B14635
:10C2500011E0F08A314909684988884209D130499A
:10C2600030684969884200D108E00EB1306800B9F1
:10C2700004E0B14600BFF668002EDDD100BF8EB1EC
:10C28000B9F1000F07D0F068C9F80C007E480068CB
:10C29000F0607D480660304600F04AFC2846FDF715
:10C2A0008BFABFE7F2E000002E2E2F4D6964646C1C
:10C2B0006577617265732F54686972645F5061724B
:10C2C00074792F4C7749502F7372632F636F7265A7
:10C2D0002F7463705F696E2E630000007463705F7B
:10C2E000696E7075743A20696E76616C696420704D
:10C2F00062756600417373657274696F6E202225E2
:10C300007322206661696C6564206174206C696EBB
:10C310006520256420696E2025730A007C000020BA
:10C32000C4C601208000002084000020820000207C
:10C33000702D3E6E65787420213D204E554C4C008A
:10C34000702D3E6C656E203D3D203000702D3E749A
:10C350006F745F6C656E203D3D20702D3E6E65787C
:10C36000742D3E746F745F6C656E00008C0000204D
:10C370009000002098000020960000206C00002013
:10C380007463705F696E7075743A20616374697666
:10C3900065207063622D3E737461746520213D20B9
:10C3A000434C4F53454400007463705F696E707571
:10C3B000743A20616374697665207063622D3E7300
:10C3C0007461746520213D2054494D452D574149E4
:10C3D000540000007463705F696E7075743A206178
:10C3E0006374697665207063622D3E737461746551
:10C3F00020213D204C495354454E00007463705F2A
:10C40000696E7075743A207063622D3E6E65787443
:10C4100020213D2070636220286265666F7265206E
:10C4200063616368652900007463705F696E70758D
:10C43000743A207063622D3E6E65787420213D2031
:10C440007063622028616674657220636163686549
:10C4500029000000700000207463705F696E7075C1
:10C46000743A2054494D452D574149542070636218
:10C470002D3E7374617465203D3D2054494D452D1A
:10C48000574149540000000068000020002C73D080
:10C4900000209149086028890881084645608F4836
:10C4A0000068C86000208E4908608E4908708E4977
:10C4B00008808E48007800F0080018B1687B40F0D2
:10C4C00001006873A06F80B1204602F05FFA0D3062
:10C4D00028B1A06F48B186480088002805DD608D2E
:10C4E00010B9204603F026FEBCE0824804602046D6
:10C4F00001F0AAFE804608F10D00002816D0794808
:10C50000007800F0080090B100BFD4F8900028B186
:10C510006FF00D01D4F890202069904700BF2146AC
:10C52000754801F0A5FD2046FFF756FB99E04FF056
:10C5300000086D480088002819DD6B48B0F800A09D
:10C5400000BFD4F8800038B152462146D4F880307C
:10C5500020699847804601E04FF0000800BF08F1CD
:10C560000D0000B97EE000205F49088000BF204632
:10C5700000F0D8F808B175E084E059480068A8B325
:10C5800000BFA06F50B100BFAFF2E4234FF4F372CD
:10C590005AA1AFF2A020F7F717FB00BF00BFA07EA3
:10C5A00000F0100038B14E480068FDF705F920464C
:10C5B000FEF74EFC56E000BFD4F8840048B10023DB
:10C5C0004749D4F884C020690A682146E04780467C
:10C5D00007E00023424821460268184603F004F9A8
:10C5E000804600BF08F10D0008B93BE005E0B8F156
:10C5F000000F02D03A480068A0673A48007800F07F
:10C60000200018B3A06F30B1A06F407B40F0200035
:10C61000A16F48731AE0208DB0F5066F02D0208D0F
:10C62000401C208500BFD4F8840040B100231A4686
:10C630002146D4F884C02069E047804601E04FF0ED
:10C64000000800BF08F10D0000B90BE000202949E7
:10C650000860204600F066F800B103E0204600F0D4
:10C6600003FE00BF0020234908601D4908601A48E6
:10C67000406840B318494868FDF79EF80020164905
:10C68000486020E0154909688889FAF7A6FF00F09C
:10C690000400A8B911480068008810490968498851
:10C6A0001D4ACDE9002102901C4800681049098804
:10C6B0004218194B1B1D1A480168002003F032FC78
:10C6C0002846FDF779F800BF00BFABE52846FDF727
:10C6D00073F800BFA6E50000DCC601207C00002046
:10C6E0009C00002099000020940000209800002069
:10C6F00096000020A00000206C0000207063622DD6
:10C700003E726566757365645F64617461203D3D6A
:10C71000204E554C4C000000D4C601208C00002057
:10C720009000002010B5044600BF002C08D100BFC7
:10C7300013A340F25A221FA128A0F7F745FA00BF21
:10C7400000BF3048007800F01000B8B1A07E00F0C3
:10C75000100050B900BFD4F8900028B16FF00E015E
:10C76000D4F890202069904700BF2146264801F068
:10C770007FFC2046FFF730FA012010BD0020FCE7C7
:10C780002E2E2F4D6964646C6577617265732F542A
:10C79000686972645F50617274792F4C7749502FC9
:10C7A0007372632F636F72652F7463705F696E2E8F
:10C7B000630000007463705F696E7075745F646518
:10C7C0006C617965645F636C6F73653A20696E763E
:10C7D000616C6964207063620000000041737365DE
:10C7E0007274696F6E2022257322206661696C6500
:10C7F00064206174206C696E6520256420696E2058
:10C8000025730A00990000206C0000202DE9F041FA
:10C810000446002600BF002C08D100BF14A340F638
:10C82000240220A126A0F7F7CFF900BF00BF216D99
:10C83000481EFAF7C5FE8046434600223146204690
:10C8400000F0C4FE05461DB94FF0FF30BDE8F08191
:10C85000334600222946204601F036F8231D2246A1
:10C860002946204600F0B2FF07463846EEE70000B2
:10C870002E2E2F4D6964646C6577617265732F5439
:10C88000686972645F50617274792F4C7749502FD8
:10C890007372632F636F72652F7463705F6F75744B
:10C8A0002E6300007463705F6B656570616C697600
:10C8B000653A20696E76616C69642070636200007D
:10C8C000417373657274696F6E202225732220662E
:10C8D00061696C6564206174206C696E65202564F3
:10C8E00020696E2025730A002DE9F04107467F2F4D
:10C8F00001DD7F2000E0384606460EB9BDE8F08134
:10C90000701EC6B24FF0000800250F48046813E0FF
:10C91000607DB04208DB607DB0420CD10B49206ADB
:10C920000968081A404506D30849206A0968A1EB3E
:10C9300000082546667DE468002CE9D115B128463B
:10C94000FEF786FA00BFD9E76C00002060000020E7
:10C950002DE9F041054600BF082D0AD0092D08D069
:10C9600000BF13A340F2DD621DA121A0F7F72CF94F
:10C9700000BF00BF00270026274804680EE0207D86
:10C98000A8420AD12549206A0968081AB84204D386
:10C990002249206A09680F1A2646E468002CEED165
:10C9A0001EB100213046FEF769F9BDE8F0810000B4
:10C9B0002E2E2F4D6964646C6577617265732F54F8
:10C9C000686972645F50617274792F4C7749502F97
:10C9D0007372632F636F72652F7463702E63000030
:10C9E000696E76616C69642073746174650000001F
:10C9F000417373657274696F6E20222573222066FD
:10CA000061696C6564206174206C696E65202564C1
:10CA100020696E2025730A006C0000206000002051
:10CA200070B5002600250B4804680BE00A49206A0F
:10CA30000968081AB04204D30749206A09680E1A27
:10CA40002546E468002CF1D115B12846FEF700FA1E
:10CA500070BD0000700000206000002070B504462A
:10CA600000BF44B900BF12A340F211121CA11FA0C5
:10CA7000F7F7AAF800BF00BF00BF207D012808D04B
:10CA800000BF0BA34FF4897222A118A0F7F79CF8FE
:10CA900000BF00BF012507E0244951F825100868B0
:10CAA000214602F091FF6D1C042DF5D370BD0000EE
:10CAB0002E2E2F4D6964646C6577617265732F54F7
:10CAC000686972645F50617274792F4C7749502F96
:10CAD0007372632F636F72652F7463702E6300002F
:10CAE00070636220213D204E554C4C0041737365AC
:10CAF0007274696F6E2022257322206661696C65ED
:10CB000064206174206C696E6520256420696E2044
:10CB100025730A007063622D3E7374617465203D55
:10CB20003D204C495354454E00000000FC43010891
:10CB30002DE9FE4305465448007800F0040008B192
:10CB4000BDE8FE8300BF002D08D100BF4FA340F217
:10CB500081225BA162A0F7F737F800BF00BF4A4807
:10CB6000007800F01000B0B167480068008866499E
:10CB700009684988654ACDE9002102906448006847
:10CB8000644909884218614B1B1D634801682846A7
:10CB900003F0C8F975E03C48007800F00200002876
:10CBA0006FD0687DFEF7B8F9044674B900BFA86974
:10CBB00038B14FF0FF320021AB69286998478046B1
:10CBC00001E06FF00F0800BFBAE750481038406925
:10CBD00020604E48103800696060E88AE0824A4868
:10CBE0000068008820830320207549480068401CA5
:10CBF0006062606AE062204600F048FA0646A66578
:10CC000026656664E66542480068401E60652869DE
:10CC10002061E567687A00F00C006072287A207263
:10CC200000BF00BF3D480068E0603C48046004F07D
:10CC300093F800BF01203A49087000BF204601F078
:10CC400055F831480068C08924F8600F208860805A
:10CC5000603C201DF9F7C6FE8046608E221D4146CD
:10CC6000FEF7A2FD608612212046FEF707FE07466A
:10CC700027B100212046FEF701F861E7204600F0C9
:10CC8000F3FA00BF5CE70000980000202E2E2F4D25
:10CC90006964646C6577617265732F546869726446
:10CCA0005F50617274792F4C7749502F7372632FE4
:10CCB000636F72652F7463705F696E2E630000008E
:10CCC0007463705F6C697374656E5F696E707574A0
:10CCD0003A20696E76616C696420706362000000BE
:10CCE000417373657274696F6E202225732220660A
:10CCF00061696C6564206174206C696E65202564CF
:10CD000020696E2025730A007C000020D4C6012013
:10CD10008C00002096000020900000206C00002075
:10CD20007400002070B504460D46002229462046B6
:10CD300000F002F870BD00002DE9F041044688467D
:10CD40001746002500BF002C0BD100BF38A340F2CE
:10CD5000593243A14EA0F6F737FF00BF6FF00F0620
:10CD600060E000BF00BF207D00280BD000BF30A3D3
:10CD700040F25A3250A146A0F6F726FF00BF6FF0EE
:10CD80000E064FE000BF207D012803D125466FF03D
:10CD9000080647E00220FBF7A3F9054615B94FF056
:10CDA000FF363FE020692861E08AE882012028758B
:10CDB000607D6875607A687200202872E07AE87297
:10CDC000A07AA87220682860E08AD8B100BF4848DD
:10CDD0000068A04205D146480068C0684449086020
:10CDE0000DE04349086806E0C168A14202D1E1684C
:10CDF000C16002E0C0680028F6D100BF00BF00207B
:10CE0000E06000BF2046FEF7E7FE3A48A86100BF99
:10CE100039480068E8603848056003F09DFF00BFAE
:10CE2000002600BF07B13E702846BDE8F081000033
:10CE30002E2E2F4D6964646C6577617265732F5473
:10CE4000686972645F50617274792F4C7749502F12
:10CE50007372632F636F72652F7463702E630000AB
:10CE60007463705F6C697374656E5F776974685F13
:10CE70006261636B6C6F675F616E645F6572723A6B
:10CE800020696E76616C6964207063620000000046
:10CE9000417373657274696F6E2022257322206658
:10CEA00061696C6564206174206C696E652025641D
:10CEB00020696E2025730A007463705F6C69737457
:10CEC000656E5F776974685F6261636B6C6F675FE3
:10CED000616E645F6572723A2070636220616C7289
:10CEE0006561647920636F6E6E65637465640000CC
:10CEF0006400002071AE00086800002070B506468E
:10CF00000D46D6B13068C0B10C480168304600F01B
:10CF10001BF80B480168304600F016F86DB1286820
:10CF200058B10848046806E020683168884201D199
:10CF300028682060E468002CF6D170BD6C000020E9
:10CF400064000020680000202DE9F04105460E46EF
:10CF5000344600BF002D08D100BF0CA34FF410626F
:10CF600016A123A0F6F730FE00BF00BF0AE020683C
:10CF70002968884205D1E7682046FDF769FF3C46ED
:10CF800000E0E468002CF2D1BDE8F0812E2E2F4D98
:10CF90006964646C6577617265732F546869726443
:10CFA0005F50617274792F4C7749502F7372632FE1
:10CFB000636F72652F7463702E6300007463705F1B
:10CFC0006E657469665F69705F616464725F6368EF
:10CFD000616E6765645F7063626C6973743A20693F
:10CFE0006E76616C6964206F6C645F61646472006A
:10CFF000417373657274696F6E20222573222066F7
:10D0000061696C6564206174206C696E65202564BB
:10D0100020696E2025730A0010B54020FDF77CFFC3
:10D0200010BD000010B5002300BF16480088401C4A
:10D03000144C2080204600884FF6FF74A04203D194
:10D040004FF440400F4C2080002116E00E4850F86D
:10D05000210002680DE0D08A0A4C2488A04207D142
:10D06000581C83B2B3F5804F01DB002010BDDCE714
:10D07000D268002AEFD1481CC1B20429E6DB01487E
:10D080000088F3E75C000020FC43010810B504466B
:10D0900000BF002C08D100BF09A340F6AF0214A1C5
:10D0A0001AA0F6F791FD00BF00BF22480068224990
:10D0B000096808441F4908600846006810BD000060
:10D0C0002E2E2F4D6964646C6577617265732F54E1
:10D0D000686972645F50617274792F4C7749502F80
:10D0E0007372632F636F72652F7463702E63000019
:10D0F0007463705F6E6578745F6973733A20696EEC
:10D1000076616C696420706362000000417373652E
:10D110007274696F6E2022257322206661696C65C6
:10D1200064206174206C696E6520256420696E201E
:10D1300025730A00780000206000002070B50546C5
:10D140000C4600BF002D08D100BF25A340F21F42AE
:10D1500030A13AA0F6F738FD00BF00BFE968888922
:10D16000FAF73BFA00F0010020B1204602F0D5FFAB
:10D17000002433E013E0E1688889FAF72EFA00F022
:10D18000010038B10120FAF728FAE96889890843D3
:10D19000E968888126462468304602F0B1FF4CB128
:10D1A000E06840682189084429892E4A12681144A0
:10D1B000081AE0D594B128892A4909680844E16829
:10D1C0004968401A002809DDE068808825490988F7
:10D1D000401A288129896868FCF74AFC2C6070BDD8
:10D1E0002E2E2F4D6964646C6577617265732F54C0
:10D1F000686972645F50617274792F4C7749502F5F
:10D200007372632F636F72652F7463705F696E2E24
:10D21000630000007463705F6F6F735F696E7365A6
:10D2200072745F7365676D656E743A20696E7661BE
:10D230006C69642063736567000000004173736567
:10D240007274696F6E2022257322206661696C6595
:10D2500064206174206C696E6520256420696E20ED
:10D2600025730A008C0000202DE9F84F044600BF0A
:10D27000002C08D100BFA7A340F2E142B2A1B8A0A0
:10D28000F6F7A2FC00BF00BF00BF207D012808D137
:10D2900000BFA0A340F2E342BBA1B1A0F6F794FC0B
:10D2A00000BF00BFC2480068A04202D10020BDE814
:10D2B000F88FB4F86000B4F84810884202DAB4F885
:10D2C000600001E0B4F848008146E56E45B9A07EF3
:10D2D00000F0020018B1204602F02CFFE7E710E151
:10D2E000221D2146204602F00DFE074617B96FF0B9
:10D2F0000300DCE70CB1206858B90FB1381D00E01D
:10D300000020014611B96FF00300D0E708682060E3
:10D3100000BFE9684868FAF753F9616C401A298937
:10D320000844484519D9B4F8600048450CD1206F2D
:10D3300050B994F8990038B9002004F8980F0120EA
:10D3400060700020A070983CA07E00F0020018B130
:10D35000204602F0EFFEAAE7D3E0002084F899000F
:10D36000266F26B100E0366830680028FBD1B5E0B2
:10D3700000BFE9688889FAF730F900F0040040B18D
:10D3800000BF64A340F236528AA175A0F6F71CFCD8
:10D3900000BF00BF206FA0B1A07E00F0440080B9A4
:10D3A000E06E38B1E06E006858B9E06E0089618EB9
:10D3B000884206DAB4F8640018B1B4F866000928A7
:10D3C00001DB012000E0002020B9A07E00F0A000D9
:10D3D00000B98FE0207D022807D01020FAF7FDF871
:10D3E000E96889890843E96888813A4621462846E0
:10D3F00000F0FCFA0090009838B100BF608B40F05C
:10D400008000608300BF009851E72868E066207DB7
:10D41000022806D000BF608B4FF6FC710840608385
:10D4200000BFE9684868FAF7CBF88046E968888960
:10D43000FAF7D3F800F0030008B1012000E0002063
:10D440002989084408EB000A206DB0EB0A0001D5D9
:10D45000C4F850A0E9688889FAF7BFF800F0030023
:10D4600008B1012000E000202989084488B3002089
:10D470002860206F10B925672E462EE0E9684868BD
:10D48000FAF79EF88046F1684868FAF799F8B8EB21
:10D4900000001BD504F1700801E0D8F80080D8F82E
:10D4A000000068B1D8F80010C9684868FAF788F831
:10D4B0008346E9684868FAF783F8BBEB0000ECD4D0
:10D4C000D8F800002860C8F8005006E035603668DB
:10D4D00003E0FFE7284602F013FEE56E55B1E96868
:10D4E0004868FAF76DF8616C401A29890844484584
:10D4F0007FF63EAF00BFE06E10B90020A4F86800D0
:10D5000000BF00BF608B4FF67F710840608300BF93
:10D510000020CCE62E2E2F4D6964646C6577617215
:10D5200065732F54686972645F50617274792F4C0F
:10D530007749502F7372632F636F72652F74637016
:10D540005F6F75742E6300007463705F6F75747025
:10D5500075743A20696E76616C696420706362004C
:10D56000417373657274696F6E2022257322206681
:10D5700061696C6564206174206C696E6520256446
:10D5800020696E2025730A00646F6E277420636122
:10D590006C6C207463705F6F757470757420666F47
:10D5A00072206C697374656E2D7063627300000085
:10D5B000A0000020525354206E6F7420657870656F
:10D5C0006374656420686572652100002DE9FF4180
:10D5D00004460E461746984600BF002C08D100BFEF
:10D5E00010A340F242721CA125A0F6F7EDFA00BF8D
:10D5F00000BF608D1023218BE28ACDE901130092D8
:10D60000039043463A463146606A00F04DF80546BD
:10D610001DB1618D606A0844E062284604B0BDE82F
:10D62000F08100002E2E2F4D6964646C6577617265
:10D6300065732F54686972645F50617274792F4CFE
:10D640007749502F7372632F636F72652F74637005
:10D650005F6F75742E6300007463705F6F75747014
:10D6600075745F616C6C6F635F6865616465723A65
:10D6700020696E76616C696420706362000000004E
:10D68000417373657274696F6E2022257322206660
:10D6900061696C6564206174206C696E6520256425
:10D6A00020696E2025730A002DE9F05F82460D4641
:10D6B00017469846DDF830B005F11400384481B2C1
:10D6C0004FF420722220FBF7E1FB0646002E34D0F7
:10D6D00000BF718905F11400814208DA00BF18A368
:10D6E00040F2237223A12FA0F6F76EFA00BF00BF0D
:10D6F00074680A98F9F771FF20800B98F9F76DFFAD
:10D700006080C4F804805046F9F75AFFA060A9462B
:10D71000E91705EB91718910491D4FF6FF7202EA76
:10D72000013141EA0B00F9F758FFA0810D98F9F794
:10D7300054FFE0810020208260823046BDE8F09FE7
:10D740002E2E2F4D6964646C6577617265732F545A
:10D75000686972645F50617274792F4C7749502FF9
:10D760007372632F636F72652F7463705F6F75746C
:10D770002E630000636865636B20746861742066C3
:10D780006972737420706275662063616E20686FC1
:10D790006C6420737472756374207463705F686462
:10D7A00072000000417373657274696F6E202225E8
:10D7B0007322206661696C6564206174206C696EF7
:10D7C0006520256420696E2025730A002DE9FE4F2F
:10D7D00004460E4692469B4600BF002E08D100BF6D
:10D7E00017A340F2877223A12DA0F6F7EDF900BF31
:10D7F00000BF5A465146204602F084FB054615B943
:10D800006FF0030715E024B194F80B8094F80A90A8
:10D8100003E04FF0FF084FF00009062043465A4648
:10D820005146CDE9009002953046F8F773FE074661
:10D8300000BF3046FBF7C0FF3846BDE8FE8F000052
:10D840002E2E2F4D6964646C6577617265732F5459
:10D85000686972645F50617274792F4C7749502FF8
:10D860007372632F636F72652F7463705F6F75746B
:10D870002E6300007463705F6F75747075745F63FE
:10D880006F6E74726F6C5F7365676D656E743A204E
:10D89000696E76616C6964207062756600000000D4
:10D8A000417373657274696F6E202225732220663E
:10D8B00061696C6564206174206C696E6520256403
:10D8C00020696E2025730A002DE9F04781460D4638
:10D8D00014469A464FF0000800BF002D08D100BF43
:10D8E0001CA340F2567228A131A0F6F76DF900BFD3
:10D8F00000BF6E6806F1140700BF384600EB8800D1
:10D9000004F0010109B1042100E00021084404F001
:10D91000020109B1002100E00021084404F00801DF
:10D9200009B1002100E00021084404F0100109B110
:10D93000002100E000210844B84208D000BF05A340
:10D9400040F2757224A11AA0F6F73EF900BF00BF9D
:10D95000BDE8F0872E2E2F4D6964646C6577617287
:10D9600065732F54686972645F50617274792F4CCB
:10D970007749502F7372632F636F72652F746370D2
:10D980005F6F75742E6300007463705F6F757470E1
:10D9900075745F66696C6C5F6F7074696F6E733AF3
:10D9A00020696E76616C69642070627566000000A3
:10D9B000417373657274696F6E202225732220662D
:10D9C00061696C6564206174206C696E65202564F2
:10D9D00020696E2025730A006F7074696F6E732062
:10D9E0006E6F742066696C6C656400002DE9FE4FF3
:10D9F00004460D46164600BF002C08D100BF58A3B0
:10DA00004FF4B76263A16BA0F6F7DEF800BF00BF6A
:10DA100000BF002D08D100BF51A340F2B9526FA141
:10DA200064A0F6F7D1F800BF00BF00BF002E08D1F8
:10DA300000BF4BA340F2BA5270A15EA0F6F7C4F843
:10DA400000BF00BF204600F0F7F810B10020BDE88D
:10DA5000FE8F686AF9F7B4FDE1688860688DF9F7B0
:10DA6000BCFDE168C881698D686A0844E862E068C5
:10DA700000F11407A07A00F0010068B12A1D3146B8
:10DA80004FF40670FDF790FE82464AF00170F9F7F8
:10DA900097FD38603F1D00BFB5F93000002801DA5E
:10DAA00000202886686B38B95D4800686863E168C3
:10DAB0004868F9F785FDA863A08961688988401ADC
:10DAC0001FFA80F860684089A0EB0800616848810F
:10DAD00060680089A0EB0800616808816168E068FF
:10DAE00048600020E168088200BFE0681430A17A35
:10DAF00001F0010109B1042100E000210844A17AEC
:10DB000001F0020109B1002100E000210844A17ADE
:10DB100001F0080109B1002100E000210844A17AC8
:10DB200001F0100109B1002100E000210844B842D1
:10DB300008D000BF0AA340F21C623AA11DA0F6F76C
:10DB400043F800BF00BF0621A87A8DE84300EB7AB6
:10DB50002A1D29466068F8F7DDFC8146484676E7CD
:10DB60002E2E2F4D6964646C6577617265732F5436
:10DB7000686972645F50617274792F4C7749502FD5
:10DB80007372632F636F72652F7463705F6F757448
:10DB90002E6300007463705F6F75747075745F73CB
:10DBA00065676D656E743A20696E76616C69642094
:10DBB00073656700417373657274696F6E20222507
:10DBC0007322206661696C6564206174206C696EE3
:10DBD0006520256420696E2025730A007463705FD8
:10DBE0006F75747075745F7365676D656E743A20D8
:10DBF000696E76616C696420706362007463705F43
:10DC00006F75747075745F7365676D656E743A20B7
:10DC1000696E76616C6964206E65746966000000E7
:10DC2000600000206F7074696F6E73206E6F7420D7
:10DC300066696C6C6564000010B5044600BF002C7A
:10DC400008D100BF08A340F29A5214A11DA0F5F715
:10DC5000BBFF00BF00BF6068807B012801D00120AE
:10DC600010BD0020FCE700002E2E2F4D6964646C6F
:10DC70006577617265732F54686972645F50617271
:10DC800074792F4C7749502F7372632F636F7265CD
:10DC90002F7463705F6F75742E6300007463705F20
:10DCA0006F75747075745F7365676D656E745F62B0
:10DCB0007573793A20696E76616C69642073656763
:10DCC00000000000417373657274696F6E20222535
:10DCD0007322206661696C6564206174206C696ED2
:10DCE0006520256420696E2025730A002DE9F04126
:10DCF000054600BF002D08D100BF28A340F27D7269
:10DD000033A13AA0F5F760FF00BF00BF414800888B
:10DD1000002840D000204049088036E0FEF7ACF8EB
:10DD2000074627B1012F04D0022F1FD102E0BDE822
:10DD3000F08128E0FEF7A0F8042806D136480088D4
:10DD4000801C34490988884200DDF0E7FEF794F82A
:10DD50000602FEF791F80643B6F5067F00DC16B919
:10DD60004FF4067000E0304668860CE0FEF784F859
:10DD70000446022C00DADAE7A01E27490988084485
:10DD80002549088000BF00BF00BF23480088214903
:10DD900009888842C2DB00BFC9E700002E2E2F4D44
:10DDA0006964646C6577617265732F546869726425
:10DDB0005F50617274792F4C7749502F7372632FC3
:10DDC000636F72652F7463705F696E2E630000006D
:10DDD0007463705F70617273656F70743A20696EFE
:10DDE00076616C6964207063620000004173736542
:10DDF0007274696F6E2022257322206661696C65DA
:10DE000064206174206C696E6520256420696E2031
:10DE100025730A0080000020880000202DE9F84FBB
:10DE200081460C4617469846DDE90BAB0A9E0094E6
:10DE300000BFB8F1000F07D100BF29A3E82235A128
:10DE40003DA0F5F7C1FE00BF00BF00BF002E07D107
:10DE500000BF23A3E92242A137A0F5F7B5FE00BF1A
:10DE600000BFBC421BDA0AF0020050B9B07E00F0DD
:10DE70004000A0B9BBF1000F03D0F06E08B9306FBD
:10DE800068B104F21B2020F00300B84201D93846E3
:10DE900003E004F21B2020F0030080B200904FF456
:10DEA000207248460099FAF7F1FF054615B900209F
:10DEB000BDE8F88F00BF286840B100BF08A340F25A
:10DEC0000B122FA11CA0F5F77FFE00BF00BF6889D1
:10DED000001BA8F800002C816C812846E8E70000B0
:10DEE0002E2E2F4D6964646C6577617265732F54B3
:10DEF000686972645F50617274792F4C7749502F52
:10DF00007372632F636F72652F7463705F6F7574C4
:10DF10002E6300007463705F706275665F70726577
:10DF2000616C6C6F633A20696E76616C6964206F16
:10DF300076657273697A6500417373657274696F8F
:10DF40006E2022257322206661696C6564206174ED
:10DF5000206C696E6520256420696E2025730A0097
:10DF60007463705F706275665F707265616C6C6F10
:10DF7000633A20696E76616C6964207063620000A8
:10DF80006E65656420756E636861696E6564207096
:10DF90006275660010B5044600BF002C09D100BFB1
:10DFA00016A340F6510221A127A0F5F70DFE00BFF0
:10DFB00010BD00BF207DF8B1207D0A281CD0207D37
:10DFC000012819D0A06F20B1A06FFBF7F5FB00204E
:10DFD000A067606F10B12046FDF744FF4FF0FF309F
:10DFE0002086E06E02F099F8206F02F096F800208B
:10DFF000E0662067A4F8680000BFD9E72E2E2F4DF9
:10E000006964646C6577617265732F5468697264C2
:10E010005F50617274792F4C7749502F7372632F60
:10E02000636F72652F7463702E6300007463705F9A
:10E030007063625F70757267653A20696E76616CB5
:10E040006964207063620000417373657274696F64
:10E050006E2022257322206661696C6564206174DC
:10E06000206C696E6520256420696E2025730A0086
:10E0700070B505460C4600BF002C08D100BF3AA37E
:10E0800040F6830244A14BA0F5F79EFD00BF00BF00
:10E0900000BF002D08D100BF33A340F684024FA17A
:10E0A00044A0F5F791FD00BF00BF00BF2868A04263
:10E0B00003D12868C06828600CE0286806E0C168C1
:10E0C000A14202D1E168C16002E0C0680028F6D137
:10E0D00000BF00BF0020E06000BF2046FFF75AFFEE
:10E0E000207D0A280FD0207D01280CD0A07E00F0D2
:10E0F000010040B100BF608B40F00200608300BFB0
:10E100002046FFF7B1F8207D012826D000BFE06E41
:10E1100040B100BF14A340F6930238A125A0F5F743
:10E1200053FD00BF00BF00BF206F40B100BF0EA372
:10E1300040F6940237A11FA0F5F746FD00BF00BFCF
:10E1400000BF606F40B100BF07A340F6960238A140
:10E1500018A0F5F739FD00BF00BF00202075E08250
:10E1600000BF00BF70BD00002E2E2F4D6964646C8F
:10E170006577617265732F54686972645F5061726C
:10E1800074792F4C7749502F7372632F636F7265C8
:10E190002F7463702E6300007463705F7063625F3E
:10E1A00072656D6F76653A20696E76616C69642080
:10E1B00070636200417373657274696F6E2022250B
:10E1C0007322206661696C6564206174206C696EDD
:10E1D0006520256420696E2025730A007463705FD2
:10E1E0007063625F72656D6F76653A20696E766105
:10E1F0006C6964207063626C69737400756E73651A
:10E200006E74207365676D656E7473206C65616BE9
:10E21000696E6700756E61636B6564207365676D19
:10E22000656E7473206C65616B696E670000000039
:10E230006F6F736571207365676D656E7473206CA5
:10E2400065616B696E6700002DE9FE430446002797
:10E25000002600BF002C08D100BFE5A34FF4477291
:10E26000F0A1F7A0F5F7B0FC00BF00BFFE480078B2
:10E2700000F00400002845D0207D022806D1FB498B
:10E28000206D096888421BD1012719E0F849606AAE
:10E290000968884201D1012712E0F549606A0968DE
:10E2A000081A0DD4218D606A0844F1490968081ADA
:10E2B000002805DC00BF608B40F00200608300BFD7
:10E2C000002F1DD000BF207D40B900BFC8A34FF470
:10E2D0004E72E8A1DAA0F5F777FC00BF00BFED4869
:10E2E000007840F00800EB49087000BF608B4FF6E3
:10E2F000FE710840608300BF6FF00D00BDE8FE8333
:10E300000020FBE7D848007800F0020068B1207DCB
:10E3100002280AD0207D032807D000BF608B40F080
:10E320000200608300BF0020E8E7A07E00F010003C
:10E3300010B9D94800682062002084F89B0084F856
:10E340009A002046FFF7D2FC207D801E082875D257
:10E35000DFE800F004CDF4F3F2F1F0EFC24800780A
:10E3600000F0100000286AD0BF48007800F00200DA
:10E370000028F8D0606C401CBC49096888425ED116
:10E38000BB480068401C6062606AE062B748006891
:10E390006064C2480068C089A4F86000B4F86000F6
:10E3A000A4F86200B2480068401E60650420207531
:10E3B000201DF8F717FB8046608E221D4146FDF7B1
:10E3C000F3F96086608E8100400041F21C12904299
:10E3D00002D9608E400001E041F21C10814202D25D
:10E3E000608E80000AE0608E400041F21C1188427D
:10E3F00002D9608E400001E041F21C10A4F84800F0
:10E4000000BFB4F86600002808DC00BF78A34FF412
:10E410005B72A3A18AA0F5F7D7FB00BF00BFB4F8D9
:10E420006600401EA4F86600256F95B9E56E00BF32
:10E430005DB900BF6EA34FF45D7201E08DE231E083
:10E440009DA17FA0F5F7C0FB00BF00BF2868E06674
:10E4500001E028682067284601F052FE206F18B9B5
:10E460004FF0FF30208603E00020208684F8420031
:10E4700000BFD4F8880038B100222146D4F8883093
:10E4800020699847064600E0002600BF06F10D000F
:10E4900010B96FF00C0031E700BF608B40F0020054
:10E4A000608323E07048007800F01000F0B17B48F2
:10E4B00000680088794909684988844ACDE90021C3
:10E4C00002906B4800688249098842187F4B1B1DE7
:10E4D00066480168204601F025FD94F842000628B0
:10E4E00004DA00202086204601F0D0FB36E25E48A8
:10E4F000007800F01000002876D0606C401C5B496A
:10E500000968081A71D45949206D0968081A002849
:10E510006BDC04202075E06F10B96FF0050623E076
:10E5200000BFE06F806978B900BF31A34FF46A7211
:10E5300005E0FCE1BCE107E17CE117E105E165A153
:10E540003FA0F5F741FB00BF00BF00BFE06F80694F
:10E5500038B1E16F206900228B6921469847064651
:10E5600001E06FF00F0600BF46B106F10D0010B1DB
:10E570002046FCF76DFC6FF00C00BFE6204600F073
:10E580009FFA5C48008820B15A480088401E5949CB
:10E590000880608E8100400041F21C12904202D936
:10E5A000608E400001E041F21C10814202D2608E78
:10E5B00080000AE0608E400041F21C11884202D9BE
:10E5C000608E400001E041F21C10A4F84800314880
:10E5D000007800F0200048B100BF608B40F00200DE
:10E5E000608300BF072087E09FE087E0ABE000008A
:10E5F0002E2E2F4D6964646C6577617265732F549C
:10E60000686972645F50617274792F4C7749502F3A
:10E610007372632F636F72652F7463705F696E2E00
:10E62000630000007463705F70726F636573733AA8
:10E6300020696E76616C696420706362000000007E
:10E64000417373657274696F6E2022257322206690
:10E6500061696C6564206174206C696E6520256455
:10E6600020696E2025730A00980000209000002089
:10E670008C0000207463705F696E7075743A20704E
:10E6800063622D3E737461746520213D20434C4FBD
:10E690005345440099000020600000207C000020C9
:10E6A0007063622D3E736E645F71756575656C6530
:10E6B0006E203E20300000006E6F207365676D6530
:10E6C0006E7420746F20667265650000D4C60120E8
:10E6D000960000207063622D3E6C697374656E65F0
:10E6E000722D3E61636365707420213D204E554C50
:10E6F0004C00000094000020207524E09948006838
:10E700000188984800684088974ACDE90020029126
:10E7100096480068964909884218934B1B1D9548F6
:10E720000168204601F0FEFB0DE09348007800F000
:10E73000020040B1606A401E8C490968884202D1DB
:10E74000204601F09BF909E100BF204600F0B8F92E
:10E750008A48007800F0200038B100BF608B40F09C
:10E760000200608300BF07202075F7E0204600F01C
:10E77000A7F98248007800F02000E8B37E480078CE
:10E7800000F01000C8B37B49206D0968884239D178
:10E79000E06E90BB00BF608B40F00200608300BF62
:10E7A0002046FFF7F7FB00BF00BF75480068A04296
:10E7B00005D173480068C068714908600DE0704970
:10E7C000086806E0C168A14202D1E168C16002E0C8
:10E7D000C0680028F6D100BF00BF0020E06000BF85
:10E7E00001206849087000BF0A20207500BF6648F4
:10E7F0000068E060644801E00DE003E0046002F0BE
:10E80000ABFA16E000BF608B40F00200608300BFEF
:10E81000082020750DE05848007800F0100040B145
:10E820005449206D0968884203D1E06E08B906207A
:10E83000207593E0204600F043F95048007800F03E
:10E840002000A0B300BF608B40F00200608300BFD7
:10E850002046FFF79FFB00BF00BF49480068A04269
:10E8600005D147480068C068454908600DE0444943
:10E87000086806E0C168A14202D1E168C16002E017
:10E88000C0680028F6D100BF00BF0020E06000BFD4
:10E8900001203C49087000BF0A20207500BF3A489B
:10E8A0000068E0603848046002F056FA00BF55E0A6
:10E8B000204600F005F93048007800F01000A8B3B9
:10E8C0002C49206D0968884230D1E06E70BB20462B
:10E8D000FFF760FB00BF00BF29480068A04205D1D8
:10E8E00027480068C068264908600DE02449086888
:10E8F00006E0C168A14202D1E168C16002E0C068DF
:10E900000028F6D100BF00BF0020E06000BF01205A
:10E910001C49087000BF0A20207500BF1A48006813
:10E92000E0601948046002F017FA00BF16E02046C4
:10E9300000F0C6F81048007800F0100060B10D49F2
:10E94000206D0968884207D1E06E28B90B4800782D
:10E9500040F010000949087000E000BF00BF00202F
:10E96000CCE400007C000020D4C601208C000020F4
:10E9700096000020900000209800002099000020C0
:10E980006C00002074000020700000202DE9F04190
:10E99000044600BF002C0CD100BF29A340F209623D
:10E9A00033A13DA0F5F710F900BF6FF00F00BDE8EF
:10E9B000F08100BFA06F477BA66F0020A06700BF5B
:10E9C000D4F8840040B1002332462146D4F884C0F4
:10E9D0002069E047054606E00023324621461846F6
:10E9E00000F002FF054600BFF5B907F0200028B38C
:10E9F000208DB0F5066F02D0208D401C208500BF11
:10EA0000D4F8840040B100231A462146D4F884C0CB
:10EA10002069E047054600E0002500BF05F10D0034
:10EA200060B96FF00C00C2E705F10D0010B96FF08E
:10EA30000C00BCE7A6676FF00400B8E70020B6E75B
:10EA40002E2E2F4D6964646C6577617265732F5447
:10EA5000686972645F50617274792F4C7749502FE6
:10EA60007372632F636F72652F7463702E6300007F
:10EA70007463705F70726F636573735F72656675E0
:10EA80007365645F646174613A20696E76616C6974
:10EA90006420706362000000417373657274696F73
:10EAA0006E2022257322206661696C656420617482
:10EAB000206C696E6520256420696E2025730A002C
:10EAC0002DE9F05F04464FF0000900BF002C08D18B
:10EAD00000BFE5A340F27B42F0A1F7A0F5F774F880
:10EAE00000BF00BF00BF207D042808DA00BFDEA3FE
:10EAF00040F27C42FAA1F0A0F5F766F800BF00BF33
:10EB0000FE48007800F01000002870D0B4F86000D3
:10EB1000A16D00EB0108FA49606D0968401A15D42F
:10EB2000F749606D0968884204D1F649A06D09680B
:10EB3000401A0BD4F349A06D096888421AD1F248F3
:10EB40000068C089B4F86010884213D9EE480068A4
:10EB5000C08924F8600F608834F86019884203DAAD
:10EB6000B4F86000A4F86200E54800686065E54814
:10EB70000068A065E349606C0968081A00284ADC4F
:10EB8000E248008890BBB4F86010A06D084440458E
:10EB90003AD1B4F93000002836DBDA49606C0968F4
:10EBA000884231D14FF0010994F84300401CC0B2B3
:10EBB00094F84310884204DD94F84300401C84F824
:10EBC000430094F84300032817DD00BFB4F8480061
:10EBD000618E084480B2B4F84810884208DBB4F86B
:10EBE0004800618E0844A4F8480005E00CE02AE1E2
:10EBF0004FF6FF70A4F8480000BF94F843000328C4
:10EC000002DB204600F0BCFFB9F1000F02D100206A
:10EC100084F84300EBE0606C401CBA490968081AAC
:10EC20007ED4B849206D0968081A002878DCA07ED7
:10EC300000F0040060B100BF608B4FF6FB7108402C
:10EC4000608300BF48346088208000206084483C96
:10EC500000202434A077608BB4F9181000EBE10099
:10EC600000B2A083208CA7490988081A85B2002029
:10EC7000E077A4480068206214F8100C243C0428B3
:10EC800065DBB4F84800B4F84A10884227DA628B92
:10EC900002F400620AB1012200E002221146628EF3
:10ECA0004A4392B2AA4201DD2A4602E0628E4A43FA
:10ECB00092B2104600BFB4F84820024492B2B4F8B1
:10ECC00048309A4205DBB4F848200244A4F84820B2
:10ECD00003E04FF6FF72A4F8482000BF37E000BF02
:10ECE000B4F86A00284480B2B4F86A10884205DBA0
:10ECF000B4F86A002844A4F86A0003E04FF6FF70F5
:10ED0000A4F86A0000BFB4F86A00B4F8481088425A
:10ED10001DDB4834608C2188401A6084483C00E048
:10ED200062E000BFB4F84800618E084480B2B4F8D5
:10ED30004810884206DBB4F84800618E0844A4F805
:10ED4000480003E04FF6FF70A4F8480000BF70A22F
:10ED50002046D4E91B31FCF789FF20676EA22046CC
:10ED6000D4E91B13FCF782FFE066206F18B94FF05F
:10ED7000FF30208601E00020208600202077E06E12
:10ED800010B90020A4F86800B4F864006449098848
:10ED90000844A4F86400608B00F4006018B3206F8E
:10EDA00088B9E06E40B1E16EC9684868F8F708FCC0
:10EDB000E16C081A002816DC00BF608B4FF2FF716F
:10EDC000084060830FE0216FC9684868F8F7F8FBD6
:10EDD000E16C081A002806DC00BF608B4FF2FF715F
:10EDE0000840608300BF02E0204601F0A3F9606B99
:10EDF00048B34449A06B0968401A24D5A08E4949FC
:10EE00000988081A07B2B4F93C00A7EBE00007B282
:10EE1000A08F384400B2A087002F01DA784207B2F1
:10EE2000B4F93E00A7EBA00007B2E08F384400B26F
:10EE3000E087E08FB4F93C1000EBE10000B2A4F8E9
:10EE40004000002060633148008800286CDD207D90
:10EE5000072869DA2A48616A0068401C081A7CD4CD
:10EE60002748616A006860E02E2E2F4D6964646C4B
:10EE70006577617265732F54686972645F5061725F
:10EE800074792F4C7749502F7372632F636F7265BB
:10EE90002F7463705F696E2E630000007463705F8F
:10EEA000726563656976653A20696E76616C69643E
:10EEB0002070636200000000417373657274696FB3
:10EEC0006E2022257322206661696C65642061745E
:10EED000206C696E6520256420696E2025730A0008
:10EEE0007463705F726563656976653A2077726FE7
:10EEF0006E67207374617465000000009800002044
:10EF00008C000020900000207C0000209600002053
:10EF1000756E61636B656400756E73656E74000079
:10EF20009400002060000020D4E3F74A12881044C7
:10EF3000401E081A00285FDCF4484668F449606AFD
:10EF40000968A0EB010A00BFF048406860B900BF43
:10EF5000AFF2EC0340F2945200E04DE0EDA1AFF2CD
:10EF6000A800F4F731FE00BF00BF00BF4FF6FF70EE
:10EF700082450AD300BFAFF2101340F29552E9A1C7
:10EF8000AFF2CC00F4F720FE00BF00BF1FFA8AF5F5
:10EF900000BFDE4840680089A8420ADA00BFAFF22D
:10EFA000381340F29752E3A1AFF2F400F4F70CFEED
:10EFB00000BF00BFD5480089401BD44908810846DE
:10EFC00040680089401B1FFA80FB07E07089281AFF
:10EFD00085B2A6F808B00020708136687089A84212
:10EFE000F4DB29463046FAF74BFEC949606A0860EF
:10EFF000C649C96848600AE0C549606A0968081AD4
:10F0000005D500BF608B40F00200608300BFC0499F
:10F01000606A0968081A7DD4218D606A0844401E20
:10F02000BB490968081A002874DCB949606A096894
:10F03000884270D1B549C9688889F8F7CEFA00F0DE
:10F04000030008B1012000E00020B049098908440C
:10F05000AD490880208D0988884256DAAB49C968D5
:10F060008889F8F7BAFA00F0010098B1A749C96891
:10F070008889F8F7B2FA00F03E052846F8F7ADFAAD
:10F08000A249C96889894CF2FF02114008439F498F
:10F09000C9688881208D9D490881C9688889F8F7E9
:10F0A0009CFA00F0020020B198480089401E974960
:10F0B0000881964A11895068FAF7DAFC9349C968C1
:10F0C0008889F8F78AFA00F0030008B1012000E00F
:10F0D00000208E49098908448B49088000BF218D92
:10F0E000606A08448A490968874A1288114488423C
:10F0F0000AD000BFAFF2902340F2CB5291A1AFF201
:10F100004820F4F761FD00BF00BF606F002816D0F3
:10F110007E4901E0DAE2D3E1C9688889F8F75DFA4F
:10F1200000F0010060B107E0656F606F0068606724
:10F13000284600F0E5FF00BF606F0028F4D187E0AB
:10F14000656F2EE0E9688889F8F747FA00F001005A
:10F1500008B36E49C9688889F8F73FFA00F00200E1
:10F16000C8B90120F8F739FA6849C968898908439C
:10F170006649C96888816549C9688889F8F72DFAA0
:10F1800000F0030008B1012000E000205F49098978
:10F1900008445D4908802E462D68304600F0B0FFD7
:10F1A00000BF55B1E8684068298908445849096892
:10F1B000554A12881144081AC4D5002D46D0544827
:10F1C0000068514909880844E9684968401A0028DC
:10F1D0003CDDE86880884E490988401A4B4908811F
:10F1E000C9688889F8F7F9F900F0020020B14748AA
:10F1F0000089401E45490881444A11895068FAF740
:10F2000037FC4249C9688889F8F7E7F900F003003C
:10F2100008B1012000E000203C49098908443A492E
:10F22000088000BF3A48006809880844E9684968CE
:10F2300088420AD000BFAFF2D03340F2FC524FA157
:10F24000AFF28C30F4F7C0FC00BF00BF656700BFB1
:10F250002F4800682C4909880844606200BF208D4F
:10F260002949098888420ADA00BFAFF2044340F214
:10F27000076251A1AFF2C030F4F7A6FC00BF00BF97
:10F28000208D21490988401A2085204601F03EFE44
:10F290001E4840680089002806DD1C4840684E4929
:10F2A00008600020194948601849C9688889F8F73A
:10F2B00094F900F0010028B14848007840F020009F
:10F2C00046490870DAE0656F606FC06840681049B1
:10F2D0000860E9688889F8F780F900F0030008B150
:10F2E000012000E0002029890844616A0844606226
:10F2F00000BFE9688889F8F770F900F0030008B1E9
:10F3000001206EE06CE0000096000020DCC60120C9
:10F310008C000020696E7365672E7020213D204EA1
:10F32000554C4C00696E73616E65206F666673653F
:10F33000742100007062756620746F6F2073686FAF
:10F34000727421007463705F726563656976653AF3
:10F35000207365676D656E74206E6F7420747269BA
:10F360006D6D656420636F72726563746C7920746F
:10F370006F207263765F776E640A00007463705F5B
:10F38000726563656976653A207365676D656E744D
:10F39000206E6F74207472696D6D656420636F7286
:10F3A000726563746C7920746F206F6F7365712060
:10F3B00071756575650A00007463705F72656365D9
:10F3C0006976653A207463706C656E203E207263C6
:10F3D000765F776E640A00009C0000209900002090
:10F3E000002029890844218D88420AD900BFAFF244
:10F3F000885340F22B62C2A1AFF24450F4F7E4FB11
:10F4000000BF00BFE9688889F8F7E7F800F003005B
:10F4100008B1012000E0002029890844218D081A44
:10F420002085204601F072FD6868008900280DDD06
:10F43000BD48006828B1BC4869680068F9F7FEFE5D
:10F4400002E0B9496868086000206860E968888956
:10F45000F8F7C3F800F0010050B1B448007840F06C
:10F460002000B2490870207D042801D107202075B2
:10F4700028686067284600F043FE00BF606F30B127
:10F48000606FC0684068616A88423FF41CAF00BF8B
:10F49000A07E00F0010060B100BF608B4FF6FE71EE
:10F4A0000840608300BF00BF608B40F002006083B3
:10F4B00005E000BF608B40F00100608300BF1DE1EC
:10F4C000606F20B99A4800F0C1FD6067FAE000263D
:10F4D000656FF2E0E868406896490968884217D18C
:10F4E000934800892989884211DD914800F0AEFDDA
:10F4F0008246BAF1000F09D016B1C6F800A001E0AB
:10F50000C4F874A029465046FDF718FED8E0D7E0AD
:10F51000A6B9E868406887490968081A0DD5844883
:10F5200000F094FD8246BAF1000F05D0C4F874A033
:10F5300029465046FDF702FEC2E030E0F068406820
:10F54000401C7C490968081A28D4E8684068401EB5
:10F5500078490968081A002820DC754800F076FD13
:10F560008246BAF1000F18D0F0684068318908442B
:10F5700070490968401A002809DDF06880886D49E3
:10F580000988081A308131897068FAF771FAC6F86B
:10F5900000A029465046FDF7D1FD91E000BF2E4660
:10F5A000286800287DD1E868406862490968081A1F
:10F5B000002876DDE9688889F8F70FF800F0010087
:10F5C00000B17DE05A4800F041FD2860286800281D
:10F5D00071D0E86840682989084456490968401A8A
:10F5E000002809DDE868808852490988081A2881BE
:10F5F00029896868FAF73CFA218D606A08444E4907
:10F6000009884C4A12681144081A002853DD2968F9
:10F61000C9688889F7F7E1FF00F0010098B129680F
:10F62000C9688889F7F7D9FF00F03E0A5046F7F716
:10F63000D4FF2968C96889894CF2FF021140084348
:10F640002968C9688881A08C218D084439490988B6
:10F65000401A296808812A6811895068FAF708FA5F
:10F660002968C9688889F7F7B8FF00F0030008B176
:10F67000012000E000202968098908442E490880FB
:10F6800000BF218D606A01442A4800682A4A128816
:10F69000104481420ED000BFAFF634034FF4DF6256
:10F6A00001E009E007E0AFF26431AFF2F470F4F783
:10F6B0008BFA00BF00BF03E02D68002D7FF40AAF76
:10F6C00000BF00BF204600F035FD17E0204600F0E7
:10F6D00031FD13E01749606A0968081A08D4218DC2
:10F6E000606A0844401E13490968081A002805DDAD
:10F6F00000BF608B40F00200608300BFBDE8F09F58
:10F700007463705F726563656976653A206F6F73C5
:10F710006571207463706C656E203E207263765F45
:10F72000776E640A000000009C0000209900002011
:10F73000DCC601208C0000209600002070B5044635
:10F740000D46002C0FD000BF207D012808D100BF3E
:10F7500005A340F2DF7210A119A0F4F735FA00BF3B
:10F7600000BFC4F8845070BD2E2E2F4D6964646CA8
:10F770006577617265732F54686972645F50617256
:10F7800074792F4C7749502F7372632F636F7265B2
:10F790002F7463702E630000696E76616C6964205B
:10F7A000736F636B657420737461746520666F7228
:10F7B00020726563762063616C6C6261636B00002C
:10F7C000417373657274696F6E20222573222066FF
:10F7D00061696C6564206174206C696E65202564C4
:10F7E00020696E2025730A002DE9F04107460D4679
:10F7F00014461E4600BF002D0CD100BF0EA34FF4CF
:10F80000D36219A11FA0F4F7DFF900BF6FF00F005A
:10F81000BDE8F08100BF3CB12189284600F046F8E0
:10F820002046F9F7C9FF04E01EB92846FBF78CFC17
:10F83000EEE70020ECE700002E2E2F4D6964646C8B
:10F840006577617265732F54686972645F50617285
:10F8500074792F4C7749502F7372632F636F7265E1
:10F860002F7463702E6300007463705F726563763B
:10F870005F6E756C6C3A20696E76616C696420709D
:10F8800063620000417373657274696F6E20222594
:10F890007322206661696C6564206174206C696EF6
:10F8A0006520256420696E2025730A002DE9F0414A
:10F8B00004460F4600BF002C0AD100BF1CA340F233
:10F8C000CF3227A12CA0F4F77FF900BFBDE8F0816B
:10F8D00000BF00BF207D012808D100BF14A340F263
:10F8E000D2322FA124A0F4F76FF900BF00BF208D02
:10F8F000384485B2B5F5066F02DC208DA84203DDE1
:10F900004FF40660208500E02585204601F0FEFAD0
:10F910000646B6F5067F08D300BF608B40F00200B4
:10F92000608300BF2046FDF79FFC00BFCEE70000CC
:10F930002E2E2F4D6964646C6577617265732F5448
:10F94000686972645F50617274792F4C7749502FE7
:10F950007372632F636F72652F7463702E63000080
:10F960007463705F7265637665643A20696E766170
:10F970006C69642070636200417373657274696FAF
:10F980006E2022257322206661696C656420617493
:10F99000206C696E6520256420696E2025730A003D
:10F9A000646F6E27742063616C6C207463705F7287
:10F9B000656376656420666F72206C697374656E2A
:10F9C0002D7063627300000070B506460D4600BFDF
:10F9D000002D07D100BF09A3FF2214A11DA0F4F739
:10F9E000F3F800BF00BF344605E0E06FA84201D144
:10F9F0000020E067E468002CF7D170BD2E2E2F4D5B
:10FA00006964646C6577617265732F5468697264A8
:10FA10005F50617274792F4C7749502F7372632F46
:10FA2000636F72652F7463702E6300007463705F80
:10FA300072656D6F76655F6C697374656E65723A39
:10FA400020696E76616C6964206C697374656E659B
:10FA500072000000417373657274696F6E20222515
:10FA60007322206661696C6564206174206C696E24
:10FA70006520256420696E2025730A002DE9F04178
:10FA8000044600BF002C08D100BF20A340F2C16291
:10FA90002BA131A0F4F798F800BF00BF206F18B970
:10FAA0006FF00500BDE8F081256F2846FEF7C4F829
:10FAB00010B16FF00500F5E72868206704F16C06C7
:10FAC00000E03668306858B13168C9684868F7F7AF
:10FAD00077FD0746E9684868F7F772FD381AF0D4F1
:10FAE000306828603560286810B90020A4F86800E4
:10FAF00094F84200FF2804DA94F84200401C84F88D
:10FB000042000020606300BFCCE700002E2E2F4D86
:10FB10006964646C6577617265732F546869726497
:10FB20005F50617274792F4C7749502F7372632F35
:10FB3000636F72652F7463705F6F75742E6300005E
:10FB40007463705F7265786D69743A20696E76616E
:10FB50006C69642070636200417373657274696FCD
:10FB60006E2022257322206661696C6564206174B1
:10FB7000206C696E6520256420696E2025730A005B
:10FB800010B5044600BF002C08D100BF20A340F2EE
:10FB9000F9622CA133A0F4F717F800BF00BF206F63
:10FBA000A0B3A07E00F0040080BB2046FFF766FFF4
:10FBB00060BBB4F84810B4F86020914202DAB4F89F
:10FBC000481001E0B4F86010084601EBD071C1F3B1
:10FBD0004F01A4F84A10B4F84A00618E49008842E7
:10FBE00004D2608E4004000CA4F84A00B4F84A0025
:10FBF000618E032202FB0100A4F8480000BF608B65
:10FC000040F00400608300BF0020208610BD00008B
:10FC10002E2E2F4D6964646C6577617265732F5465
:10FC2000686972645F50617274792F4C7749502F04
:10FC30007372632F636F72652F7463705F6F757477
:10FC40002E6300007463705F7265786D69745F661F
:10FC50006173743A20696E76616C696420706362C6
:10FC600000000000417373657274696F6E20222575
:10FC70007322206661696C6564206174206C696E12
:10FC80006520256420696E2025730A0010B504469E
:10FC900000BF002C08D100BF08A340F2AD6214A140
:10FCA0001AA0F3F791FF00BF00BF204600F09EF8B6
:10FCB00010B9204600F03EF810BD00002E2E2F4D4A
:10FCC0006964646C6577617265732F5468697264E6
:10FCD0005F50617274792F4C7749502F7372632F84
:10FCE000636F72652F7463705F6F75742E630000AD
:10FCF0007463705F7265786D69745F72746F3A20B7
:10FD0000696E76616C69642070636200417373652B
:10FD10007274696F6E2022257322206661696C659A
:10FD200064206174206C696E6520256420696E20F2
:10FD300025730A0010B5044600BF002C08D100BF8F
:10FD40000AA34FF4D36216A11EA0F3F73DFF00BF34
:10FD500000BF94F84200FF2804DA94F84200401CE7
:10FD600084F842002046FDF77FFA10BD2E2E2F4D5D
:10FD70006964646C6577617265732F546869726435
:10FD80005F50617274792F4C7749502F7372632FD3
:10FD9000636F72652F7463705F6F75742E630000FC
:10FDA0007463705F7265786D69745F72746F5F639E
:10FDB0006F6D6D69743A20696E76616C696420704C
:10FDC00063620000417373657274696F6E2022254F
:10FDD0007322206661696C6564206174206C696EB1
:10FDE0006520256420696E2025730A0070B50446DD
:10FDF00000BF002C08D100BF22A340F263622EA1F5
:10FE000036A0F3F7E1FE00BF00BF206F10B96FF01E
:10FE1000050070BD256F07E02846FDF70DFF10B106
:10FE20006FF00500F5E72D6828680028F4D1284612
:10FE3000FDF702FF10B16FF00500EAE7E06E286001
:10FE4000206FE0660020206700BF608B40F40060F8
:10FE5000608300BFE9684868F7F7B2FB0646E968C7
:10FE60008889F7F7BAFB00F0030008B1012000E031
:10FE70000020298908443044E0640020606300BF0A
:10FE8000C7E700002E2E2F4D6964646C65776172A0
:10FE900065732F54686972645F50617274792F4C76
:10FEA0007749502F7372632F636F72652F7463707D
:10FEB0005F6F75742E6300007463705F7265786D98
:10FEC00069745F72746F5F707265706172653A20F9
:10FED000696E76616C69642070636200417373655A
:10FEE0007274696F6E2022257322206661696C65C9
:10FEF00064206174206C696E6520256420696E2021
:10FF000025730A0070B504460E4615462CB1207ABA
:10FF100018B1207AF8F744FB70BD2846F6F762FD69
:10FF2000FAE700002DE9F04F85B083460F46904672
:10FF30001D46DDF8389000BF002D08D100BF1EA37C
:10FF400040F2C47229A130A0F3F73EFE00BF00BF0B
:10FF500000BFB9F1000F08D100BF17A340F2C5726E
:10FF600033A129A0F3F730FE00BF00BF002646F200
:10FF7000080A3846F7F724FB14220490DDE90F0144
:10FF80008DE80704002231464046049BFDF78CFBB8
:10FF9000044614B905B0BDE8F08F3346002221466F
:10FFA0005846FDF791FC4B462A4621465846FDF738
:10FFB0000DFC00BFEEE700002E2E2F4D6964646C2F
:10FFC0006577617265732F54686972645F506172FE
:10FFD00074792F4C7749502F7372632F636F72655A
:10FFE0002F7463705F6F75742E6300007463705FAD
:10FFF0007273743A20696E76616C6964206C6F6309
:020000040801F1
:10000000616C5F6970000000417373657274696FA1
:100010006E2022257322206661696C6564206174FC
:10002000206C696E6520256420696E2025730A00A6
:100030007463705F7273743A20696E76616C696480
:100040002072656D6F74655F6970000070B505465C
:1000500000BF002D08D100BF0CA340F2826217A19F
:100060001DA0F3F7B1FD00BF00BF0320F8F738F87B
:1000700004460CB9002070BD95E80F0084E80F001D
:100080006068F9F7A9FD2046F5E700002E2E2F4DF8
:100090006964646C6577617265732F546869726412
:1000A0005F50617274792F4C7749502F7372632FB0
:1000B000636F72652F7463702E6300007463705FEA
:1000C0007365675F636F70793A20696E76616C69FA
:1000D0006420736567000000417373657274696F13
:1000E0006E2022257322206661696C65642061742C
:1000F000206C696E6520256420696E2025730A00D6
:1001000010B5044644B1606810B16068F9F754FB5B
:1001100021460320F7F716FF10BD70B5044605E031
:1001200025682046FFF7ECFF2C4600BF002CF7D1D6
:1001300070BD00002DE9F04704460025A94600BF28
:10014000002C08D100BF2CA340F2EA7237A13FA0D7
:10015000F3F73AFD00BF00BF05F0010008B104202D
:1001600000E0002005F0020109B1002100E00021BB
:10017000084405F0080109B1002100E0002108440D
:1001800005F0100109B1002100E0002100EB010899
:10019000206DF7F715FA8246534600224146204665
:1001A000FDF714FA06464EB900BF608B40F003001D
:1001B000608300BF6FF00100BDE8F0874B462A4620
:1001C00031462046FDF780FB231D2246314620465E
:1001D000FDF7FCFA07462FB100BF608B40F003002B
:1001E000608306E000BF608B4FF6FC7108406083BF
:1001F00000BF3846E0E700002E2E2F4D6964646C86
:100200006577617265732F54686972645F506172BB
:1002100074792F4C7749502F7372632F636F726517
:100220002F7463705F6F75742E6300007463705F6A
:1002300073656E645F656D7074795F61636B3A209E
:10024000696E76616C6964207063620041737365E6
:100250007274696F6E2022257322206661696C6555
:1002600064206174206C696E6520256420696E20AD
:1002700025730A0070B5044600BF002C08D100BFEA
:1002800016A340F2EB3222A128A0F3F79DFC00BF99
:1002900000BFE06EE8B1E56E00E02D682868002838
:1002A000FBD1E9688889F7F798F900F0070078B979
:1002B0000120F7F792F9E96889890843E96888819C
:1002C00000BF608B40F02000608300BF002070BD45
:1002D00000BF01212046FBF7D1FAF8E72E2E2F4D63
:1002E0006964646C6577617265732F5468697264C0
:1002F0005F50617274792F4C7749502F7372632F5E
:10030000636F72652F7463705F6F75742E63000086
:100310007463705F73656E645F66696E3A20696EC0
:1003200076616C69642070636200000041737365DC
:100330007274696F6E2022257322206661696C6574
:1003400064206174206C696E6520256420696E20CC
:1003500025730A002DE9F04F85B04FF00009E948F8
:100360000068401CE7490860E7480078401CE649FF
:10037000087000BF0025E5480468E3E200BF207D67
:10038000002808D100BFE2A340F2BE42ECA1F7A0D2
:10039000F3F71AFC00BF00BF00BF207D012808D181
:1003A00000BFDBA340F2BF42FAA1F0A0F3F70CFCC0
:1003B00000BF00BF00BF207D0A2808D100BFD4A322
:1003C0004FF49862FEA1E9A0F3F7FEFB00BF00BF67
:1003D000A07FCD490978884202D12546E468B1E280
:1003E000C9480078A0770026B046207D022806D1B3
:1003F00094F84200062802DB701CC6B2D1E094F8E3
:1004000042000C2802DB701CC6B2CAE094F89900C6
:1004100000285DDD00BF206F002808D000BFBCA30E
:1004200040F2D442F2A1D1A0F3F7CEFB00BF00BF4F
:1004300000BFE06E002808D100BFB5A340F2D5424E
:10044000F8A1CAA0F3F7C0FB00BF00BF94F89A0060
:100450000C2802DB701CC6B2A3E094F89900401E81
:10046000FE490F5C94F89800B84204DA94F89800BA
:10047000401C84F8980094F89800B84227DB4FF0AD
:10048000010AB4F8600030B9204601F0B7FA70B143
:100490004FF0000A0BE0B4F86010204600F0F4FAC8
:1004A00028B92046FCF7E0FE08B94FF0000ABAF17F
:1004B000000F0BD0002084F8980094F899000728CA
:1004C00004D294F89900401C84F8990000BF68E0B9
:1004D000B4F93000002809DBB4F9300047F6FF71A9
:1004E000884203DA208E401C00B22086B4F9300026
:1004F000B4F94010884254DB2046FFF777FC18B16E
:10050000206F70BBE06E60B3207D02281ED094F88F
:1005100042200C2A02D294F8422000E00C2211461C
:10052000B4F93E20B4F93C3002EBE302CC4B5B5C07
:1005300002FA03F047F6FF72904201DA024601E048
:1005400047F6FF7212B2A4F8402000BF00202086B8
:10055000B4F84800B4F86010884203DAB4F84800F0
:1005600002E01EE0B4F86000049004984010A4F883
:100570004A00B4F84A00618E4FF6FF7202EA410168
:10058000884205DA608E114601EA4000A4F84A006C
:10059000608EA4F848000020A4F86A002046FFF707
:1005A000C9FB207D06280BD1A07E00F0100038B1D9
:1005B0005449206A0968081A282801D9701CC6B253
:1005C000607A00F00800D0B3207D042802D0207D9E
:1005D000072834D1A349D4F8940008444FF4FA71A1
:1005E000B0FBF1F0474A216A1268511A884206D2DC
:1005F000701CC6B208F1010000F0FF081FE094F87B
:100600009B1042F29F4211FB02F1D4F8940000EBE0
:10061000C1004FF4FA71B0FBF1F03A4A216A126856
:10062000511A88420BD22046FCF7F0F88146B9F106
:10063000000F04D194F89B00401C84F89B00606F6D
:1006400068B13049206A0968081AB4F9401001EB12
:100650004101B0EB410F02D32046FBF703FC207DA4
:10066000032807D12749206A0968081A282801D9D0
:10067000701CC6B2207D092807D12249206A09686A
:10068000081AF02801D9701CC6B2002E37D0D4F851
:1006900090A02046FDF77EFC8DB100BF1B4800688E
:1006A000844208D100BF1AA340F26D526EA12FA060
:1006B000F3F78AFA00BF00BFE068E86011E000BF0E
:1006C00012480068A04208D000BF11A340F2715246
:1006D00070A126A0F3F778FA00BF00BF0B49E068CD
:1006E0000860B8F1000F0BD0208BE18A221DCDE904
:1006F0000021029023462046626A216DE0E0FBE083
:10070000E0E0000060000020760000206C00002087
:100710002E2E2F4D6964646C6577617265732F545A
:10072000686972645F50617274792F4C7749502FF9
:100730007372632F636F72652F7463702E63000092
:100740007463705F736C6F77746D723A2061637459
:10075000697665207063622D3E7374617465202133
:100760003D20434C4F5345440A00000041737365DC
:100770007274696F6E2022257322206661696C6530
:1007800064206174206C696E6520256420696E2088
:1007900025730A007463705F736C6F77746D723ABF
:1007A00020616374697665207063622D3E737461A5
:1007B000746520213D204C495354454E0A000000E9
:1007C0007463705F736C6F77746D723A20616374D9
:1007D000697665207063622D3E73746174652021B3
:1007E0003D2054494D452D574149540A0000000011
:1007F0007463705F736C6F7774696D723A207065A3
:100800007273697374207469636B696E67207769AA
:10081000746820696E2D666C696768742064617401
:10082000610000007463705F736C6F7774696D7240
:100830003A2070657273697374207469636B696EB2
:1008400067207769746820656D7074792073656EB0
:10085000642062756666657200000000F543010859
:10086000E8430108B84C0A007463705F736C6F77DB
:10087000746D723A206D6964646C652074637020D5
:10088000213D207463705F6163746976655F706396
:10089000627300007463705F736C6F77746D723A8B
:1008A00020666972737420706362203D3D2074631A
:1008B000705F6163746976655F70636273000000E6
:1008C000FFF730FBD4F810B0207D03902746E46892
:1008D0003846FBF781F900204849087000BFBAF19B
:1008E000000F03D06FF00C015846D04700BF4348BB
:1008F000007800B13EE524E02546E468287F401CEE
:100900002877287F697F88421BDB002028773B49B6
:10091000087000BFD5F88C0030B12946D5F88C207E
:1009200028699047814601E04FF0000900BF334835
:10093000007800B11EE5B9F1000F02D12846FCF79E
:1009400093FC00BF002C7FF419AD00252C480468EF
:100950004EE000BF207D0A280AD000BFAFF250232E
:1009600040F2A15227A1AFF2FC10F3F72DF900BF1E
:1009700000BF00262F49206A0968081AF02801D90B
:10098000701CC6B2002E31D02046FDF703FB9DB18E
:1009900000BF1B48006884420AD100BFAFF2902319
:1009A00040F2AF5224A1AFF23C20F3F70DF900BFA3
:1009B00000BFE068E86013E000BF11480068A04293
:1009C0000AD000BFAFF2B82340F2B35224A1AFF275
:1009D0006420F3F7F9F800BF00BF0949E068086038
:1009E0002746E4683846FBF7F7F801E02546E46857
:1009F000002CAED105B0BDE8F08F000074000020DF
:100A0000700000207463705F736C6F77746D723A5E
:100A10002054494D452D57414954207063622D3E65
:100A20007374617465203D3D2054494D452D5741F7
:100A300049540000600000207463705F736C6F772E
:100A4000746D723A206D6964646C65207463702003
:100A5000213D207463705F74775F70636273000080
:100A60007463705F736C6F77746D723A206669722D
:100A7000737420706362203D3D207463705F7477EF
:100A80005F706362730000002DE9F04F85B005468A
:100A90000E4600270024A34600BF002D08D100BF4A
:100AA00079A340F24B3285A18DA0F3F78DF800BFFA
:100AB00000BFEC6E24B94FF0FF3005B0BDE8F08FF9
:100AC000002E0CD100BF00BF6FA340F253328EA1A5
:100AD00083A0F3F779F800BF00BFB01FEDE72089CE
:100AE000B04201DC0020E8E700BF688EB04208DABF
:100AF00000BF65A340F25B328CA179A0F3F764F8E4
:100B000000BF00BF00BF2089002808DC00BF5EA333
:100B10004FF4577289A172A0F3F756F800BF00BFD7
:100B200094F80A8008F0010008B1042000E00020D9
:100B300008F0020109B1002100E00021084408F09A
:100B4000080109B1002100E00021084408F010016B
:100B500009B1002100E00021084404902089801B95
:100B60001FFA80FA0498504481B24FF42072362064
:100B7000F8F78CF98346BBF1000F00D16EE0606896
:100B800000892189401A304480B20290DBF8043099
:100B9000049A991860685246029BF8F76DFD50451B
:100BA00000D05BE0E1688889F6F717FD00F03F09A7
:100BB0000020039009F0080028B129F008090398E3
:100BC00040F00800039009F0010028B129F0010964
:100BD000039840F001000390E1684868F6F7F0FCE4
:100BE00030440346CDE9008059462846039AFAF777
:100BF0007DFC074607B931E06068F8F7C7FB35F8B8
:100C0000661F081A288062681289A2EB0A0291B254
:100C10006068F8F72DFF2089A0EB0A002081484684
:100C2000F6F7DBFCE16889890843E1688881606840
:100C3000F8F7ACFB2988084428807868F8F7A6FB09
:100C40002988084425F866092068386027603868D4
:100C500010B90020A5F8680000202EE700BF47B1BA
:100C600000BF09A34FF4767238A11DA0F2F7ACFFC4
:100C700000BF00BFBBF1000F02D05846F8F79CFD43
:100C80004FF0FF3019E700002E2E2F4D6964646C81
:100C90006577617265732F54686972645F50617221
:100CA00074792F4C7749502F7372632F636F72657D
:100CB0002F7463705F6F75742E6300007463705FD0
:100CC00073706C69745F756E73656E745F7365675E
:100CD0003A20696E76616C6964207063620000007E
:100CE000417373657274696F6E20222573222066CA
:100CF00061696C6564206174206C696E652025648F
:100D000020696E2025730A0043616E27742073707A
:100D10006C6974207365676D656E7420696E746F9D
:100D2000206C656E677468203000000073706C6919
:100D300074203C3D206D737300000000757365677F
:100D40002D3E6C656E203E203000000073656720EC
:100D50003D3D204E554C4C0010B50948006868B91F
:100D60000848006810B90848006838B101200449F3
:100D7000086000220549FA20F9F7FEFD10BD0000C9
:100D8000AC0000206C0000207000002095240108B9
:100D90003EB504462948007800F0040000B13EBD8D
:100DA00000BF002C08D100BF25A340F2EE2231A1E4
:100DB00038A0F2F709FF00BF00BF2048007800F01C
:100DC000020018B33D49606A0968081A26D4218DCB
:100DD000606A084439490968081A00281EDC384846
:100DE00000680088364909684988364ACDE90021FB
:100DF000029032480068344909884218314B1B1D63
:100E0000324801682046FFF78DF8C8E70B480078A4
:100E100000F0010010B12E48006820622A480088C6
:100E2000002808DD00BF608B40F00200608300BF37
:100E30002046FCF719FA00BFB1E700009800002037
:100E40002E2E2F4D6964646C6577617265732F5423
:100E5000686972645F50617274792F4C7749502FC2
:100E60007372632F636F72652F7463705F696E2E88
:100E7000630000007463705F74696D657761697405
:100E80005F696E7075743A20696E76616C69642072
:100E900070636200417373657274696F6E202225FE
:100EA0007322206661696C6564206174206C696ED0
:100EB0006520256420696E2025730A008C000020BF
:100EC0007C000020D4C60120960000209000002065
:100ED0006000002010B5FAF731FE06480078401C8B
:100EE000C0B20449087000F0010008B1FFF732FAFF
:100EF00010BD0000750000200348007840F010008D
:100F000001490870704700009900002070B5044640
:100F100000BF002C08D100BF1CA340F2A63227A1BD
:100F20002FA0F2F751FE00BF00BF218D606A451867
:100F3000608EE16AB0F5866F02DD4FF4866000E0F6
:100F4000608E0844281A04D4208D6085E06A281A2F
:100F500070BDE16A606A401A002802DD00206085E9
:100F600012E0616AE06A461A00BFB6F5803F08D316
:100F700000BF06A340F2B63223A119A0F2F724FE67
:100F800000BF00BF668500BF0020E1E72E2E2F4D79
:100F90006964646C6577617265732F546869726403
:100FA0005F50617274792F4C7749502F7372632FA1
:100FB000636F72652F7463702E6300007463705FDB
:100FC0007570646174655F7263765F616E6E5F7782
:100FD0006E643A20696E76616C69642070636200A9
:100FE000417373657274696F6E20222573222066C7
:100FF00061696C6564206174206C696E652025648C
:1010000020696E2025730A006E65775F7263765FD4
:10101000616E6E5F776E64203C3D20307866666658
:10102000660000002DE9FF4F91B004468A4617463E
:101030004FF0000B0025002010900F900E9000261E
:101040000B900A908146099000BF002C0DD100BF83
:10105000E7A34FF4CF72F3A1F8A0F2F7B5FD00BFFC
:101060006FF00F0015B0BDE8F08F00BFB4F862104C
:1010700001EBD1725210638E9A4201DD628E04E060
:10108000B4F8620000EBD072521092B20792079A45
:101090000AB1079800E0608E079000BFBAF1000F18
:1010A0000BD100BFD2A340F2AD12EEA1E3A0F2F744
:1010B0008BFD00BF6FF00F00D4E700BF394620461C
:1010C00000F0C2FB0890089808B10898CAE7B4F885
:1010D00066000D9000200C90E06E00287ED0E56E3A
:1010E00000E02D6828680028FBD1A87A00F00100F4
:1010F00008B1042000E00020A97A01F0020109B142
:10110000002100E000210844A97A01F0080109B19A
:10111000002100E000210844A97A01F0100109B182
:10112000002100E000210844069000BF29890698AC
:1011300001440798814208DD00BFADA34FF4F3726C
:10114000D5A1BEA0F2F740FD00BF00BF29890698D7
:1011500001440798401A1FFA80F8B4F868000A9012
:10116000BDF82800002831DD00BFBDF8280040454B
:1011700008DD00BF9EA34FF4FC72CDA1AFA0F2F733
:1011800023FD00BF00BF1095BDF82800B84202DA69
:10119000BDF8280000E03846404501DD404607E044
:1011A000BDF82800B84202DABDF8280000E0384651
:1011B000814606EB090086B2BDF82800A0EB0900C5
:1011C00080B20A90A8EB09001FFA80F800BFBDF8B2
:1011D000280060B1BE420AD000BF00E079E084A3DD
:1011E0004FF40072BAA195A0F2F7EEFC00BF00BF69
:1011F000BE426DDAB8F1000F6ADD2889002867DD8C
:10120000B81B404501DD404600E0B81B80B20590A8
:101210001095149800F00100E8B1012114980AAB70
:101220004246CDE90040029100200599FCF7F6FD09
:10123000B0F1000B00D18CE20AEB0601DBF80400F0
:10124000059AEFF763F85846F8F7A0F80D990844A7
:1012500080B20D9038E06868049002E0049800685D
:101260000490049800680028F8D10498007B00F0EE
:10127000C000A0B9049841684089084450450ED187
:1012800000BF46B100BF5AA340F2312298A16BA023
:10129000F2F79AFC00BF00BF0598099013E0012205
:1012A00000200599F7F7F2FDB0F1000B00D150E2F4
:1012B0000AEB0600CBF804005846F8F767F80D99DA
:1012C000084480B20D9000BF0598304486B200BF3C
:1012D0000DE000BFB4F8680040B100BF44A340F285
:1012E0004A228EA155A0F2F76FFC00BF00BF7EE13D
:1012F000B81B80B206900C990798401A80B20590EE
:10130000DDE90510884201DA069800E005980490AE
:10131000149800F0010000282FD00E9808B9012180
:1013200000E000211498CDE9004002910C9A049845
:10133000104481B20AAB3620079AFCF76FFDB0F17A
:10134000000800D105E200BFB8F80A1004988142F5
:1013500008DA00BF26A340F266227CA137A0F2F78C
:1013600033FC00BF00BF0AEB0601D8F804300C9A2A
:101370009818049AEEF7CAFF2BE000BFBDF82800CA
:1013800040B100BF1AA340F2712280A12BA0F2F756
:101390001BFC00BF00BF012236200499F7F776FD41
:1013A000039000B9D5E10AEB0601039841604FF4C0
:1013B000207236200C99F7F769FDB0F1000803D1CF
:1013C0000398F8F7F9F9C4E140460399F7F736FFB7
:1013D00000BF4046F7F7DAFF0D99084480B20D9040
:1013E0000D98092803D94046F8F7E6F9B1E1D5E0B0
:1013F0002E2E2F4D6964646C6577617265732F546E
:10140000686972645F50617274792F4C7749502F0C
:101410007372632F636F72652F7463705F6F75747F
:101420002E6300007463705F77726974653A206997
:101430006E76616C6964207063620000417373654D
:101440007274696F6E2022257322206661696C6553
:1014500064206174206C696E6520256420696E20AB
:1014600025730A007463705F77726974653A20614E
:101470007267203D3D204E554C4C202870726F679E
:1014800072616D6D65722076696F6C617465732031
:1014900041504929000000006D73735F6C6F6361F8
:1014A0006C20697320746F6F20736D616C6C000029
:1014B000696E636F6E73697374656E74206F7665A1
:1014C0007273697A652076732E207370616365008C
:1014D000696E636F6E73697374656E74206F766581
:1014E0007273697A652076732E206C656E00000039
:1014F0007463705F77726974653A20524F4D207043
:10150000627566732063616E6E6F74206265206F12
:1015100076657273697A656400000000756E7365A4
:101520006E745F6F76657273697A65206D69736D2D
:101530006174636820287063622D3E756E73656EFA
:1015400074206973204E554C4C2900007463705F01
:1015500077726974653A20636865636B20746861AB
:101560007420666972737420706275662063616EA0
:1015700020686F6C642074686520636F6D706C65A3
:101580007465207365676C656E0000006F76657228
:1015900073697A65203D3D20300000000B98009073
:1015A000E06D8319002241462046F9F79FFF109015
:1015B00000B9CEE00E9810B910980E9011E000BF5F
:1015C0000F9850B900BFAFF2D81340F2AB2275A10B
:1015D000AFF29810F2F7F8FA00BF00BFDDE90F1084
:1015E000086010980F900498304486B200BFBE4245
:1015F000FFF67EAEB9F1000F21DDD5F8048017E0CB
:10160000B8F808004844A8F80800D8F8000068B9FD
:10161000B8F80A20D8F8041088184A465146EEF760
:1016200075FEB8F80A004844A8F80A00D8F8008007
:10163000B8F1000FE4D128894844288100BFBDF8E3
:101640002800A4F86800BBF1000F17D000BF55B9FF
:1016500000BFAFF264234FF4387257A1AFF22420D9
:10166000F2F7B2FA00BF00BF59466868F7F7E6FD27
:101670002889BBF808100844288132E0099800281E
:101680002FDD00BF0DB1686850B900BFAFF2A023D5
:1016900040F2E62256A1AFF25C20F2F795FA00BFC5
:1016A00000BFD5F8048007E0B8F80810099808448E
:1016B000A8F80800D8F80080D8F800000028F3D176
:1016C000B8F8081009980844A8F80800B8F80A10F3
:1016D00009980844A8F80A0029890998084428812B
:1016E00000BF15B90E98E06601E00E98286054F826
:1016F0005C0F384420602089C01B20810D986081D8
:1017000060895C3C80B100BF206F60B9E06E50B969
:1017100000BFAFF2243340F2123243A1AFF2E42013
:10172000F2F752FA00BF00BF109880B11098C0685D
:1017300068B1149800F0020048B90820F5F74DFF91
:101740001099C968898908431099C968888100205F
:1017500088E400BF608B40F08000608300BFBBF175
:10176000000F02D05846F8F727F80E9810B10E98DF
:10177000FEF7D3FCB4F8660080B100BF206F60B9FB
:10178000E06E50B900BFAFF2983340F2273226A185
:10179000AFF25830F2F718FA00BF00BF4FF0FF3039
:1017A00060E40000707265765F73656720213D20FC
:1017B0004E554C4C000000007463705F7772697482
:1017C000653A2063616E6E6F7420636F6E6361743F
:1017D000656E617465207768656E207063622D3E6A
:1017E000756E73656E7420697320656D7074790011
:1017F0007463705F77726974653A20657874656E9A
:1018000073696F6E206F66207265666572656E63C0
:10181000652072657175697265732072656665729F
:10182000656E6365000000007463705F77726974B1
:10183000653A2076616C6964207175657565206C08
:10184000656E67746800000070B504460D4600BF01
:10185000002C08D100BF2EA340F2331239A141A0C1
:10186000F2F7B2F900BF00BF207D04280BD0207D25
:10187000072808D0207D022805D0207D032802D02B
:101880006FF00A0070BD0DB90020FBE7B4F86400EA
:10189000A84208DA00BF608B40F08000608300BF80
:1018A0004FF0FF30EEE7B4F86600092808D300BF18
:1018B000608B40F08000608300BF4FF0FF30E1E7B5
:1018C000B4F86600002810D000BF206F00280BD1AC
:1018D000E06E002808D100BF0DA340F255122BA1E5
:1018E00020A0F2F771F900BF0FE000BF206F10B920
:1018F000E06E002808D000BF05A34FF4AC7232A1FF
:1019000018A0F2F761F900BF00BF0020BAE700009D
:101910002E2E2F4D6964646C6577617265732F5448
:10192000686972645F50617274792F4C7749502FE7
:101930007372632F636F72652F7463705F6F75745A
:101940002E6300007463705F77726974655F63680B
:1019500065636B733A20696E76616C6964207063AD
:1019600062000000417373657274696F6E202225F6
:101970007322206661696C6564206174206C696EF5
:101980006520256420696E2025730A007463705FEA
:1019900077726974653A207062756673206F6E2085
:1019A0007175657565203D3E206174206C656173BD
:1019B00074206F6E65207175657565206E6F6E2D74
:1019C000656D7074790000007463705F777269747C
:1019D000653A206E6F207062756673206F6E20719D
:1019E00075657565203D3E20626F74682071756570
:1019F00075657320656D7074790000002DE9FC5FDA
:101A000004464FF0000A00BF002C08D100BF37A3E6
:101A100040F64F0242A14BA0F2F7D6F800BF00BF3C
:101A2000E56E15B90020BDE8FC9F94F89A00FF28E8
:101A300004DA94F89A00401C84F89A00E9688889CE
:101A4000F5F7CBFD00F0010018B1288908B9012095
:101A500000E000208146B9F1000F01D1012000E033
:101A600000208346E86843685A4651462046FBF703
:101A7000ADFD064616B94FF0FF30D4E77768B9F1EF
:101A8000000F09D01120F5F7A8FDB9894CF2FF022B
:101A900011400843B8810DE0706814300090696807
:101AA00009892A89891A8BB2012268680099F7F797
:101AB000E3FD00BFE9684868F5F782FD00F1010821
:101AC000206DB0EB080001D5C4F8508053460022C9
:101AD00031462046FBF7F8FE231D224631462046BC
:101AE000FBF774FE019001989DE700002E2E2F4D0C
:101AF0006964646C6577617265732F546869726498
:101B00005F50617274792F4C7749502F7372632F35
:101B1000636F72652F7463705F6F75742E6300005E
:101B20007463705F7A65726F5F77696E646F775FF9
:101B300070726F62653A20696E76616C69642070BC
:101B400063620000417373657274696F6E202225B1
:101B50007322206661696C6564206174206C696E13
:101B60006520256420696E2025730A0070B505463E
:101B70000C46164602492046FDF7E0FD002070BDE8
:101B8000ED1C010870B505460C4616460249204674
:101B9000FDF7D4FD002070BD451D010870B5054658
:101BA0000C46164602492046FDF7C8FD002070BDD0
:101BB0009D1D010870B505460C4616460249204693
:101BC000FDF7BCFD002070BDF51D010870B5054690
:101BD0000C46164602492046FDF7B0FD002070BDB8
:101BE0004D1E010870B505460C46164602492046B2
:101BF000FDF7A4FD002070BDA51E010870B50546C7
